:020000040800F2
:1000000000200010613C0308098B020841530008DE
:10001000078B0208058B0208038B02080000000012
:10002000000000000000000000000000018B02083A
:10003000FF8A020800000000FD8A0208314F000814
:10004000C93C0308C93C0308C93C0308C93C030870
:10005000C93C0308C93C0308C93C0308C93C030860
:10006000C93C0308C93C0308C93C0308D521000862
:10007000C5210008B5210008A52100089521000828
:10008000812100086D210008C93C0308C93C030810
:10009000D18C0208C93C0308C93C0308C93C0308C9
:1000A000C93C0308A546000845460008CD4600089F
:1000B000954600088546000875460008C93C0308B7
:1000C000C93C0308C93C0308C93C0308C93C0308F0
:1000D000C93C0308AD51000831510008B550000873
:1000E000C93C0308C93C0308ED8A0208C93C03085F
:1000F00055460008C93C030865460008C93C03088A
:10010000000000000000000000000000C93C0308DF
:1001100039500008BD4F0008A1BA020885BA02088C
:100120005921000845210008312100081D2100083F
:1001300009210008C93C030800000000000000007D
:10014000C93C0308C93C0308C93C0308000000007F
:10015000000000000000000000000000000000009F
:100160000000000000000000C93C0308C93C03086F
:10017000C93C03080000000000000000000000006F
:0801800000000000C93C030867
:100188000378407840EA032010FB01F04FF48071B7
:1001980090FBF1F000F30F0000B27047437800784D
:1001A80040EA032010FB01F04FF4807190FBF1F05E
:1001B80000F30F0000B270472DE9F04F654B664E13
:1001C800B3F80AC03468B3F8048087B04FEA0C2A41
:1001D80005901889B4EB0A0A4FF000024FF00005A9
:1001E80065EB020BA0FB0A4500FB0B55E00940EA52
:1001F80045604FEA084407198E46D8884FEAE5114A
:1002080041EB0208A0FB0A45CDE90278B3F8028069
:1002180000FB0B55200A40EA05604FEAC83410EB92
:1002280004084FEA252141EB02099A89A2FB0A0139
:1002380002FB0B11C20D42EA412212F5FA604FEAA5
:10024800E15343F10001B0F5FA6FCDE9000171F116
:100258000001B4465EDA0524A2FB040104FB031185
:1002680000FB03F402FB0144DDE90267A0FB020185
:1002780021444D104FEA3004361B4FEA900444EAFB
:10028800817467EB05078D10B8EB040869EB050965
:10029800DDE9004531484FF0FF31844275EB01013B
:1002A800CDE9026723DA40F6AC5012184FF000018E
:1002B8004B4102FB03F1A2FB022303EB4103D900EC
:1002C800D000101A41EA527163EB0101341847EB70
:1002D8000105CDE902450B24A2FB040104FB03112F
:1002E80049104FEA3000B8EB000869EB01090AFB36
:1002F8000BF3DDE90001AAFB0AAB0BEB430B4FEA5A
:10030800DA7242EA4B02801A4FEAEB7361EB03019F
:10031800CDE90001DCF80410A1FB082301FB093337
:10032800540D5D1544EAC324DDE90223A21A65EBE6
:1003380003031D46D30B059A43EA454302B11360F4
:10034800BEF1000F02D0009BCEF8003007B0BDE828
:10035800F08F00BFA47A0020181E002024FAFFFFA7
:100368002DE9F74F6A4CDFF8ACE123880091DEF8FD
:100378000810B4F90480C3EB21125B00C3EBE1035E
:10038800B4F9021052435943131308FB03F84FEA18
:10039800A83808EBE12101EB8102B1F5FA3802F146
:1003A80080024FEAE1794FEA222349F1FF39B4F993
:1003B80008200193A8FB08AB08FB09F30BEB430BE0
:1003C800A161D31702FB09F108FB0311A2FB082363
:1003D8000B441F03160347EA1257B4F90A2002FB1D
:1003E8000BF1D3170AFB03130546A2FB0A011944B4
:1003F800020A42EA016292194FEA2123E6887B4108
:10040800003243F50043A2FB060106FB03114A1024
:10041800CB1752EA03016FD0B4F91060B4F90E009B
:10042800F71706FB0BF10AFB0711A6FB0AAB8B4477
:1004380000FB09F6C11708FB0161A0FB0889894484
:10044800DEF80C104FEA4846C1F5801E4FEA4947CE
:1004580047EAD8371AEB060AB4F90C8076464BEB14
:10046800070BF71700264FEACE70F90716EB0A06B6
:100478004FEAC80741EA5E0147EB0B0740F6354EE5
:10048800861B61EB0707A6FB0E010EFB071133F075
:100498000FFAB4F916204E13470B47EAC14702FB7F
:1004A80006FED31707FB03EEA2FB0723734456434C
:1004B80007FB0366A2FB07233344560E46EAC3161E
:1004C8003218B4F914604FEA636747EB01037143CC
:1004D800F71700FB0717A6FB00013944C60C46EACC
:1004E800413692194FEAE147B4F912607B41100A8C
:1004F80040EA0360320112180DB1120A2A60009B0B
:1005080013B11A46019B136003B0BDE8F08F00BF1A
:10051800B87A0020181E0020704770472DE9F04176
:10052800324E334F74893B8AB6F91420B6F902E08B
:10053800B6F90E80B6F920C01B1B34895C43E3135F
:10054800B6F912401A44E4020A2594FBF2F41C445A
:10055800B6F90430F4616543A4F57A6404FB04F247
:1005680004FB0EFE5C43B6F90C30121302FB08F8CC
:100578005A4312144FEAEE2E02EB64340EEBE828CD
:10058800B6F900E0F3887E690234A41008EB8E08FF
:1005980004F5004408FA0CF863434CF2503208F1B1
:1005A8000208DC0BA6EBA80642FA0CF3734353BF10
:1005B8005B00B3FBF4F35B00B3FBF4F31A1202FB2A
:1005C80002F440F6DE3262430A4C12145C4302EB3A
:1005D8002442083502F6CF622D1103EB221300B135
:1005E800036001B10D60BDE8F08100BF807A002092
:1005F800181E002043E3FFFF10B5064C237E0BB9FD
:10060800002010BD04F04CFBE369C01AD0F5FA5085
:10061800F6D410BD181E00204FF480538382704713
:100628004FF480538382704707B5032301AA002142
:100638000DF021F99DF805309DF804001B0243EAEE
:1006480000439DF80600184303B05DF804FB08B5A5
:10065800FFF7EAFF014B586008BD00BF181E0020D5
:1006680008B5FFF7E1FF014B186008BD181E002010
:1006780007B5032301AAF6210DF0FDF89DF8053012
:100688009DF804201B0243EA02439DF80620134309
:10069800054AB2F92020C2F10802D340034A536147
:1006A80003B05DF804FB00BF807A0020181E00200C
:1006B80037B504466A460D460C30032123F000F98D
:1006C800024690B1B4F91A106846FFF759FD288020
:1006D800B4F91E100DF10200FFF752FDA880B4F91D
:1006E8001C1001A8FFF74CFD6880104603B030BD10
:1006F80007B5F7216A4623F0E3F89DF801309DF825
:1007080000100C4A1B0143EA01339DF8021043EA2A
:100718001113D3609DF804309DF803101B0143EAC0
:1007280001339DF8051043EA1113936003B05DF897
:1007380004FB00BF181E002038B504460D46FFF71D
:100748005BFF246808B104F0F7FA054B00221A761B
:1007580049215B7E2A4620460DF016F8012038BD57
:10076800181E002070474FF40063838270474FF4CF
:1007780000638382704790F8203033B1012B03D196
:100788004FF400638382704770474FF4806383821D
:10079800704707B5F62101AA23F0C8F89DF8042090
:1007A8009DF8053043EA0223024A138203B05DF83C
:1007B80004FB00BF181E00200346407F20B1002222
:1007C8005A77DA821A835A83704770470120704734
:1007D800034690F8510028B1002283F851201A8767
:1007E8005A879A877047704770B40468037B2268F9
:1007F800022101FA03F31A4213D042690A495C2024
:1008080000FB02124FF6FE7650685289C5680068F0
:10081800296831402960C168D24392B20A40C26057
:10082800636070BC704700BF9C5E002030B40A4B08
:100838001D7875B1094B002003EBC5051A68998826
:100848005062D4682143D160083323F8040CAB42CA
:10085800F4D130BC704700BFEC620020F062002089
:1008680010B40268047B11680223A340194209D01E
:100878000649406800240C7001684FF6FE74214058
:10088800016053605DF8044B704700BF294D00209C
:10089800F0B4334C00EB800004EB80046468002C57
:1008A8005BD0304E49004FF42040CDB23062A16990
:1008B800090444D460682C4F45F08071384041F4F5
:1008C800903101434FF420406160306203E0411EE3
:1008D800002838D00846A1698F07F8D54FF4204082
:1008E800A262306202E0421E68B31046A269110695
:1008F800F9D562681C4945F0007545F480350A4011
:1009080015434FF420406560306202E0421ED0B1CA
:100918001046A2699207F9D5A362A3694FF4204053
:100928009B06306205D4431E68B11846A3699B062E
:10093800F9D520233062E3610120F0BC7047411EE5
:1009480008B10846B3E7094A138801339BB24FF050
:10095800FF3131621380F0BC70472046F0BC70470D
:1009680018690020181E0020009800FC04260020AA
:10097800002310B52A2204461C211846FFF788FFD9
:1009880002230E221C210020FFF782FF03230F22DF
:100998001C210020FFF77CFF12232B221C210020A2
:1009A800FFF776FF02232C221C210020FFF770FF9F
:1009B80001232D221C210020FFF76AFF002318467F
:1009C8002E221C21FFF764FF05232A221C21002068
:1009D800FFF75EFF4FF48073A38210BD10B50823A4
:1009E80004460F2218210020FFF752FF0E23102281
:1009F80018210020FFF74CFF4FF48053A38210BD4D
:100A080038B5194B1C78054608232D22532194B973
:100A18002046FFF73DFF0A23312253212046FFF7E6
:100A280037FF0A2320462C225321FFF731FF4FF4CA
:100A38008073AB8238BD0020FFF72AFF0A233122DA
:100A480053210020FFF724FF0C232C2253210020E0
:100A5800FFF71EFF9023382253210020FFF718FFCD
:100A68004FF48073AB8238BDA82E002010B58023C8
:100A78002422192104460020FFF70AFF642004F00D
:100A8800B5F99723202219210020FFF701FF0A203A
:100A980004F0ACF91023232219210020FFF7F8FEF7
:100AA800642004F0A3F94FF48053A38210BD2DE90C
:100AB800F04F4FF4807385B043838383C38300F181
:100AC8000C050446322004F091F911220021284631
:100AD8000CF006FF6022012128460CF001FF64207B
:100AE80004F084F902A920460027FFF7E1FD01235D
:100AF800B946B8463E460193012E14BF1122122270
:100B0800002128460CF0ECFE002E0CBF4FF0010B24
:100B18004FF0FF3B4FF00A0A0122022128460CF051
:100B2800DFFE142004F062F902A92046FFF7C0FD99
:100B3800BDF90A20BDF90C00BDF90810224B82420C
:100B48000BFB0299A8BF02468A42A8BF0A469A42EE
:100B580001FB0B880BFB007733DB012004F006FC5C
:100B6800BAF1010AD8D10136022EC5D1174B93FB31
:100B7800F8F893FBF9F97022A3F58423002193FB7D
:100B8800F7F7A4F81A80A4F81C90E78328460CF01D
:100B9800A7FE2022012128460CF0A2FE00223146A1
:100BA80028460CF09DFE642004F020F9019B23B92F
:100BB8004FF480736383A383E383012005B0BDE80A
:100BC800F08F00230193CEE701F0FFFF00D03B0038
:100BD800F0B500F10C0585B004460F4601230DF170
:100BE8000702022128460CF046FE18B900263046B6
:100BF80005B0F0BD9DF80730DB07F7D502AA032141
:100C0800284622F05DFE01230DF10702092128463E
:100C18000CF031FE06460028E8D011220A212846A9
:100C28000CF05EFE9DF8073013F00C0FDED1B4F91E
:100C38001A1002A8FFF7B2FA40423880B4F91C1023
:100C48000DF10A00FFF7AAFA40427880B4F91E10A5
:100C580003A8FFF7A3FA4042B880C8E737B500F108
:100C68000C04054600220A2120460CF039FE142007
:100C780004F0BCF80F220A2120460CF031FE0A20AD
:100C880004F0B4F801AA0323102120460CF0F3FD68
:100C98000A2004F0ABF89DF8043080336B839DF88C
:100CA80005308033AB839DF806308033EB83002218
:100CB8000A2120460CF014FE0A2004F097F80DF1E2
:100CC80003020123022120460CF0D5FD01230DF17A
:100CD8000302092120460CF0CEFD11220A212046EC
:100CE8000CF0FEFD012003B030BD012248210CF0BC
:100CF800F7BD012258210CF0F3BD3122F4210CF08C
:100D0800EFBD054B93F820209201343202F0FC022B
:100D1800F4210CF0E5BD00BF807A00202E22F421DA
:100D28000CF0DEBD38B500F11004054680226B21B9
:100D380020460CF0D5FD642004F058F807226821FD
:100D480020460CF0CDFD642004F050F800226B2101
:100D580020460CF0C5FD642004F048F801226B2100
:100D680020460CF0BDFD0F2004F040F895F84F30F8
:100D7800032B8CBF1A2218221B2120460CF0B0FD31
:100D88000F2004F033F818221C2120460CF0A8FD8F
:100D98000F2004F02BF895F84E201A2120460CF06D
:100DA8009FFD0F2004F022F895F8502019212046C5
:100DB8000CF096FD642004F019F820461022372123
:100DC8000CF08EFD0F2004F011F80F20BDE838401C
:100DD80004F00CB838B500F11004054680226B21E8
:100DE80020460CF07DFD642004F000F82046032224
:100DF8006B210CF075FD95F85020192120460CF058
:100E08006FFD0F2003F0F2FF95F84E2020461A21BF
:100E18000CF066FD204618221B210CF061FD2046CF
:100E280018221C210CF05CFD204602223721BDE867
:100E380038400CF055BDF0B5836983B0054613B151
:100E48001A689B8813856869264F8389C3244FF4E1
:100E58007A734FF0060E6E464FF6FF71013703E0C6
:100E6800013B9BB28B421DD002899207F8D50473CF
:100E78004FF47A7302E0A3B28B4213D00289D207EF
:100E880003F1FF34F7D5027BD2B20EB132700136CE
:100E9800BEF1000F08D00EF1FF3EFF24002FE3D073
:100EA8003C78DBE70CF055FCAB6913B11A689B88FA
:100EB80093619DF805009DF801609DF802109DF86A
:100EC80003409DF804209DF8063041EA062143EAD4
:100ED800002342EA0422012029876A87AB8703B0EE
:100EE800F0BD00BFD85003082DE9F043384E736AAF
:100EF80083B0814613B11A689B88138540F2E933A1
:100F0800344901E0002B5ED00A89013B12F0020F40
:100F18009BB2F7D0304B2F49E8221A7040F2E933E0
:100F280001E0002B4FD00A89013B12F0010F9BB260
:100F3800F7D0294B1B78274C274D6F460DF1060833
:100F480040F2E93301E0002B38D02289013B12F04E
:100F5800020F9BB2F7D000232B7040F2E93300E078
:100F680063B32289013B12F0010F9BB2F8D02878B5
:100F7800C0B207F8010B4745E2D1736A13B11A688A
:100F88009B8893619DF804009DF800509DF801101E
:100F98009DF802409DF803209DF8053041EA05219F
:100FA80043EA002342EA04220120A9F83810A9F8EC
:100FB8003A20A9F83C3003B0BDE8F08320460CF095
:100FC800C8FBC0B2D5E703480CF0C3FBB3E700BFCA
:100FD800181E0020003001400C30014010B50446B6
:100FE80001206269138823F040031B041B0C138043
:100FF80013889BB223F0380343F03003138013881F
:101008009BB243F04003138003F096FE2046FFF79F
:1010180089FEA36913B11A689B881385606940F239
:10102800E93301E0002B4BD00289013B12F0020F9B
:101038009BB2F7D06A23037340F2E93301E0002B37
:101048003ED00289013B12F0010F9BB2F7D0037B1F
:10105800606940F2E93301E0002B34D00289013B9A
:1010680012F0020F9BB2F7D01023037340F2E9335A
:1010780000E043B30289013B12F0010F9BB2F8D0A4
:10108800037BA36913B11A689B889361642003F0FA
:10109800ADFE6269138823F040031B041B0C138008
:1010A800138823F038031B041B0C138013889BB28E
:1010B80043F0400313800120BDE8104003F03CBE1C
:1010C8000CF047FBC4E70CF044FBDAE738B500F155
:1010D80010040546192003F089FE20460022152138
:1010E8000CF0FEFB08B922F0E9F895F84E2016211D
:1010F80042F0180220460CF0F3FB0022172120468C
:101108000CF0EEFB01223D2120460CF0E9FB2046C5
:1011180001223E21BDE838400CF0E2BB10B590F842
:101128004E304E2B1ED05D2B1AD0362B0CBF4F24C1
:101138000F24642003F05AFEF023232268210020A4
:10114800FFF7A6FB08B922F0B9F8052003F04EFE18
:101158002346202268210020BDE81040FFF798BBF5
:10116800CF24E6E78F24E4E710B490E80600047B78
:1011780040690223A3404B6013685DF8044B4FF6A7
:10118800FE710B40136004F04BB808B50CF030FB4F
:101198000A2003F0D1FD012008BDF8B50F4D4668BF
:1011A8006A761446027A0F4642F0800225213046BC
:1011B800FFF7EBFF3A4626213046FFF7E6FF04F03B
:1011C8000F0242F0800227213046FFF7DEFF03F0CE
:1011D80067FDE86101202876F8BD00BF181E0020D1
:1011E80070B50478032C0E46154603D0BDE8704050
:1011F8000CF076BB4468027A25212046FFF7C5FF2C
:10120800324626212046FFF7C0FF2A4663212046A2
:10121800FFF7BBFF812227212046FFF7B6FF0120F9
:1012280070BD2DE9F0410478032C884617461E4608
:1012380021D14468027A252142F080022046FFF736
:10124800A4FF424626212046FFF79FFF06F00F0223
:1012580042F0800227212046FFF797FF042003F081
:10126800C5FD72B6492133463A4620460CF08CFA41
:1012780062B6BDE8F081BDE8F0410CF0FCBA37B5C4
:1012880000F10C04054600220A212046FFF7A8FFBA
:101298000F220A212046FFF7A3FF01AA03231021EA
:1012A8002046FFF7BEFF9DF8043080336B839DF81E
:1012B80005308033AB839DF806308033EB83002202
:1012C8000A212046FFF78CFF0DF1030201230221BA
:1012D8002046FFF7A6FF01230DF10302092120464E
:1012E800FFF79FFF11220A212046FFF779FF01200F
:1012F80003B030BD2DE9FF47037B0546884600F162
:101308000C061BB1022B06D9032B3DD00024204626
:1013180004B0BDE8F08701230DF107020221304631
:10132800FFF77FFF0028F1D09DF80730D907EDD5EA
:10133800072302AA03213046FFF773FF0446002C57
:10134800E4D09DF80E7011220A213046FFF748FFBD
:101358003B07DBD4B5F91A1002A8FEF71FFF40427D
:10136800A8F80000B5F91C100DF10A00FEF716FFE9
:101378004042A8F80200B5F91E1003A8FEF70EFFB8
:101388004042A8F80400C2E7234F4FF0010A0024A6
:10139800B94697F82830012B1BD00FD3022BCED19A
:1013A800FFF72AF981460028B0D102A905F11000FB
:1013B800FFF7C2F987F828900446C0E73B7E23B9B7
:1013C800012202213046FFF7E8FE012389F8283080
:1013D8009CE7FFF711F9002898D102A905F1100040
:1013E800FFF7AAF99DF80830044608B1DA0707D4D0
:1013F800002389F82830BAF1000F87D09A46C8E749
:101408003B7E23B9072203213046FFF7C6FE02239D
:1014180089F828307AE700BF181E002008B540F286
:10142800E93300E09BB10289013B12F0020F9BB245
:10143800F8D0017340F2E93300E043B10289013B7F
:1014480012F0010F9BB2F8D0007BC0B208BD0CF0BF
:1014580080F9C0B208BD38B504460D4600BF8068A3
:101468000CF01DF929466068FFF7D8FFA0680CF05A
:101478001BF900BF38BD2DE9F04F87B08368019094
:101488000391934613B11A689B881385012003F0D2
:1014980053FC019C03996068FFF7C0FF606840F245
:1014A800E93302E0002B00F02A820289013B12F0A6
:1014B800020F9BB2F6D080F80CB040F2E93302E09C
:1014C800002B00F01C820289013B12F0010F9BB235
:1014D800F6D0037B019B9B6813B11A689B889361C4
:1014E800012003F029FC642003F026FC039B824DB5
:1014F800DFF81482DFF81492804C814E43F08003A9
:10150800029315230593019B9B6813B11A689B8866
:10151800138503F0C5FB4FF0100C82464FF47A7E1A
:101528000120D9F80430C3F30803002B40F06F8181
:10153800EFF31183002B40F06A812B68A16800BF8C
:101548002A689342F9D1D8F800700EFB07F2521AB4
:10155800B2FBF7F20EFB03239A45E2D0019B5868D1
:1015680040F2E93302E0002B00F0BC810289013B24
:1015780012F0020F9BB2F6D09DF80830037340F2C8
:10158800E93302E0002B00F0AD810289013B12F043
:10159800010F9BB2F6D0037B019B5868838940F208
:1015A800E93302E0002B00F09A810289013B12F036
:1015B800020F9BB2F6D0FF23037340F2E93302E037
:1015C800002B00F08C810289013B12F0010F9BB2C5
:1015D800F6D0037BDBB20493019B9B6813B11A68B6
:1015E8009B88936103F05CFB4FF0100C82464FF42C
:1015F8007A7E0120D9F80430C3F30803002B40F0A9
:10160800EC80EFF31183002B40F0E7802B68A16892
:1016180000BF2A689342F9D1D8F800700EFB07F290
:10162800521AB2FBF7F20EFB03239A45E2D0049A52
:10163800934500F06081334B324ADB880133D38015
:10164800019B9B6813B11A689B88138503F028FBDC
:101658004FF0100C82464FF47A7E0120D9F80430FE
:10166800C3F30803002B40F02081EFF31183002B14
:1016780040F01B812B68A16800BF2A689342F9D10A
:10168800D8F800700EFB07F2521AB2FBF7F20EFB05
:1016980003239A45E2D0019B586840F2E93302E0FF
:1016A800002B00F022810289013B12F0020F9BB24D
:1016B800F6D09DF80C30037340F2E93302E0002BBA
:1016C80000F013810289013B12F0010F9BB2F6D0A2
:1016D800037B019B586840F2E93302E0002B00F0DD
:1016E80007810289013B12F0020F9BB2F6D080F805
:1016F8000CB040F2E9330EE07869002010E000E019
:1017080074690020583600207C69002000ED00E054
:10171800002B00F0ED800289013B12F0010F9BB213
:10172800F6D0037B019B9B6813B11A689B88936171
:1017380003F0B6FA4FF0100C82464FF47A7E01207F
:10174800D9F80430C3F30803002B40F09480EFF37A
:101758001183002B40F08F802B68A16800BF2A6896
:101768009342F9D1D8F800700EFB07F2521AB2FB77
:10177800F7F20EFB03239A45E2D003F091FA4FF0FB
:10178800100C82464FF47A7E0120D9F80430C3F356
:101798000803002B55D1EFF31183002B51D12B688F
:1017A800A16800BF2A689342F9D1D8F800700EFBEF
:1017B80007F2521AB2FBF7F20EFB0323A3EB0A035C
:1017C800632BE2D9059B013B13F0FF0305937FF4DC
:1017D8009AAE184607B0BDE8F08FEFF311818CF38D
:1017E8001288A7682368DA0344BF3060A7682B68AB
:1017F8003268C9B281F31188D8F800101A440EFB78
:1018080001F3DB1BB3FBF1F30EFB02330DE7EFF340
:1018180011818CF31288A7682368DB0344BF30600A
:10182800A7682B683268C9B281F31188D8F800100C
:101838001A440EFB01F3DB1BB3FBF1F30EFB02337F
:101848008AE6EFF311818CF31288A7682368DB031B
:1018580044BF3060A7682B683268C9B281F3118829
:10186800D8F800101A440EFB01F3DB1BB3FBF1F3AD
:101878000EFB0233A2E7EFF311818CF31288A768FD
:101888002368DA0344BF3060A7682B683268C9B29E
:1018980081F31188D8F800101A440EFB01F3DB1B02
:1018A800B3FBF1F30EFB023365E7EFF311818CF321
:1018B8001288A7682368DB0344BF3060A7682B68D9
:1018C8003268C9B281F31188D8F800101A440EFBA7
:1018D80001F3DB1BB3FBF1F30EFB0233D9E60BF08C
:1018E80038FF79E60BF035FF56E60BF032FFF0E6ED
:1018F8000BF02FFF16E7012007B0BDE8F08F0BF0C3
:1019080028FFE7E570B5624C624E2068624DA4F589
:1019180006721C2382F81E3200F138439B0A00210C
:10192800F35C82F81F1203F01F065B090121022BEA
:1019380082B06C6201FA06F163D0032B66D0012BEA
:101948005AD0B2F81C320093694640F20133019331
:1019580024F0DAFC6E6A002E5DD032684F4CB188F4
:101968009161238823F040031B041B0C23802388E8
:101978009BB223F0380343F00803238023889BB2EB
:1019880043F040032380204611852421FFF746FDBC
:1019980020468021FFF742FD3368B2889A616420AF
:1019A80003F0CAF96C6A002C56D02368A2881A85FD
:1019B80020213A48FFF732FDAF213848FFF72EFDC6
:1019C8002368A2889A61012003F0B6F96C6A002C9A
:1019D80050D02368A2881A8523213048FFF71EFDBE
:1019E80060212E48FFF71AFD2368A2889A616420B7
:1019F80003F0FCF902B070BD294B5C6921435961C1
:101A08009FE7274B9C69214399619AE7244BDC693E
:101A18002143D96195E7214C238823F040031B0417
:101A28001B0C238023889BB223F0380343F0080360
:101A3800238023889BB243F040032380204624213F
:101A4800FFF7ECFC20468021FFF7E8FC642003F058
:101A580073F96C6A002CA8D120211048FFF7DEFC2E
:101A6800AF210E48FFF7DAFC012003F065F96C6A34
:101A7800002CAED123210948FFF7D0FC602107488C
:101A8800FFF7CCFC642003F0B1F902B070BD00BFD1
:101A9800445B0020CC730308181E0020003001406E
:101AA80000100240F8B584894FF6FF764FF47A7437
:101AB8002BB311B30F78013101E0B44217D0058977
:101AC800013CAD07A4B2F8D507734FF47A7402E06D
:101AD800BCB2B4420BD00589ED0704F1FF37F7D546
:101AE800057BEDB20AB115700132013BE0E70BF05E
:101AF80030FE003018BF0120F8BDFF27DFE70120C6
:101B0800F8BD038823F040031B041B0C03800388E3
:101B180023F038031B041B0C59B141F480710029D0
:101B280091FAA1F2B2FA82F108BF4FF0FF31013900
:101B3800C900194389B2018003889BB243F040036E
:101B480003807047B0F1FF3F0AD0022810B403DCCD
:101B58005DF8044BFEF79CBE00205DF8044B70470F
:101B680000207047F0B55B4B5B4A97B0196891420B
:101B780000AF00F0A3805949594A00234FF4700080
:101B8800C1F888003B607B60136843F480331360BE
:101B980003E03B68B3F5A04F09D0136803F40033A2
:101BA8007B603B6801333B607B68002BF1D04C4B7A
:101BB8001B6813F4003318BF01237B607B68012B7B
:101BC80052D0464C464B474AE260474A596A116030
:101BD8005A6A42F080725A625A6942F4FC025A61A7
:101BE8000025032207F10801012341F6FF764FF093
:101BF8009040FD60BE603A73BB7324F085FB4FF6DE
:101C0800FF7307F108013948BB6024F07DFB07F139
:101C180008013748374E24F077FB07F108013648AA
:101C280024F072FB07F10801344824F06DFB07F13A
:101C38000801334824F068FB07F1080024F0BEFBD4
:101C4800BB683049304AA1FB031330499B0CF02094
:101C58004FF0070E5C370B60566084F823009560E0
:101C6800C2F800E0BD46F0BD294A1D4B12211160A3
:101C78005A685A605A685A605A6842F480625A60D0
:101C88005A6822F47C125A605A6842F4E8125A6080
:101C98001A6842F080721A601A689201FCD5596875
:101CA8000F4A21F003015960596841F00201596057
:101CB800536803F00C03082BFAD182E700221A605C
:101CC80062B6144B1B6883F30888134B1B6898474C
:101CD800FEE700BFFC9F0020EFBEADDE00ED00E098
:101CE800001002400005FA05886C00200004004836
:101CF800000800483F190100000C00480010004887
:101D08000014004883DE1B4310E000E07C690020DB
:101D18000020024000D8FF1F04D8FF1F70B50F4CE9
:101D28000F4DC0EBC00004EB80046869266930439E
:101D3800686182B09209667BA1600025012101A833
:101D480063618DF804608DF805208DF806508DF8D4
:101D5800071024F0A3FA02B070BD00BFC81A002013
:101D680000100240074BC0EBC00030B403EB80000A
:101D7800054C056963692B4363610176427630BC83
:101D8800704700BFC81A0020001002402DE9F04F2C
:101D98005E4C54F8204083B0002C71D0A66D984654
:101DA80091465B4B72682265A160236004F15E0175
:101DB8004FF4807304F5AF726161A261E36023613F
:101DC8000746307E2CF07CFEF068A8B1514B00210C
:101DD8005A68904203F11C0300F0928001310C29EB
:101DE800F6D100207A1CD2B20C21FFF7BBFF236D7D
:101DF800F26862632433E364B068D8B1454B0021CC
:101E08005A68904203F11C0378D001310C29F7D1AC
:101E180000257A1CD2B20B212846FFF7A3FF2346E0
:101E2800F27E3D492846FFF779FF236DB268A26329
:101E38002833A36494F85D000AF0E1FF054694F89E
:101E48005C000AF0DCFF18F0080F824696F819B01B
:101E58001AD0CDB118F0110F4FF00B0307F101079D
:101E680014BF4E213E21EF715A46AB7128460BF044
:101E780089F818F0010F45D0636B5BB3A36B4BB3C4
:101E8800204603B0BDE8F08F18F0010F0CBF4FF0EB
:101E98002E084FF04E0819F0020F09D045B10B2259
:101EA8007B1CAA71EB7128465A4641460BF06AF82A
:101EB80019F0010FE0D0BAF1000FDDD001370C2383
:101EC8008AF807705A4641468AF8063050460BF0A1
:101ED80059F8D1E7337FB27E8DF804209B090021A1
:101EE800012201A88DF805308DF806108DF807201D
:101EF80024F0D4F9204603B0BDE8F08FCDB288E7CE
:101F0800C8B26FE728460BF0CAFBB5E728470020A0
:101F1800E0500308C81A00207111000800B9704782
:101F2800F0B595B005462DF04FF86C4EC3680268C1
:101F380032600446002B00F0C38028460AF05FFF99
:101F4800674BD86218B1292200238271C371227AA3
:101F5800644D2E210BF016F8306802F031FD2CF09C
:101F6800AFFD3068604A038823F001031B041B0C93
:101F7800038014A91E232B8001270F23002513801B
:101F880021F84C7D2D230293ADF80C50ADF8065086
:101F9800ADF80E502CF0C6FFE379ADF8145060226E
:101FA8009907ADF816500695ADF81C50ADF81E50BF
:101FB800ADF82050ADF82250049200F1838013F060
:101FC800010F0CBF002202224FF48073ADF8147089
:101FD800ADF81C20ADF82030002304AA61793068E0
:101FE800069302F02FF961793068404F2CF07AFFA0
:101FF80033685A6C42F400425A641A8892B242F02A
:1020080080021A80E2796079196A92074CBF04222B
:102018000122824021EA02011962196A0A431A62FE
:102028001A8892B242F001021A80207C00222921EB
:10203800FFF798FE2E49207C00236022FFF76EFEF2
:10204800E068386024F096F8386803684FF6FE7246
:102058001340036024F08EF809A824F05DF8336873
:102068006279244938680A913433134409938022E9
:102078001023002509A940F22A3E0E920B934FF433
:1020880000724FF400530D951095139511950F920A
:102098001293ADF830E024F04DF8627933680C2AD9
:1020A80098BF1549D86898BF31F812503A68134953
:1020B8000543DD601368012043F0020313600870D4
:1020C80015B0F0BD13F0010F0CBF2A4608220423F7
:1020D800ADF81E20ADF816307EE700BFB4640020CE
:1020E800181E0020AA640020A8640020B064002004
:1020F80069080008CC4E0020E4730308AC64002093
:102108000348D0F83C3113B100F59A70184770476E
:10211800C81A00200348D0F8203113B100F58C709C
:1021280018477047C81A00200348D0F804310BB18B
:10213800FC301847704700BFC81A00200348D0F881
:10214800E8300BB1E0301847704700BFC81A0020CC
:102158000348D0F8CC300BB1C4301847704700BFE3
:10216800C81A00200348D0F8B0300BB1A83018477F
:10217800704700BFC81A00200348D0F894300BB14C
:102188008C301847704700BFC81A00200248836F78
:102198000BB1703018477047C81A00200248C36D49
:1021A8000BB1543018477047C81A00200248036C16
:1021B8000BB1383018477047C81A00200248436AE4
:1021C8000BB11C3018477047C81A002002488368B2
:1021D80003B11847704700BFC81A0020F8B5574C1C
:1021E8000601A7190546387A2CF06AFC3B7A03F0F9
:1021F8001F015B090122022B02FA01F278D0032B9E
:1022080071D0012B67D0A319013518790AF0F7FDB1
:10221800EDB2074610B11223C5718371A31958791D
:102228000AF0EDFD10B11323C5718371A3199879D4
:102238000AF0E5FD10B11423C5718371A5190E21AB
:10224800EA7938460AF09EFE68790AF0D8FDEA79FC
:102258000E210AF097FEA8790AF0D1FDEA790E213D
:102268000AF090FEA359364A934251D0354A934218
:1022780059D0354A934240D03444227B002A2FD18A
:10228800012002249A8822F480521204120C9A80A7
:10229800998889B241F4805199801A8802F4415290
:1022A80042F44572024322431A809A8822F47062EB
:1022B8001204120C42F4E0629A809A8B22F40062B3
:1022C8001204120C07219A8319821A8892B242F0DA
:1022D80040021A80F8BD1D4B996A0A439A6292E738
:1022E80000200446CEE7194B19690A431A618AE7A8
:1022F800164BD9680A43DA6085E702F5EA321169B4
:1023080041F400411161116921F400411161B3E701
:1023180002F56042D16841F48051D160D16821F45E
:102328008051D160A8E702F5EC32116941F480418F
:102338001161116921F4804111619DE79C550020CC
:102348000030014000380040003C004000100240CE
:10235800F0B53E4C059D00EB800004EB80046468FA
:10236800002C71D03A4E49004FF42040CFB2306271
:10237800A169090454D46068DFF8E0E047F49031BB
:1023880000EA0E0001434FF420406160306203E030
:10239800411E002848D00846A1698907F8D54FF49E
:1023A8002040A262306203E0421E00283CD0104662
:1023B800A2695206F8D5274A6168DFF8A0E03062C2
:1023C80042EA0342174301EA0E0217436760C3B1AA
:1023D800013BDBB201332B44A0694FF4204210F0DB
:1023E800040002F1FF3207D1511C26D0A06910F079
:1023F800040002F1FF32F7D0626A05F8012B9D4212
:10240800EAD14FF42040306202E0431E60B1184622
:10241800A3699B06F9D520233062E3610120F0BD52
:10242800411E08B10846A3E70B4A138801339BB243
:102438004FF0FF3113803162F0BD074932620B88DB
:1024480001339BB20B80F0BD2046F0BD1869002017
:10245800181E00200024000204260020009800FC1A
:102468002DE9F04F344E96F8303089B00446002BF1
:1024780000F060834369314A934200F04883A2F533
:102488007842934200F03C831A8822F040021204FA
:10249800120C1A801A8822F038021204120C1A80C0
:1024A8001A8892B242F040021A80227C012A00F077
:1024B8001183022A3DD1A26912B1116892880A8556
:1024C8001846C321FEF7AAFF062306AA0021606961
:1024D800FFF7E8FAA36913B11A689B8893619DF81E
:1024E8001A709DF81B209DF818609DF819009DF83A
:1024F8001C509DF81D10636942EA072212B240EA97
:10250800062041EA052162872087A18752B201325D
:1025180003D194F93820013212D0084A934200F0CE
:10252800D182A2F57842934200F0C48209B0BDE896
:10253800F08FB4F93A20E9E7181E00200030014076
:10254800AD4A934200F0B382A2F57842934200F07C
:10255800A7820A23A94DAA4FAA4CAB4E0593322055
:10256800DFF8BC922CF044FF4FF4FA7A4FF0100CCD
:102578004FF47A70D9F80430C3F30803002B40F005
:10258800E681EFF31183002B40F0E1812968A2680E
:1025980000BF2B689942F9D1D7F800E000FB0EF391
:1025A8009B1AB3FBFEF300FB01314FF0010E0391C0
:1025B800D9F80430C3F30803002B40F07481EFF31B
:1025C8001183002B40F06F812B68A16800BF2A6837
:1025D8009342F9D1D7F800B000FB0BF2521AB2FBC4
:1025E800FBF200FB0323039A9B1AB3F57A7FDFD330
:1025F800BAF1010ABED1854B1978854BC1F3400168
:1026080058680BF056F8814B1978814BC943186804
:1026180001F001010BF04DF8072304937C4B5B6834
:1026280033B11A689B88918A0B4218BF1B049361C7
:10263800774B1B6833B11A689B88918A0B4218BF85
:102648001B049361734B1B88002B40F0D781724A9F
:10265800724B117818680BF02CF8DFF8C4914FF022
:10266800FA0A4FF0100C4FF47A70D9F80430C3F31B
:102678000803002B40F0A581EFF31183002B40F0F5
:10268800A0812968A26800BF2B689942F9D1D7F8C0
:1026980000E000FB0EF39B1AB3FBFEF300FB0131D5
:1026A8004FF0010E0391D9F80430C3F30803002B4F
:1026B80040F03181EFF31183002B40F02C812B681F
:1026C800A16800BF2A689342F9D1D7F800B000FB8F
:1026D8000BF2521AB2FBFBF200FB0323039A9B1A7C
:1026E800B3F57A7FDFD3BAF1010ABED1484B5B68F4
:1026F80033B11A689B88918A0B4218BF1B049361F7
:10270800434B1B6833B11A689B88918A0B4218BFE8
:102718001B0493613F4B1B88002B40F07E813E4A8F
:102728003E4B1178186881F001010AF0C2FFDFF80A
:10273800F0904FF0FA0A4FF0100C4FF47A70D9F875
:102748000430C3F30803002B40F01E81EFF311831C
:10275800002B40F019812968A26800BF2B689942B4
:10276800F9D1D7F800E000FB0EF39B1AB3FBFEF398
:1027780000FB01314FF0010E0391D9F80430C3F387
:102788000803002B40F0AB80EFF31183002B40F0DF
:10279800A6802B68A16800BF2A689342F9D1D7F8B0
:1027A80000B000FB0BF2521AB2FBFBF200FB032352
:1027B800039A9B1AB3F57A7FDFD3BAF1010ABED127
:1027C800049B013B13F0FF0304937FF427AF4FF4FE
:1027D8007A7ADFF84C9050464FF0100CD9F8043054
:1027E800C3F30803002B40F03E81EFF31183002B65
:1027F80040F0398116E000BF0030014078690020C0
:102808007C69002010E000E0746900204069002025
:102818004469002050690020526900205469002052
:1028280000ED00E02968A26800BF2B689942F9D141
:10283800D7F800E000FB0EF39B1AB3FBFEF300FB96
:1028480001314FF0010E0391D9F80430C3F30803A6
:10285800002B40F0EC80EFF31183002B40F0E78071
:102868002B68A16800BF2A689342F9D1D7F800B055
:1028780000FB0BF2521AB2FBFBF200FB0323039A94
:102888009B1AB3F57A7FDFD3BAF1010AA6D1059B6B
:10289800013B05937FF463AE9E499F4B9F48A04A36
:1028A8000860DA6042E6EFF311888CF31288A168B9
:1028B8002368DB0344BFC6F800E0A1682B683268D0
:1028C8005FFA88F888F31188D7F800801A4400FB6B
:1028D80008F35B1AB3FBF8F300FB023383E6EFF36C
:1028E80011888CF31288A1682368DB0344BFC6F8FB
:1028F80000E0A1682B6832685FFA88F888F31188CD
:10290800D7F800801A4400FB08F35B1AB3FBF8F30E
:1029180000FB02334CE7EFF311888CF31288A168AF
:102928002368DB0344BFC6F800E0A1682B6832685F
:102938005FFA88F888F31188D7F800801A4400FBFA
:1029480008F35B1AB3FBF8F300FB0233C6E6EFF3B8
:1029580011828CF31288D4F808E02368D90303D5D0
:1029680001233360D4F808E02B683168D2B282F3CF
:1029780011883A68194400FB02F3A3EB0E03B3FB7A
:10298800F2F300FB013110E6EFF311828CF31288A9
:10299800D4F808E02368D90303D501233360D4F8B9
:1029A80008E02B683168D2B282F311883A6819447A
:1029B80000FB02F3A3EB0E03B3FBF2F300FB0131C0
:1029C800D8E6EFF311828CF31288D4F808E0236874
:1029D800D90303D501233360D4F808E02B683168A4
:1029E800D2B282F311883A68194400FB02F3A3EBD0
:1029F8000E03B3FBF2F300FB013151E6494B5A6970
:102A0800002A3FF42AAE484A19681088474A92FBC0
:102A1800F0F201200A6058741FE6424B5A69002AF6
:102A28003FF485AE196800220A605A747FE6EFF316
:102A380011888CF31288A1682368DB0344BFC6F8A9
:102A480000E0A1682B6832685FFA88F888F311887B
:102A5800D7F800801A4400FB08F35B1AB3FBF8F3BD
:102A680000FB02330BE7EFF311828CF31288D4F8E2
:102A780008E02368D90303D501233360D4F808E0BC
:102A88002B683168D2B282F311883A68194400FB86
:102A980002F3A3EB0E03B3FBF2F300FB0131D0E624
:102AA800234A012302EB03120023538151E500233B
:102AB8001F4AF7E71E4A538B9BB2002B3FF436ADF3
:102AC8000123EFE71A4A53899BB2002B3FF42EAD3E
:102AD8000023E7E794F91400617D451C3FF429AD14
:102AE80002283FF726AD06AB009343220623FFF7E3
:102AF8002FFC00287FF4F3ACB4F93A20636905E5AC
:102B080001210B4A02EB011200215181BCE4002192
:102B1800F7E700BFFC9F002000ED00E0EFBEADDE50
:102B28000400FA05586900207069002020A10700F8
:102B38009C5500204269138823F040031B041B0C9A
:102B4800138013889BB223F0380343F038031380B3
:102B580013889BB243F040031380836900F110058A
:102B680013B11A689B881385012002F0E5F86B21E0
:102B78006069FEF753FC80216069FEF74FFCA3698A
:102B880013B11A689B889361012002F0D5F83220AE
:102B980002F02CF901226B212846FEF76CFC94F810
:102BA8004F30042B34BF18221A221B212846FEF767
:102BB80062FC94F84E30042B2DD0032B94BF0722CF
:102BC80000221A212846FEF756FC94F850201921B5
:102BD8002846FEF750FC10221C212846FEF74BFC25
:102BE800122237212846FEF746FC63691A8822F02C
:102BF80040021204120C1A801A8822F038021204B9
:102C0800120C1A801A8892B242F0400201211A80EE
:102C180086F830102FE401221A212846FEF72BFCF3
:102C2800D3E72DE9F04FA44D95F8313085B004462F
:102C3800002B00F070816069038823F040031B04B7
:102C48001B0C038003889BB223F0380343F038033E
:102C5800038003889BB243F040030380A36994F880
:102C68004E5013B11A689B88138540F2E93302E08D
:102C7800002B00F03D820289013B12F0020F9BB24B
:102C8800F6D01A23037340F2E93302E0002B00F078
:102C98002F820289013B12F0010F9BB2F6D0037B11
:102CA800606940F2E93302E0002B00F01E820289DD
:102CB800013B12F0020F9BB2F6D0057340F2E933E4
:102CC80002E0002B00F011820289013B12F0010F93
:102CD8009BB2F6D0037BA36913B11A689B889361F2
:102CE800012002F029F86069038823F040031B04DF
:102CF8001B0C0380038823F038031B041B0C038080
:102D080003889BB243F040030380237C012B00F02F
:102D1800E980022B40F0F680A36913B11A689B88FA
:102D28001385C321FEF77AFB062302AA00216069F6
:102D3800FEF7B8FEA36913B11A689B8893619DF8E2
:102D48000A609DF80B309DF808509DF809109DF811
:102D58000C009DF80D2043EA06231BB263875BB283
:102D680041EA052142EA002201332187A28740F087
:102D7800CF8094F93830013340F0CA80DFF85CA185
:102D88004E4DDFF85C814E4F4FF00A0932202CF08F
:102D98002FFB4FF4FA7601F083FF044601F080FF21
:102DA800001BB0F57A7FF9D3013EF4D19AF80010F0
:102DB8006868C1F340010AF07CFC9AF800102868A2
:102DC800C94301F001010AF074FC07266B6833B1AE
:102DD8001A689B88918A0B4218BF1B0493612B6861
:102DE80033B11A689B88918A0B4218BF1B04936100
:102DF800B8F80030002B40F08781324B324A18680F
:102E080011780AF056FC4FF0FA0B01F049FF04461E
:102E180001F046FF001BB0F57A7FF9D3BBF1010B37
:102E2800F3D16B6833B11A689B88918A0B4218BF3B
:102E38001B0493612B6833B11A689B88918A0B42F3
:102E480018BF1B049361B8F80030002B40F0538181
:102E58001D4B19781B4B81F0010118680AF029FCF9
:102E68004FF0FA0B01F01CFF044601F019FF001B9C
:102E7800B0F57A7FF9D3BBF1010BF3D1013E16F01F
:102E8800FF06A3D14FF47A7601F00AFF044601F059
:102E980007FF001BB0F57A7FF9D3013EF4D1B9F1F1
:102EA80001097FF473AF0949094B0A480A4A0860C7
:102EB800DA6005B0BDE8F08F181E002044690020D4
:102EC800586900205469002052690020FC9F0020A6
:102ED80000ED00E0EFBEADDE0400FA054069002019
:102EE8005069002094F91400431C0BD0022809DC17
:102EF80002AB617D009343220623FFF729FA0028DD
:102F08007FF41DAFB4F93A305BB201333FF431AF0F
:102F180005B0BDE8F08F4069038823F040031B0427
:102F28001B0C038003889BB223F0380343F038035B
:102F3800038003889BB243F040030380A36913B165
:102F48001A689B8813856B21FEF768FA80216069EF
:102F5800FEF764FAA36913B11A689B8893619620F7
:102F680001F044FFA36913B11A689B88138568218F
:102F78006069FEF753FA03216069FEF74FFAA36907
:102F880013B11A689B889361962001F02FFFA369FB
:102F980013B11A689B8813856B216069FEF73EFAA6
:102FA80003216069FEF73AFAA36913B11A689B888E
:102FB80093610F2001F0C0FEA36913B11A689B88C2
:102FC80013856A216069FEF729FA10216069FEF706
:102FD80025FAA36913B11A689B8893610F2001F041
:102FE800ABFEA36913B11A689B8813856C216069CD
:102FF800FEF714FA00216069FEF710FAA36913B10D
:103008001A689B8893610F2001F096FEA36994F8D3
:10301800506013B11A689B88138519216069FEF7FF
:10302800FDF931466069FEF7F9F9A36913B11A6829
:103038009B8893610F2001F07FFEA36913B11A6882
:103048009B8813851B216069FEF7E8F918216069E0
:10305800FEF7E4F9A36913B11A689B8893610F20FE
:1030680001F06AFEA36913B11A689B8813851C21B5
:103078006069FEF7D3F910216069FEF7CFF9A369FB
:1030880013B11A689B8893610F2001F055FEA3695C
:1030980013B11A689B88138537216069FEF7BEF95A
:1030A80010216069FEF7BAF9A36913B11A689B8801
:1030B80093610F2001F040FE6269138823F04003FA
:1030C8001B041B0C1380138823F038031B041B0CF0
:1030D800138013889BB243F040031380012001F052
:1030E8002BFE012385F83130A5E50AF032FBF2E525
:1030F8000AF02FFBD4E57B69002B3FF4B1AE3A68A8
:10310800002313607B74ABE67B69002B3FF47BAE36
:10311800044B39681B88044A92FBF3F301220B60C5
:103128007A7470E67069002020A1070030B5037C2E
:10313800012B85B004460D4628D0022B2CD183697B
:1031480013B11A689B8813859B216069FEF766F99D
:10315800022303AA00216069FEF7A4FCA36913B146
:103168001A689B889361BDF80C30124A43F290317B
:103178005BBA11FA83F382FB03121A44DB17C3EB21
:103188002223233301202B8005B030BD90F9140091
:10319800431C01D0022802DD002005B030BD03AB7E
:1031A800617D00931B220223FFF7D2F80028DAD1B1
:1031B800F2E700BFEBA00EEA70B5037C012B84B0E8
:1031C80004462DD0022B31D1836913B11A689B882C
:1031D80013859D216069FEF721F9062302AA0021C3
:1031E8006069FEF75FFCA36913B11A689B88936155
:1031F8009DF80C009DF808609DF809109DF80A508C
:103208009DF80B209DF80D3041EA062143EA002382
:1032180042EA0522012021876287A38704B070BD96
:1032280090F91400431C01D0022802DD002004B0EC
:1032380070BD02AB617D00931D220623FFF788F85D
:103248000028D5D1F2E770B5037C012B84B0044681
:103258002DD0022B31D1836913B11A689B8813854D
:10326800C3216069FEF7DAF8062302AA0021606923
:10327800FEF718FCA36913B11A689B8893619DF83F
:103288000C009DF808609DF809109DF80A509DF8FB
:103298000B209DF80D3041EA062143EA002342EA5B
:1032A8000522012021876287A38704B070BD90F9A9
:1032B8001400431C01D0022802DD002004B070BDB8
:1032C80002AB617D009343220623FFF741F80028F3
:1032D800D5D1F2E770B5037A012B84B004462DD01E
:1032E800022B31D1036913B11A689B881385BB215E
:1032F800E068FEF793F8062302AA0021E068FEF7CB
:10330800D1FB236913B11A689B8893619DF80C005F
:103318009DF808609DF809109DF80A509DF80B204B
:103328009DF80D3041EA062143EA002342EA0522CE
:103338000120E1822283638304B070BD90F90C0000
:10334800431C01D0022802DD002004B070BD02AB8E
:10335800617B00933B220623FEF7FAFF0028D5D1B4
:10336800F2E710B584B002AB0446009301220623AD
:103378001C210020FEF7ECFF30B39DF808209DF8D3
:1033880009309DF80A1043EA022343F38D03002B0A
:10339800B8BF03339DF80B209B1042EA0122E38259
:1033A8009DF80C109DF80D3042F38D0243EA01237D
:1033B800002A43F38D03B8BF0332002BB8BF033391
:1033C80092109B102283638304B010BDF0B585B0C2
:1033D80002AB04460093A822062319210020FEF719
:1033E800B7FF00B39DF809709DF808109DF80B60B1
:1033F8009DF80A209DF80D509DF80C3041EA0721F0
:1034080042EA062243EA052309B212B21BB201EBD3
:10341800D17102EBD27203EBD373491052105B10D7
:10342800E1822283638305B0F0BDF0B585B002ABBD
:1034380004460093A822062368210020FEF788FF8F
:10344800A0B19DF808709DF809109DF80A609DF8D4
:103458000B209DF80C509DF80D3041EA072142EAF7
:10346800062243EA052321876287A38705B0F0BDBA
:10347800F0B585B002AB044600930222062318215A
:103488000020FEF765FFB8B19DF809109DF80B20E4
:103498009DF80D309DF808709DF80A609DF80C5055
:1034A800090212021B0201EB970102EB960203EBE1
:1034B8009503E1822283638305B0F0BD2DE9F04FC7
:1034C800364B1B7885B08146002B3FD0002425461B
:1034D800264627460DF1080800E043B30134CDF82D
:1034E80000800823322253210020E4B2FEF730FF87
:1034F800A8B39DF809B09DF808109DF80BA09DF899
:103508000A209DF80DC09DF80C309DF80FE003EBE4
:103518000C2301EB0B2102EB0A22202C05FA83F580
:1035280007FA81F706FA82F60EF07F03D5D197FBEA
:10353800F4F796FBF4F6A9F8167095FBF4F4A9F8DD
:103548001860A9F81A4005B0BDE8F08F02AA18461D
:103558000092062332225321FEF7FAFE18B9002002
:1035680005B0BDE8F08F9DF809609DF808109DF83A
:103578000B509DF80A209DF80D409DF80C3001EB8A
:10358800062102EB052203EB0423A9F81610A9F87B
:103598001820A9F81A3005B0BDE8F08FA82E002031
:1035A8001749184B184A194810B4D1F8884044F400
:1035B8007004C1F888401C6844F001041C605C6811
:1035C80022405A601A6822F0847222F480321A600B
:1035D8001A6822F480221A605A6822F4FE025A609D
:1035E800DA6A22F00F02DA621A6B002410404FF0F8
:1035F800006218639C608A605DF8044B704700BFE6
:1036080000ED00E0001002400CC07FF8CCFC00FF89
:1036180038B50B4C23688BB15A68821A002A0546C4
:1036280004DA0CE05A68AA1A002A07DB9A682260B2
:1036380018461A6890472368002BF3D138BD38BD67
:10364800CC3000200B4B002210B4027203F58274B8
:10365800112102E0072A09DC9979890702D519792D
:10366800815401329C4203F11403F3D15DF8044BF9
:10367800704700BFC478030828230370704700BF51
:1036880030B4012330253324312132224570C471EE
:103698004171C2700372037083710371837030BC0F
:1036A800704700BF2C22022302704370704700BF8E
:1036B800436A8269D154436A0169826B01338B4240
:1036C80028BF00234362002A2FD0EFF31181502333
:1036D80083F31288836B1A68D2072CD470B45E689F
:1036E8006EB9456A826A954217D084691444DC60D1
:1036F8000ED9AA1A5A608562002280F854201A68E6
:1037080042F00102C9B21A6081F3118870BC704797
:103718000469A21A5A608662EEE7012380F85430E1
:10372800C9B281F3118870BC7047026D136843F009
:10373800800313607047C9B281F31188704700BFD6
:10374800426B10B462B1436CC2684469D11A013B40
:10375800615C5DF8044B08BF13464364C8B2704708
:10376800016A4369C4685B5C0131A14228BF114604
:1037780001625DF8044BD8B2704700BF836B13B188
:1037880090F854007047836A406A181AB0FA80F0BB
:1037980040097047416A836A99420AD3CB1A816B00
:1037A800026961B14968501E0B4483420AD2C01AAB
:1037B800704702691144CB1A816B0029F2D1501E5F
:1037C800C01A704700207047436B43B1426C5B6876
:1037D80093422FBF981AC0689B1AC0187047C269D5
:1037E800036A9A422FBFD01AC0688018C01A70475F
:1037F8000A4B30B503F1140493F900205D78072AC9
:10380800C8BF143A811804338D7213F8025C8554CA
:1038180013F8012C0A75A342EED130BD08510308F4
:1038280003682DE9F041DF691FB13B46BDE8F0416F
:103838001847002A164611DD04460D460E4400E0DE
:1038480023689B68204698470028F9D0236815F814
:10385800011B1B6820469847AE42F1D1BDE8F081B4
:1038680010B45A2158240022032304704170827036
:10387800C3705DF8044B70472DE9F0470569C368CC
:103888001D4028D00F4606464FF000484FF000096B
:10389800B5FA85F328FA03F2D2431B3B326115408F
:1038A800042B16D8DFE803F03129211903007B6ABD
:1038B800002B32D003F1FF3A1FFA8AFAC7F8249096
:1038C8003C6A34B123682046514698476468002C06
:1038D800F8D1002DDCD1BDE8F0873868716B03683A
:1038E80089B29847002DD3D1F5E77868B16B0368A2
:1038F80089B29847002DCBD1EDE7B868F16B036822
:1039080089B29847002DC3D1E5E7F868316C0368A0
:1039180089B29847002DBBD1DDE7F36A1FFA83FA15
:10392800CEE700BF30B50446006D61710368A26838
:1039380023F00103036087B0A379009213F0040217
:103948003DD04FF4805213F00203019244D1029308
:103958004FF480630022039311F00103059237D1DD
:10396800049308238D07694648BF049322F016FF85
:103978006079236DA17900F00202002A15BF4FF487
:1039880040324FF480324FF40034002410F0010F1D
:10399800586808BF2246CC074CBF024320EA0202FF
:1039A8005A609A6809074CBF42F0080222F00802E0
:1039B8009A601A6842F001021A6007B030BD13F02D
:1039C800020301920BD04FF4005513460295C1E74C
:1039D800042304930C23C5E74FF40053B7E702937D
:1039E800B8E700BF10B50446006DA160036823F076
:1039F80001030360A37986B013F00402009141D05B
:103A08004FF4805213F00203019244D102934FF411
:103A1800806362790393D1074FF000030493059301
:103A280045BF0423049308230C236946920748BF23
:103A3800049322F0B3FE6079236DA17900F00202AD
:103A4800002A15BF4FF440324FF480324FF400344F
:103A5800002410F0010F586808BF2246CC074CBF5D
:103A6800024320EA02025A609A6809074CBF42F0F2
:103A7800080222F008029A601A6842F001021A60ED
:103A880006B010BD13F00203019207D04FF40051A5
:103A980013460291BDE74FF40053B7E70293B8E726
:103AA800022828BF022010B4084C094B207000EBF4
:103AB8008002C0EBC20207495DF8044B013003EBFA
:103AC8004203C0B20B602EF01BBB00BFB8560020EB
:103AD800CC320020D439002008B517F0B7FA09F025
:103AE800F1FFBDE8084017F099BA00BF2DE9F04F83
:103AF800013085B0C3B203938E4D8F4F8F4C904EDB
:103B08000A2302933220DFF840922BF071FC4FF425
:103B1800FA7A4FF0100C4FF47A70D9F80430C3F3E6
:103B28000803002B40F0C880EFF31183002B40F00E
:103B3800C3802968A26800BF2B689942F9D1D7F8D9
:103B480000E000FB0EF39B1AB3FBFEF300FB013110
:103B58004FF0010E0191D9F80430C3F30803002B8C
:103B680040F08E80EFF31183002B40F089802B68A2
:103B7800A16800BF2A689342F9D1D7F800B000FBCA
:103B88000BF2521AB2FBFBF200FB0323019A9B1AB9
:103B9800B3F57A7FDFD3BAF1010ABED1039B002BBC
:103BA80040F0C4804FF47A7ADFF89C9150464FF089
:103BB800100CD9F80430C3F30803002B40F09980A7
:103BC800EFF31183002B40F094802968A26800BFAE
:103BD8002B689942F9D1D7F800E000FB0EF39B1A45
:103BE800B3FBFEF300FB01314FF0010E0191D9F850
:103BF8000430C3F308033BBBEFF3118323BB2B68EB
:103C0800A16800BF2A689342F9D1D7F800B000FB39
:103C18000BF2521AB2FBFBF200FB0323019A9B1A28
:103C2800B3F57A7FE3D3BAF1010AC2D1029B013B13
:103C380002937FF467AF4349434B4448444A0860C2
:103C4800DA6005B0BDE8F08FEFF311888CF31288C5
:103C5800A1682368DB0344BFC6F800E0A1682B68AD
:103C680032685FFA88F888F31188D7F800801A4418
:103C780000FB08F35B1AB3FBF8F300FB0233CDE754
:103C8800EFF311888CF31288A1682368DB0344BF23
:103C9800C6F800E0A1682B6832685FFA88F888F3F4
:103CA8001188D7F800801A4400FB08F35B1AB3FBAD
:103CB800F8F300FB023369E7EFF311828CF3128803
:103CC800D4F808E02368D90303D501233360D4F876
:103CD80008E02B683168D2B282F311883A68194437
:103CE80000FB02F3A3EB0E03B3FBF2F300FB01317D
:103CF8002EE7EFF311828CF31288D4F808E02368DA
:103D0800D90303D501233360D4F808E02B68316860
:103D1800D2B282F311883A68194400FB02F3A3EB8C
:103D28000E03B3FBF2F300FB01315DE718462BF0FD
:103D3800CFF937E7786900207C69002010E000E0BF
:103D480074690020FC9F002000ED00E0EFBEADDEAE
:103D58000400FA0538B5434B5A899989914224BF22
:103D680000225A81198ADA89914224BF0022DA8115
:103D7800DA788AB3072A2FD03B493C4D91F8530093
:103D8800012400210A282C709C70D9713DD00C2880
:103D980065D0DFED377A8ABB364C9FED370AA278BB
:103DA800002918BFF0EE407A062A04D8334901EBFF
:103DB800820191ED050A217959B3013A032A4DD8B8
:103DC800F7EE007A87EE800A30F056F92388984299
:103DD80028BF1846208038BDD97921B198780428A1
:103DE800B8BF04209870204890F853000A280CD0D7
:103DF8000C28CED1DFED227A002ACDD0072ACBD0ED
:103E08000A282CD1DFED1F7AC6E70A20DFED1E7ADB
:103E1800C1E79B78154A07EE103A1178B8EEC77AD1
:103E280027EE277A07EE901AF8EEE77A67EE877A98
:103E3800B4EEE70AF1EE10FA10DDC0EE077AFDEEF7
:103E4800E77A17EE903A102BA8BF1023012BB8BFC2
:103E58000123DBB28B4238BF0B46137038BDDFED50
:103E68000B7A99E7EC5B002010530020644A00208D
:103E78006F120339705E00206F120338085103086F
:103E88000AD7A3390F506E3A5304E9386F12833AB0
:103E98002DE9F047A84FA94E17F0D8F8BE421ED218
:103EA800DFF81483DFF814934446258862197DB13E
:103EB8004A450DD2052D0BD933886188C3F30B030E
:103EC800994200F0DD80144625886219002DEFD153
:103ED80071683046143609F081FDBE42E4D3984A31
:103EE8001378A3F1170102290FD9964911F8330065
:103EF800002840F0F180D8000144497829B192495E
:103F080011F83330002B00F00F81904B5A78022AB9
:103F180040F2DC8000228E495A701A788D48022AB5
:103F2800016000F2CF8002EB82018B4BC2EBC10231
:103F380003EB4203998C5A8C884C9142236001D33D
:103F480000225A84864B9A78042A00F0E48032B919
:103F58001A88B2F5F07F84BF4FF4F0721A80814D51
:103F6800FFF7F8FE2B68804A1A40002A00F0DF802D
:103F7800D80700F1CB80590400F1C3801A0700F17B
:103F8800BB809B0400F1B18020F0D0F910B97748CC
:103F98002DF038FD402009F057FD802009F054FD30
:103FA8004FF4802009F050FD4FF4001009F04CFD4B
:103FB8004FF0007009F048FD4FF0806009F044FDB3
:103FC8002AF03AFA00213022694831F012F82068C4
:103FD8002CF054FD674B276803F1500102E00433CD
:103FE80099426DD01A78002AF9D19C78D878844201
:103FF800F5D26149614B0D79614962480A70624E98
:10400800624C0460C822642111FB0521002259601A
:104018009A60DA601A615A619A61DA6183F820203D
:1040280083F82120376015F07BFB594B9FED595AD7
:104038001B88594A9FED596A5079594906EE903ABA
:10404800F8EEE66A1388C5EE265A07EE103A53884A
:104058001279C1ED005A07EE903AB8EEC77A514B83
:10406800F8EEE77A18725A7227EE067A67EE867AC1
:10407800BDE8F04783ED017AC3ED007A16F0CEBFB4
:1040880063799B077FF41FAF716894F804A03046EA
:1040980009F0A4FC3388BAEB133F04D01436BE42AF
:1040A800FFF402AF1BE773887068AA1FC3F30B0302
:1040B8009A4204F10601A8BF1A462FF09DFEEDE7CB
:1040C800012296E700221A70234B33E7204902EBBE
:1040D800420201EB820120E7D8000C186468002C2A
:1040E8007FF40AAF1724147006E72F4809F0ACFCD8
:1040F800402009F0A9FC47E72C4809F0A5FC2B68EB
:104108003FE72B4809F0A0FC2B6837E7294809F05E
:104118009BFC2B682FE71A8BB2F57A7FBFF41FAF91
:104128004FF47A721A831AE718231370EDE643F4F2
:1041380000532B601CE700BF24B7030888B20308AC
:10414800B44A0020987B0308E8790308B856002091
:10415800C4560020D8390020CC320020D4390020A1
:10416800705E00200034002009600002FC55002029
:10417800981F002030310020B4680020105700201C
:10418800C41A0020DC1F0020CC1F0020764A002023
:1041980088250020C0C9FB48D81E002017B7D13891
:1041A8008C250020B0670020094000020160000251
:1041B800092000020860000202F003080000040859
:1041C80008B516F043FF09F07DFC16F027FFFFF74E
:1041D8005FFE0120BDE808402DF092BF38B50C4CB9
:1041E8000C4DAC4206D261682046143409F0F6FB47
:1041F800AC42F8D3084A094B094C1460002209491B
:104208001A705A7008480860BDE8384021F0B2B802
:1042180088B2030824B70308D4390020B856002010
:10422800CC320020D8390020C456002008B5FFF74A
:10423800D5FF16F00BFF09F045FCBDE8084016F065
:10424800EDBE00BFF0B50C292BD8DFE801F06F2ACE
:104258002A2A4C2A2A2A2B2A2A2A0700046AB2F870
:104268000CE097881668674D24F480540462036A4A
:104278004468C16923F4005343EA0E3321F4E6414C
:10428800A84243EA073341EA062100F0B58005F564
:104298000065A84200F0B08092684460C161026481
:1042A8000362F0BD046A96899588D2F800E0554FFC
:1042B80024F480740462036A4468C16923F40073B7
:1042C80043EA062321F07301B84243EA052341EA91
:1042D8000E017ED04C4DA8427BD092684460C161EB
:1042E800C2630362F0BD046A96899588D2F800E03B
:1042F800444F24F010040462036A4468816923F07F
:10430800200321F0807143EA061321F4E641B84204
:1043180043EA051341EA0E2148D03B4DA84245D057
:1043280092684460816182630362F0BD046A938984
:10433800B2F804E01768334E24F001040462056AF9
:104348004468816943EA0E0321F4803125F00205AF
:104358009BB221F07301B04243EA050341EA070129
:1043680014D0294DA84211D005F54065A8420DD0BA
:1043780005F58065A84209D005F58065A84205D0F5
:1043880092684460816142630362F0BDD689158AF0
:10439800578A23F0080333433D43D68824F44074F6
:1043A80023F00403ADB233432C43E9E7D589178AD8
:1043B800D68823F0800343EA051324F44064558A21
:1043C80023F0400344EA870443EA061344EA8504D9
:1043D800A6E7D589178AD68823F4006343EA05231C
:1043E80024F44054558A23F4806344EA071443EACA
:1043F800062344EA051470E7158A24F4804444EA45
:10440800851449E7002C0140003401402DE9F04FA4
:104418004FF48C72002183B07848794CDFF804920D
:10442800784D794E794FDFF8008230F0E2FD784818
:104438007849DFF8F8E1DFF8F8C100221359834220
:1044480000F0C280B3F1804F00F0C080AB4200F0B2
:10445800C980B34200F0C880BB4200F0C7807345F2
:1044680000F0C680634500F0C580434500F0C48075
:10447800DFF8C0A153457FD00AF5806A534508BFCD
:1044880009237AD01432B2F58C7FD7D15C4C624DB7
:10449800624E604F04F58C7802E01434A04568D071
:1044A800A379002BF9D023794FEA131909F1FF39C1
:1044B800B9F1050F03F00F03EFD835F8190040FAEA
:1044C80003F2D207E9D54FF0010A0AFA03F3013BD8
:1044D80018402FF03DFA16F809305149184411EBED
:1044E800C002DAD051F83000DFF84CE1217A00F14F
:1044F80038439B0A1EF8033003F01F0E5B09022B9A
:104508000AFA0EFA69D0032B62D0012B03D17B691A
:104518004AEA03037B6193880093B3FA83F3C3F1F8
:104528001F039BB2DA0800EB820203F00703D2F8FC
:1045380020E09B004FF00F0C0CFA03FC2EEA0C0E47
:10454800C2F820E0D2F820E001FA03F343EA0E03B0
:10455800136269460023022214348DF804208DF872
:1045680005308DF806308DF8073021F0CDFEA045D6
:1045780096D103B0BDE8F08F082309EBC3034FF0D1
:10458800010B93F834A00AF01F034FEA5A1ABAF144
:10459800020F0BFA03F30BD0BAF1030F0ED0DA4572
:1045A8007FF470AFD1F814A043EA0A034B6169E7BE
:1045B800D1F818A043EA0A038B6163E7D1F81CA07D
:1045C80043EA0A03CB615DE70023D6E70123D4E77A
:1045D800FB694AEA0303FB619DE7BB694AEA0303F7
:1045E800BB6198E70223C8E70323C6E70423C4E7AF
:1045F8000523C2E70623C0E70723BEE7C0640020FF
:10460800C47803080004004000080040001000407F
:10461800002C014000100240B8730308C47303085B
:104628002C590020085103080040014000140040A4
:104638000034014000440140CC730308014902489A
:10464800FFF71AB9B0650020004801400149024847
:10465800FFF712B9606500200034014001490248A3
:10466800FFF70AB96065002000340140014902489B
:10467800FFF702B9386500200008004001490248E8
:10468800FFF7FAB8106500200004004002494FF017
:104698008040FFF7F1B800BFE864002010B5064C71
:1046A80006482146FFF7E8F804F1C8010448BDE8C8
:1046B8001040FFF7E1B800BFC0640020002C0140A3
:1046C8000044014001490248FFF7D6B8C064002001
:1046D800002C01402DE9F0410468514DA30AAB427A
:1046E80000F084800AD94F4DAB4277D00135AB42F8
:1046F8005FD0053DAB426DD0BDE8F0814A3DAB428D
:1047080070D00135AB4258D0B3F5801FF4D14FF0CB
:10471800480E012647794FEA970C00296AD0B00065
:10472800634685190227D4F80C809F400CEB45039B
:10473800BFB23D4D03F1040C47EA080745F82310C2
:1047480045F82C20E760EFF31181502282F312889C
:10475800821905EBC2021369002B32D013620433AD
:10476800821905EBC202576917B11F6053690433F8
:10477800821905EBC202976917B11F609369043368
:10478800821905EBC202D76917B11F60D3690433D8
:104798000027CAB21F6082F31188304405EBC000BD
:1047A800036A8BB9E3684FF6FE721340E360BDE815
:1047B800F0814FF4887E0626ACE74FF0980E03266A
:1047C800A8E705EB0E03CBE7E36843F00103E360DA
:1047D800BDE8F0814FF0C00E04269BE74FF0E80ECD
:1047E800052697E74FF0700E022693E74FF0200E4C
:1047F80000268FE7BF08022306FA03F0BB40DB431D
:10480800E768094D9BB23B4087190CEB470CE36006
:104818000CF1040345F82C1045F8232093E700BF5A
:104828004B00100051001000C064002030B5036830
:104838005C4D18885C4CB4FBF2F20139013AAB428A
:1048480094B283B089B282B266D05848834263D0AA
:10485800B3F1804F60D0A0F5983083425CD000F56A
:104868008060834258D0524883425BD000F5806014
:1048780083427DD022F4407200F58C3092B283429C
:104888001A80D9621C850ED0484A93420BD002F593
:104898004062934207D002F58062934203D002F54A
:1048A8008062934201D100221A8601225A611A8835
:1048B8003C4992B242F001028B421A8062D0B3F1B5
:1048C800804F61D03B4A934260D002F580629342A8
:1048D8005ED002F5006293425CD002F5806293429A
:1048E8005AD002F59032934258D002F54062934272
:1048F80056D002F5806293421ED002F58062934240
:1049080008BF092219D002A84FF0012340F8043D3E
:1049180021F0C4FC03B030BD254822F07002834268
:1049280092B2A3D101201A80D9621C8558611A88D5
:1049380092B202431A80C5E708221F4B03EBC20359
:1049480001A893F835408DF80440012300228DF822
:1049580005308DF807308DF8062021F09FFC1B2CC0
:10496800D8D1164B019301A821F098FC03B030BDB3
:1049780001201A80D9621C8558611A8892B20243B4
:104988001A809CE70022D8E70122D6E70222D4E762
:104998000322D2E70422D0E70522CEE70622CCE79D
:1049A8000722CAE7002C014000A24A040034014053
:1049B80000100040000400400851030819010001DC
:1049C800204B98422DD0B0F1804F2CD0A3F59433D2
:1049D80098422AD003F58063984228D003F50063F3
:1049E800984226D003F58063984224D003F590338B
:1049F800984222D003F54063984220D003F58063A3
:104A0800984207D003F58063984208BF092202D074
:104A18000020704708220C4B03EBC20393F83400C4
:104A280070470022F7E70122F5E70222F3E70322A5
:104A3800F1E70422EFE70522EDE70622EBE707227C
:104A4800E9E700BF002C0140085103082DE9F04FA9
:104A5800013085B0C3B203930B4602918B4C8C4E48
:104A6800002B00F09A8032208A4D8B4FDFF82C9271
:104A78002AF0BEFC4FF4FA7A4FF0100C4FF47A701B
:104A8800D9F80430C3F30803002B40F0DE80EFF3BD
:104A98001183002B40F0D9802968A26800BF2B68D9
:104AA8009942F9D1D7F800E000FB0EF39B1AB3FB4B
:104AB800FEF300FB01314FF0010E0191D9F80430EB
:104AC800C3F30803002B40F08780EFF31183002B1A
:104AD80040F082802B68A16800BF2A689342F9D110
:104AE800D7F800B000FB0BF2521AB2FBFBF200FB46
:104AF8000323019A9B1AB3F57A7FDFD3BAF1010A2F
:104B0800BED1039B002B40F0BD804FF47A7ADFF8CA
:104B18008C9150464FF0100CD9F80430C3F30803B9
:104B2800002B75D1EFF31183002B71D12968A2688E
:104B380000BF2B689942F9D1D7F800E000FB0EF3CB
:104B48009B1AB3FBFEF300FB01314FF0010E0191FC
:104B5800D9F80430C3F3080313BBEFF31183FBB98F
:104B68002B68A16800BF2A689342F9D1D7F800B032
:104B780000FB0BF2521AB2FBFBF200FB0323019A73
:104B88009B1AB3F57A7FE3D3BAF1010AC4D1029B29
:104B9800013B0293002B7FF466AF05B0BDE8F08FB0
:104BA800EFF311888CF31288A1682368DB0344BFF4
:104BB800C6F800E0A1682B6832685FFA88F888F3C5
:104BC8001188D7F800801A4400FB08F35B1AB3FB7E
:104BD800F8F300FB0233D2E7EFF311888CF3128865
:104BE800A1682368DB0344BFC6F800E0A1682B680E
:104BF80032685FFA88F888F31188D7F800801A4479
:104C080000FB08F35B1AB3FBF8F300FB023370E711
:104C1800EFF311828CF31288D4F808E02368D903E3
:104C280003D501233360D4F808E02B683168D2B289
:104C380082F311883A68194400FB02F3A3EB0E03D0
:104C4800B3FBF2F300FB01317FE7EFF311828CF342
:104C58001288D4F808E02368D90303D50123336008
:104C6800D4F808E02B683168D2B282F311883A6828
:104C7800194400FB02F3A3EB0E03B3FBF2F300FBB2
:104C8800013118E718462AF023FA3EE710E000E061
:104C980074690020786900207C69002000ED00E03C
:104CA800204B5B68C3F3080330B4BBB9EFF311833F
:104CB800A3B91D4B1D4C1868A16800BF1A68904223
:104CC800F9D11B4B1C684FF47A7202FB04F3591A92
:104CD800B1FBF4F130BC02FB00107047EFF3118216
:104CE800102383F3128811498C680B6813F4803FF2
:104CF800104B02D0012018608C680B49D2B20D68A5
:104D0800186882F311880A4B19684FF47A7228449C
:104D180002FB01F31B1B30BCB3FBF1F302FB0030B9
:104D2800704700BF00ED00E07869002010E000E067
:104D38007C690020746900202DE9F84F8046FFF750
:104D4800AFFF254E2549DFF8A0E0254A254D8446CA
:104D580010274FF47A740120DEF80430C3F30803F7
:104D6800D3B9EFF31183BBB90B68D2F808A000BF21
:104D7800D1F800904B45F7D1D6F800B004FB0BF9F9
:104D8800A9EB0A09B9FBFBF904FB0393A3EB0C039A
:104D98004345E1D3BDE8F88FEFF3118A87F3128812
:104DA800D2F808B01368DB0344BF2860D2F808B013
:104DB8000B68D5F800905FFA8AFA8AF31188D6F85A
:104DC80000A0994404FB0AF3A3EB0B03B3FBFAF32B
:104DD80004FB0933DAE700BF7C690020786900200A
:104DE80010E000E07469002000ED00E02DE9F04FCC
:104DF800DFF830C1474A4849484E494D8046102798
:104E080018F1FF38C0F08480DCF80430C3F30803DD
:104E1800002B5CD1EFF31183002B58D10B689468F9
:104E280000BF08688342F9D1D6F800904FF47A7031
:104E380000FB09FEAEEB040EBEFBF9FE00FB03EE21
:104E4800DCF80430C3F308034FF47A740120FBB98B
:104E5800EFF31183E3B90B68D2F808A000BFD1F8CB
:104E680000904B45F7D1D6F800B004FB0BF9A9EB3D
:104E78000A09B9FBFBF904FB0393A3EB0E03B3F593
:104E88007A7FBDD2DCF80430C3F30803002BDFD0EF
:104E9800EFF3118A87F31288D2F808B01368DB039E
:104EA80044BF2860D2F808B00B68D5F800905FFAC4
:104EB8008AFA8AF31188D6F800A0994404FB0AF309
:104EC800A3EB0B03B3FBFAF304FB0933D5E7EFF3CA
:104ED800118487F31288D2F808901368D80303D591
:104EE80001232B60D2F808900B682868E4B284F399
:104EF8001188D6F800A04FF47A7400EB030E04FB77
:104F08000AF3A3EB0903B3FBFAF304FB0E3E97E79E
:104F1800BDE8F08F10E000E0786900207C6900208F
:104F28007469002000ED00E030B4EFF31183102223
:104F380082F312880649074C0A680748013200259F
:104F48000A602560DBB2026883F3118830BC7047C1
:104F5800786900207469002010E000E00F4B1B887E
:104F6800014643B90E4B0F4A1B7810680BB981F004
:104F7800010108F09EBB0C4B5A691AB118B91A689E
:104F8800106058747047094A18681188084A92FBDB
:104F9800F1F2012102605974704700BF5069002086
:104FA8005269002054690020586900207069002067
:104FB80020A107001D4B70B51C69236D626BDD696C
:104FC800C2B1A36B2BB12B0702D5236D08221A623D
:104FD80070BD2A06F7D5A26A616A8A4220D0511CA0
:104FE800A069A162825C2069266D81423285EAD37C
:104FF800A362E8E7A906E4D5E26A22B1988C216B9E
:1050080080B29047DDE7E1699B8C6069DBB24E1C9A
:10501800E6614354E169E368994228BFE261D0E759
:10502800226D136823F080031360CCE72847002023
:105038001D4B70B5DC68236D626BDD69C2B1A36B73
:105048002BB12B0702D5236D08221A6270BD2A06E0
:10505800F7D5A26A616A8A4220D0511CA069A16270
:10506800825C2069266D81423285EAD3A362E8E733
:10507800A906E4D5E26A22B1988C216B80B29047E8
:10508800DDE7E1699B8C6069DBB24E1CE661435445
:10509800E169E368994228BFE261D0E7226D1368AD
:1050A80023F080031360CCE7284700201D4B70B520
:1050B8009C68236D626BDD69C2B1A36B2BB12B07B2
:1050C80002D5236D08221A6270BD2A06F7D5A26A96
:1050D800616A8A4220D0511CA069A162825C206961
:1050E800266D81423285EAD3A362E8E7A906E4D5B2
:1050F800E26A22B1988C216B80B29047DDE7E169C2
:105108009B8C6069DBB24E1CE6614354E169E3683D
:10511800994228BFE261D0E7226D136823F080032B
:105128001360CCE7284700201D4B70B55C68236DE1
:10513800626BDD69C2B1A36B2BB12B0702D5236D5E
:1051480008221A6270BD2A06F7D5A26A616A8A42E5
:1051580020D0511CA069A162825C2069266D814221
:105168003285EAD3A362E8E7A906E4D5E26A22B168
:10517800988C216B80B29047DDE7E1699B8C606970
:10518800DBB24E1CE6614354E169E368994228BFEB
:10519800E261D0E7226D136823F080031360CCE747
:1051A800284700201D4B70B51C68236D626BDD69B4
:1051B800C2B1A36B2BB12B0702D5236D08221A624B
:1051C80070BD2A06F7D5A26A616A8A4220D0511CAE
:1051D800A069A162825C2069266D81423285EAD38A
:1051E800A362E8E7A906E4D5E26A22B1988C216BAC
:1051F80080B29047DDE7E1699B8C6069DBB24E1CA9
:10520800E6614354E169E368994228BFE261D0E767
:10521800226D136823F080031360CCE72847002031
:1052280070B4EFF31186502383F31288836B1A68E6
:10523800D20720D45D686DB9446A826A944217D057
:1052480081691144D9600ED9A21A5A608462002279
:1052580080F854201A6842F00102F1B21A6081F312
:10526800118870BC704701698A1A5A608562EEE736
:10527800012380F85430F1B281F3118870BC704773
:1052880003685B6A03B11847704700BF03681B6A6D
:1052980003B11847704700BF03682DE9F041DF6983
:1052A8001FB13B46BDE8F0411847002A164611DDFC
:1052B80004460D460E4400E023689B682046984744
:1052C8000028F9D0236815F8011B1B682046984769
:1052D800AE42F1D1BDE8F08103689B69184700BF71
:1052E8000368DB68184700BF03689B68184700BF5E
:1052F80003685B68184700BF03681B68184700BF4E
:1053080010B40B4B0B4A1C7801238340234052F8FE
:10531800200031B9B3FA83F149095DF8044B08F06C
:10532800C8B9191C18BF01215DF8044B08F0C1B9B0
:10533800406900204469002008B501210220FFF7D8
:10534800DFFF094B1B7803F00503052B08D000216C
:105358000120FFF7D5FF00210846FFF7D1FFFEE740
:1053680028F00AFBF3E700BF24470020054B53F859
:10537800203033B11A689B88918A0B4218BF1B04EE
:1053880093617047446900202DE9F04FC04B1E78A7
:105398008BB0002E40F0BC80BE4BBF4C1D78DFF8B0
:1053A80018A3DFF81893DFF8188305F00105A4F1B6
:1053B8000A0B54F80A3CBBB1CC2707FB06B71846C2
:1053C800FFF796FF80B154F80A0CFFF789FF14F82D
:1053D800023C8BB9242831D0F5B154F80A3C184660
:1053E800FFF786FF0028EED10136032E04F1CC0426
:1053F800DFD10BB0BDE8F08F012B23D0022B2BD0CF
:10540800032B37D0042B67D0052B40D0062B4FD069
:1054180054F80A2C1346D2E754F80A3C23281A46B3
:1054280000F089819D4991F832108142C7D19C4B87
:10543800CAF80090C3F80C801346C0E7012304F8AB
:10544800023CCAE74D2854F80A2C0CBF022300235B
:1054580004F8023C1346B2E700233C2804F8023C57
:1054680045D03E28D4D10122032304F8012C04F8A6
:10547800023CB2E7C02814D80022042304F8050C23
:1054880004F8040C04F8062C04F8023CA5E714F808
:10549800063C14F8052C9A422FD814F8043C834291
:1054A80003D0002304F8023C97E7062304F8023CE3
:1054B80014F801ECBEF1000F00F08081BEF1010F7D
:1054C80000F0C48101360023032E04F8023C04F1E5
:1054D800CC047FF46EAF8CE714F8043C04F8030C9A
:1054E8005840052304F8040C04F8023C75E703222D
:1054F80004F8013C04F8022C6FE714F8042CF9189E
:105508004240013304F8042C04F8063C887264E72E
:10551800644B186800283FF46CAF08F00BFADFF80A
:10552800A4A1614DDFF8A091DAF80000FFF7E0FED2
:1055380000283FF45EAFDAF80000FFF7D1FE092833
:105548001BD03F2819D02B68002B67D1042800F006
:10555800A7810C2800F0E8807F28E5D0A0F1200280
:10556800D2B25E2AE0D80BB92028DDD05A1C09F83F
:1055780003002A602AF05EF9D6E72C68002C5BD17C
:105588004A4FA34607F59878BBF1000F08BFBB4602
:1055980008374745F8D1BBF1000F00F07681083F86
:1055A800DBF800003A68065D135D9E42204402EB7A
:1055B800040140F06881661E4E4422460BB9FD2A5C
:1055C8005DD906F8013F01322A6010F8013F11F851
:1055D80001EF9E45F2D00AB15F4512D034482AF057
:1055E80031F95F4508D35BF8080B2AF02BF909203D
:1055F8002AF020F9BB45F6D92E482AF023F92A6863
:105608000024944290D2661E4E4416F8010F2AF0E8
:1056180011F92B6801349C42F7D385E70C2800F078
:1056280083800A2852D00D2850D07F2800F0FB80B4
:10563800FF2B3FF679AF91E71C4E002706F59878C7
:10564800BB4602E0083646450DD02246316848463A
:1056580008F036FD0028F5D1B346002FF2D13746C1
:1056680008364645F1D13B465F469B46002B97D10D
:10567800002F3FF459AF0E482AF0E4F8B3E7511C65
:10568800202009F80200296009F801300A46A3E73A
:105698009D560020F757002046750020FC55002035
:1056A80000ED00E03C26002044270020B059030804
:1056B800C8800308D0800308FC9F0020EFBEADDE41
:1056C8000400FA0540260020442600202AF03BF971
:1056D80023217B482FF0A4FC002800F0DF80A0EBFA
:1056E8000900286088B1431E19F80310202940F0EA
:1056F800E58009EB030204E012F8011D202946D1D8
:105708000346581E002BF7D12B604FF480720021FE
:1057180048462FF06EFC6B4B1B78002B3FF469AEAC
:1057280069482AF08FF8FFE668482AF08BF866483F
:105738002AF088F8F8E666496648C978664ADFF8C4
:10574800C8E11360003118BF01210170634951603D
:105758004021936011735573614962480B600432AC
:10576800CEF80020574A012313702AF0F1F9564861
:105778002AF068F84FF400600FF0BEFD5A4B93F81A
:105788003230232B00F0928014F8023C3EE62B6066
:10579800564C002204F5987809F8032002E00834F2
:1057A800444577D02168484611F002F80028F6D021
:1057B80044456FD2636898470023A5E74C4BADF882
:1057C80022E00FCB0DF1280C02AF87E80F004CF850
:1057D80024ED14F8051C14F8033C069404EB010EA0
:1057E800624639464FF0010C06A8CDF81CE0ADF82A
:1057F80020308DF824C000F089F8E8B9019F002313
:1058080004F8023C002F3FF4EFAD54F80A0C19F0ED
:1058180035FE013654F80A0CB847032E04F1CC04BF
:105828007FF4C7ADE5E5013B002232482B6009F85B
:1058380003202AF007F877E6029A2F4B039239469D
:10584800A4F10A00029319F059FDD7E714F8053CB2
:1058580014F8032C0694234407936E2A4FF0000390
:1058680008930993ADF820207FF42CAE06A808F021
:10587800A6FC06A808F098FC06A808F095FC06A85F
:1058880008F092FC1EE62246A5E61C48083F29F0CF
:10589800D9FFA8E61A4829F0D5FF8DE7286821E73F
:1058A800074810F0CEFB0BB0BDE8F08F154A14F88E
:1058B800023CC2F80C80CAF80090A7E5034667E7E7
:1058C800442600209D560020D0800308D880030875
:1058D800B8560020343B00207C1E002029380008E0
:1058E8004026002004810308FC550020B059030815
:1058F8008851030800810308FC7A0020C880030847
:10590800E480030800ED00E03C2600202DE9F04F7C
:1059180095B0B0F908500D81EDB2442D00AF0C469A
:10592800904600F04684064643D9812D00F07D83D9
:1059380000F29880542D00F0CC8040F262836E2DE6
:1059480000F00584802D40F0CD80734B93F800A0C3
:105958000AF1020A1AF0FF0A00F097806F4BDFF88D
:10596800EC816F4EDFF8E8B19A4403F101090A258A
:1059780016E0322D01F03E83A5F13C00C0B2132899
:1059880041F2428300232268511C2160157022686D
:10599800CA4502F101012160137076D019F8015B44
:1059A8000A2DE6D1BBF80030FF2BA8BFFF23DBB2DE
:1059B800E9E7052D00F0EB8320D8022D00F0818067
:1059C80040F20C83032D00F0B783042D40F08A8049
:1059D8002A465449204608F0F7FB0021204608F0E3
:1059E80021FC22680021531C0125236028462B46F0
:1059F800543711706381BD46BDE8F08F242D5ED009
:105A080040F2A282282D00F05983382D6AD10A6805
:105A1800454B0125511C216015702268052150193C
:105A28002060117022680A215019206011702268C4
:105A380000215019206011702268197850192060CF
:105A4800117022685978501920601170226899786D
:105A5800531923602B461170284654376381BD467D
:105A6800BDE8F08FA02D18D040F28D82B82D00F03F
:105A78006183FE2D36D12D4D05F1080635F8021B40
:105A8800204608F0CFFBB542F8D101252B46284621
:105A980054376381BD46BDE8F08F254B0846196829
:105AA80008F0A9FB234B2046196808F0A4FB224BF9
:105AB80019682046012508F09EFB2B46E7E71F4B97
:105AC800F6E704221E492046012508F07DFB2B46F7
:105AD800C2E70B681B491022581C20601A70226804
:105AE800097880E7214628460EF0D6FB03460028B1
:105AF800CBD1742D00F08B82772D2BD13268716851
:105B080091421EBF531C336011780F4A08BF1946D3
:105B180020462CF0AFFBB8E7353600209851030833
:105B28006C3A0020BE560020B732002058360020BC
:105B3800ACF7FF1FB0F7FF1FB4F7FF1F00340020BA
:105B48000C810308D01E0020011A030867666666E8
:105B5800943A0020F52D01F0FE82472D00F056837F
:105B6800292D336801F0BD82392D01F0A782212D3E
:105B780001F0848271680B3DCA1AEF2D00F2B084DF
:105B880001A050F825F000BF836E0008E964000802
:105B9800E9640008E9640008E9640008E9640008A9
:105BA800E9640008E9640008E9640008E964000899
:105BB800E9640008E9640008E9640008E964000889
:105BC800E9640008E9640008E9640008E964000879
:105BD800E9640008E9640008E9640008E964000869
:105BE800E9640008E9640008296E0008E96400080F
:105BF800076E0008E9640008DD6D0008E964000824
:105C0800E9640008E9640008C36F0008E964000853
:105C18004D6F0008E9640008E16E0008E9640008B7
:105C2800BB6E0008E9640008EB6F0008E96400082F
:105C3800856D0008E9640008316D0008E964000812
:105C4800E9640008E9640008E9640008935A000858
:105C5800E9640008056D0008E9640008E9640008C3
:105C6800EB6C0008E9640008916C0008E96400081E
:105C7800E9640008E9640008E9640008856C000824
:105C8800E9640008E9640008E9640008456C000854
:105C9800E9640008BD6B0008E9640008E9640008CD
:105CA8007F6B0008E9640008E9640008E9640008FB
:105CB800E9640008E9640008E9640008E964000888
:105CC800116B0008E96400088F6A0008E96400089D
:105CD800AD690008E9640008FF680008E964000885
:105CE800676A0008E1680008C5680008E9640008F8
:105CF800E9640008E9640008E9640008E964000848
:105D0800E9640008E9640008E9640008E964000837
:105D1800E9640008E9640008E9640008E964000827
:105D2800E9640008E9640008E9640008E964000817
:105D3800E9640008E9640008E9640008E964000807
:105D4800E9640008E9640008E9640008E9640008F7
:105D5800E9640008E9640008E9640008E9640008E7
:105D6800E9640008E9640008E9640008E9640008D7
:105D7800E9640008E9640008E9640008E9640008C7
:105D8800E9640008E9640008E9640008E9640008B7
:105D9800E9640008E9640008E9640008E9640008A7
:105DA800E9640008E9640008E9640008E964000897
:105DB800E9640008E9640008E9640008E964000887
:105DC800E9640008E9640008E9640008E964000877
:105DD800E9640008E9640008E9640008E964000867
:105DE800E9640008E9640008E9640008E964000857
:105DF800E9640008E9640008E9640008E964000847
:105E0800E9640008E9640008E9640008E964000836
:105E1800E9640008E9640008E9640008E964000826
:105E2800E9640008E9640008E9640008E964000816
:105E3800E9640008E964000851680008E96400089A
:105E4800356800080B680008E9640008E964000880
:105E5800E9640008E9640008E9640008E9640008E6
:105E6800E9640008E9640008E9640008E9640008D6
:105E7800E9640008E9640008E9640008916700081B
:105E8800E964000859670008E9640008B766000873
:105E98009D660008EF670008E9640008836600084B
:105EA800E96400085B66000849660008E9650008BF
:105EB800E9640008B9650008E9640008E9640008B5
:105EC8008F650008616500081B650008F364000819
:105ED800CB640008A1640008E9640008896400082C
:105EE800E9640008E9640008E9640008E964000856
:105EF800E9640008E9640008E9640008E964000846
:105F0800E9640008E9640008E9640008E964000835
:105F1800E9640008E964000869640008E9640008A5
:105F2800E964000811640008E9640008E9640008ED
:105F3800E9640008AD630008E9640008E964000842
:105F4800E964000893630008202D7FF4CBAD0B684B
:105F58009C4D591C6A7821601A7023682A78591C4C
:105F680021601A702368AA78591C21601A7029893F
:105F7800204608F057F923686A79591C21601A707D
:105F88002268A9792FE5822D7FF4ACAD0B688E4A83
:105F98008E4D11788B4A581C206019701189204643
:105FA80008F040F98A4B22681B88FF2B02F1010197
:105FB800A8BFFF2321601370A96881F3100189B27B
:105FC800204608F02FF9296801F30F0189B220460D
:105FD80008F028F97F4B2268197804E5012D7FF431
:105FE80081AD0B680022591C21601A7023685A1C65
:105FF80022601D7022682521531C23602B461170D6
:106008002AE5522D7FF46EAD22680021EBE4326858
:10601800716891421EBF531C336011786E4A08BFE5
:10602800194620462CF026F92FE56C4B1E780336CE
:1060380016F0FF063FF429AD694BDFF8C8811E440E
:1060480003F1010A4FF00A0920E0B9F1500F00F0FE
:10605800D887B9F1320F00F0ED87A9F13C00C0B242
:10606800132840F2EB870025294623685A1C226032
:10607800204683F8009008F0D5F82946204608F015
:10608800D1F8B2453FF401AD1AF8019BB9F10A0FF6
:10609800DBD1544B9D68196805EB85054FF6FF73F6
:1060A8006D009D42A8BF1D469942A8BF194625EA22
:1060B800E57521EAE171ADB289B2D6E70B68DFF880
:1060C8004891494E591C022221601A7023684FF0EA
:1060D80006085A1C226083F8008023680A22591C8B
:1060E80021601A70236801255A1922601D70B9F8B9
:1060F8000010204608F096F8B9F80210204608F07B
:1061080091F823685A19226083F800802368502286
:10611800591921601A7023680022591921601A70D0
:106128003188204608F07EF87188204608F07AF811
:106138002B4691E42D4BBBE40B685A1C0A601D707A
:106148000B685A1C0A601D700A6800214BE4204B3A
:106158000A681B881D4DFF2BA8BFFF23511C216017
:106168001370A96881F3100189B2204608F05AF823
:106178001F4B2046198808F055F8296801F30F01CC
:1061880089B22046012508F04DF82B4664E40B221D
:106198001849204608F018F808221749204608F040
:1061A80013F8012507221549204608F00DF82B465B
:1061B80052E4002A3FF469AC114B136001252B46C9
:1061C8004AE400BF583900209A3700206839002077
:1061D80084370020544D0020611A0308353600200A
:1061E800A8510308203A0020543A0020F42800203F
:1061F800504D002014810308208103082C810308D6
:1062080075420108643A0020604A002072683568C7
:106218007B623046551B07F0B0FF052D38627B6A5C
:1062280001F22E808026B346012594E80600521A12
:10623800103AB242B8BF1FFA82FBBB4A396A926869
:106248003A61521A9345396A7B622046FA6088BFE0
:106258001FFA82FB07F0CFFF7B6A002B00F0D8877C
:10626800002D40F057872368C7F800D05D71C0B093
:106278000533C7F808D0FB61BBF1000F01F0D480EB
:106288003B6A3A69934281F0CB80AA463E6A7D62B6
:106298007C6080255446FB681C1BA34BB4F5807FAB
:1062A80028BF4FF480749B6832199A4288BF9C1BA0
:1062B80008F0D4FC2246BC683046214608F054FD5C
:1062C800F969B86104EB000C0B787B61644530D246
:1062D800DFF87C920CF1FF3C04F1FF3E1EF8013F11
:1062E80009EB830219F823405688FCB100234FF4C8
:1062F800004204F1FF3816424FEA520202D00878F1
:10630800284308706D0806D10AF1010A4D701FFA7A
:106318008AFA01318025D34505D8F44500F2A586CF
:106328004345C0F2A28601339C42E4D1E645D5D16B
:10633800F9617B6ABA6913449BB2D3457B6206D97B
:106348007B6A3A6A1C46D6183B699E42A3D37C688E
:10635800802D1CBF0AF101031FFA83FA0AF102011A
:1063680089B2204607F05EFF2368796A01255A1929
:10637800226020461D7007F055FF236853442360B0
:106388002B46D7F800D0FFF767BB684B1B78DB07B5
:1063980000F1A6800125FDF79FFBFDF779FD2B464F
:1063A800FFF75ABB304607F0FFFE3368B8851A4638
:1063B800591C316012F8021B326087F82E105A7887
:1063C80087F82F20DA1C32609A7887F830201A1D57
:1063D8003260DA7887F831205A1D32601B7987F8E5
:1063E800323007F12C000023BB8607F037FE504AF5
:1063F800504B1268801A4FF0010561F10001C3E9A2
:1064080004012B46FFF728BB5A1C32601A780F2A62
:1064180066D8991C3160C2EBC20247495878885443
:10642800D81C30600A4499785170191D3160D978A8
:106438009170591D31601979D170991D3160597960
:106448001171D91D31609979517103F108013160D9
:10645800DB799371012529F06DFF2B46FFF7FCBA14
:10646800304607F0A1FEDFF8DC80A8F80E003046C1
:1064780007F09AFE0125A8F80C002B46FFF7ECBAA6
:10648800304607F091FE2D4A00EB800043000125BD
:1064980013802B46FFF7E0BA304607F085FEDFF899
:1064A800B480A8F81400304607F07EFEA8F816005D
:1064B800304607F079FE0125A8F818002B46FFF7AB
:1064C800CBBA1A46591C316012F8020B3260DA1C3A
:1064D800597832609A781CF05FFD00287FF4D5AABD
:1064E8004FF0FF352B46FFF7B7BA1A46591C3160F3
:1064F800134912F8020B0870326012495A788A70F0
:10650800DA1C32600D4A9B78937001252B46FFF701
:10651800A3BA0D4B0D4918684E2201252DF06CFCCD
:106528002B46FFF799BA00BFA0130020F7570020A9
:1065380078690020D01E002008280020804A00200A
:10654800EC5B0020704A0020D439002074780308DE
:10655800B8510308705E002019465A1C3260C54ABB
:1065680011F8020B1070316059785170D91C3160E4
:106578009B789370304607F017FEBF4B0125D880F3
:106588002B46FFF769BA304607F00EFEDFF8E882BF
:10659800A8F80000304607F007FEA8F802003046C9
:1065A80007F002FE0125A8F804002B46FFF754BAAD
:1065B800DFF8F49299F80030002B3FF466AADFF870
:1065C800EC820025304607F0EFFD27F0F9F899F83E
:1065D8000030A8EC010A01359D42F3DBFFF755BAFC
:1065E8000D2A7FF47DAF5A1C32601D78072D3FF6C7
:1065F80077AFDFF8BC9230464FF00C0807F0D4FDB7
:1066080008FB05F809EB0805A880304607F0CCFD23
:10661800E880304607F0C8FD336828811A46591CBF
:10662800316012F8021BA97232605B78EB72304657
:1066380007F0A3FD012549F808002B46FFF70CBA1F
:10664800304607F0B1FD8D4B012518802B46FFF72A
:1066580003BA5A1C32601878060600F1BD86884BCA
:106668001B78DD073FF511AA032828BF0020012564
:10667800FDF716FA2B46FFF7EFB9814B1B78D807C1
:106688003FF503AA0125FDF7D1FDFDF701FC2B46D7
:10669800FFF7E2B97A4B1B78D9073FF5F6A9794B92
:1066A8004FF4C87201251A802B46FFF7D5B9092A7D
:1066B8007FF716AFDFF8FC811A46591CD8F800504E
:1066C800316012F8021B297032605A78AA70DA1CFD
:1066D80032609A78642A03F10401A8BF64226A71BF
:1066E8003160DA78642A03F10501A8BF6422AA712F
:1066F80031601A79EA719A1D32605A79642A03F175
:106708000701A8BF64222A7231609A79EA7003F1FE
:1067180008023260DB792B71304607F045FD72685C
:1067280033686881D11A00290CDD591CD8F800009B
:106738003160521A002A1978417203DD9A1C3260BE
:106748005B784370012527F077FE2B46FFF784B965
:106758004D4A1068DA1C01462133951E356012F83F
:10676800035C0D70551E356012F8025C4D70326086
:1067780012F8015C8D700332934201F10301ECD1F0
:106788002AF04CF8FFF781B9C2F34705122D3FF6FE
:10679800A7AEC5B107F1500307F12A0903EB450A73
:1067A800C846AAF1260A304607F0FEFC28F8020F70
:1067B800C245F8D1354B39F8022F23F8022FC845C6
:1067C800F9D1112D09D8324A6B00023B134400213C
:1067D800223223F8021F9A42FBD12E4A01231D467A
:1067E8001370FFF739B9264B1B78DA073FF54DA927
:1067F800294A1378012543F0040313702B46FFF749
:106808002BB95A1C254932600A781B78002A40F0B7
:10681800EE8504220A70224A9B001380FEF740FA94
:10682800204B012598612B46FFF716B9DFF88880C1
:1068380000233046C8F8003007F09FFC0125C8F84F
:1068480000002B46FFF708B91A46591C316012F8A8
:10685800025B3260DA1C587832609978002D00F0BB
:10686800F685012D7FF411A925F024F92B46FFF7B1
:10687800F3B800BF684A00209868002086250020E9
:10688800F7570020D8680020D43900201E66002061
:10689800206600201C660020587A0020BE2A0020AE
:1068A800504D0020D01E0020353600200C26002038
:1068B80048270020D8390020F42800205A1C3260CC
:1068C8001B78002B00F098854FF4004001250EF04E
:1068D80013FD2B46FFF7C0B8CA4A127812F001011F
:1068E8007FF4FEAD5A1C32601878012525F026F891
:1068F8002B46FFF7B1B8304607F056FC304607F094
:1069080053FC304607F050FC304607F058FC33681B
:10691800BD4D1946581C2A68306011F8020B82F8E0
:106928002C003160597882F83610D91C31609B7878
:1069380082F83730304607F042FC304607F03FFC1B
:10694800304607F03CFC3046D5F8008007F02CFCB8
:10695800A8F83A003046D5F8008007F025FC3368DF
:106968007268A8F83800D11A01290ADD591C2A686A
:1069780031601B7882F82E30304607F020FC3368EF
:106988007268D31A032B0BDD3046D5F8008007F068
:106998000BFCA8F8320030462E6807F005FCB086DC
:1069A8002868EDE65A1C3260974DDFF884821B7820
:1069B80088F805303046D5F8009007F0F5FBA9F8BF
:1069C80020003046D5F8009007F0EEFB7268336877
:1069D800A9F81E00D11A072919DD304607F0E4FB93
:1069E800A8F80A00304607F0DFFBA8F80C0030468C
:1069F800D5F8009007F0D8FBA9F822003046D5F862
:106A0800009007F0D1FB33687268A9F82400D11A06
:106A180003290BDD304607F0C7FBA8F80E00304607
:106A280007F0C2FB33687268A8F81000D21A002A6F
:106A380005DD591C2A6831601B7882F82630FDF77D
:106A480089F920F00FFB714B1B68002B00F0DD84E7
:106A58002868012529F002FD2B46FEF7FDBF1A46DE
:106A6800591C31606A4912F8020BC87032606949D2
:106A78005A784A71DA1C3260674A9B78D3700125CC
:106A88002B46FEF7E9BF1A46591C3160DFF8A08192
:106A980012F8021B88F80210326060495A780A70AE
:106AA800DA1C32605E4D9A782A711A1D3260DB78E2
:106AB800092BA8BF09233046AB7007F075FB336874
:106AC80072682880D11A012905DD304607F06CFB71
:106AD8003368726868829A4207D05A1C32601B7801
:106AE800003318BF012388F80730FDF733F93368FE
:106AF80072689A423EF4C9AF5A1C32601B78EB7038
:106B080001252B46FEF7A8BF464B1B68002B3EF419
:106B1800BCAF23F0AFF9FF283EF4B7AF304607F01B
:106B280043FB3F2840F29984DFF80881002588F864
:106B3800005033687268A8F80400D21A012A7EF758
:106B4800A4AF1A46591C316012F8021B88F80210CB
:106B580007F15000326000225D7800F8242D23F000
:106B68005BF997F82C30AB423EF48FAF284623F000
:106B780077F9FEF78ABF2C4A1278012A3EF685AFCC
:106B880018465A1C3260DFF8B08010F8022B88F8DB
:106B98000220DA1C891A306001295878326040F3E3
:106BA8006C84304607F000FB0125A8F800002B464E
:106BB800FEF752BF5A1C326093F80080B8F1110FEB
:106BC8003FF68EAC9A1C3260184D5B7805F8183089
:106BD800304607F0E9FA40F6CA039842A8BF1846BB
:106BE80040F2EE23984205EB4801B8BF184601254C
:106BF800A0F2EE222B46192092FBF0F24A70FEF723
:106C08002BBF00BFF7570020D4390020984A002036
:106C1800704A0020FC520020804A0020644A00206C
:106C2800705E0020FC570020EA330020403200202C
:106C3800EC5B002000580020EC3300201A46591C59
:106C4800B24D316012F8021B297132605B786B71AA
:106C5800304607F0A9FA336828805A1C32601B783E
:106C6800AB71304607F0A0FA336868805A1C32606E
:106C78001B78EB7101252B46FEF7EEBE012508F0C7
:106C88004FF82B46FEF7E8BE5A1C3260A04A1B7824
:106C9800DFF8AC8213700023C8F80030304607F0E4
:106CA8006CFA3368D8F800209A499B4D10435A1C57
:106CB800C8F8000032601B780B72304607F074FA8F
:106CC8002860304607F070FA6860304607F06CFAC2
:106CD800A860304607F068FA304607F065FAFEF714
:106CE800D4BE8E4A03F108010133336013F8010C56
:106CF80002F8010F8B42F7D1FEF7C7BE1A46581C9F
:106D08003060874812F8025B857032605D784570A4
:106D18008A423EF4BAAEDA1C3260824A9B78137318
:106D280001252B46FEF798BE0721B2FBF1F1C1EB16
:106D3800C105521B7FF4D4ABC9B201F1FF395FFA28
:106D480089F900293EF4A1AEDFF8DCA109F10109B7
:106D580015465A1C326093F90010734B4FF0000827
:106D680093F902208A4203F1080300F0AB8208F18C
:106D78000108B8F1060FF3D1FFF7B2BB5A1C326015
:106D88001A780E2A3FF6ACAB991C31605D78032D5A
:106D98003FF6A6AB6548062101FB02F1421803F154
:106DA800030E5571C6F800E09D784554191D3160F1
:106DB800D9785170591D316019799170991D3160D8
:106DC8005979D170D91D31609B79137101252B46F2
:106DD800FEF742BE304607F0E7F9DFF83C81C8F815
:106DE8000000304607F0E0F9C8F80400304607F024
:106DF800DBF90125C8F808002B46FEF72DBEDFF8A1
:106E080040810023C8F80030304607F0B6F9D8F8BA
:106E1800003001250343C8F800302B46FEF71CBE9E
:106E28005A1C32601D78132D3FF65AAB9A1C3260FB
:106E380058787B622BF058FA00283FF451AB7B6AF4
:106E48003B4A017802F82510D91C316002EB850213
:106E580099785170191D3160D9789170591D316038
:106E68001B79D370002027F027FA324B80F00100FD
:106E7800012518702B46FEF7EFBD2F49102A13463F
:106E88004FF0000228BF10230A604A608A60CA6077
:106E98000A74002B3EF4F9AD32680139134401320B
:106EA800326012F8010C01F8010F9A42F7D1FEF78F
:106EB800ECBD591C31601D781F2D3FF611AB052A1A
:106EC8007FF40EAB304607F058F91C4B43F8250009
:106ED8001EF050FAFEF7D9BD184D05F140083046AE
:106EE80007F062F93368A5F88000591C1A4631602A
:106EF80012F8021B85F8821032605B7885F88330BF
:106F08000435A845EBD1FEF7C0BD00BFB46800202A
:106F1800B44A0020D055002054470020CF55002007
:106F2800904A0020D01E0020FC5500200029002097
:106F380030310020C41A00204C4A0020104B002099
:106F4800003400205A1C3260C24D1B782B72304628
:106F580007F02AF9A883304607F026F92883304637
:106F680007F022F932686883531C33601278EA7498
:106F78007268D31A032B00F310823368D11A0529DB
:106F88000EDD5A1C32601B78EB72304607F0F5F8BC
:106F98003368E8605A1C32601B782B743368726857
:106FA800D21A002A7EF771AD5A1C32601B7885F818
:106FB800213001252B46FEF74FBD581C3060A64AEC
:106FC8001D781570091A00297EF75FAD991C31608C
:106FD8005B78003318BF0123012553702B46FEF759
:106FE8003BBD5A1C32609B4A1B78537501252B46C2
:106FF800FEF732BD3388FF2BA8BFFF23DBB2FEF7B5
:10700800C2BC964BFFF746B816F030FF00283EF496
:10701800B9AC03780A2B2FD8B0F9023088FB0312D9
:10702800DB17C3EBA2039BB2FF2BA8BFFF23DBB286
:10703800FEF7A9BC98E82200FFF72EB816F016FF55
:1070480000283FF410A803780A2B3FF60CA8B0F9E3
:107058000430B0F9061003EB830383F3500521EAEB
:10706800E171ADB289B2FFF700B8FB697C681A46D6
:107078003B7D1370FFF76CB90023D8E71A46591CFB
:107088003160774D12F8021B697032605A782A70A5
:10709800DA1C32609B78AB70304607F085F83368AD
:1070A8002881591C1A46316012F8021B6971326036
:1070B8005B78AB7101252B46FEF7CEBC5A1C3260BB
:1070C8001A780A2A00F0EF80304607F078F8304640
:1070D80007F075F80125304607F071F82B46FEF7E2
:1070E800BBBC5A1C32601B780A2B00F0D680502B90
:1070F8007FF4EFAD304607F057F8DFF87C81A8F849
:107108000000304607F050F80125A8F802002B4689
:10711800FEF7A2BC534B3A6A9B68D4F800905A44D5
:107128009342C0F0278107F099FD5A464946386ACC
:1071380007F01AFE236803442360B042BEF6A5ACEC
:10714800002100E0236801305A1CB0422260197007
:10715800F8D1FEF79ABC336872689A4240F0E18031
:10716800414BFF22DA704FF0000A404D23F0DAFC61
:10717800514630223E4885F800A02DF03AFF87F8A6
:107188002CA097F82C300B2B00F20581DFF8EC903F
:10719800374E524697F82C3003EB430309EBC303F1
:1071A8005B7CE3B197F82C3003EB430309EBC30393
:1071B80020215B699BB197F82C3003EB430309EB63
:1071C800C303586946F8220006F0ADF82B7856F844
:1071D800230006F069FA2A780132D2B22A7097F8A9
:1071E8002C300133DBB287F82C3097F82C300B2B7E
:1071F800D0D92368591C21601A70B8F1000F3EF4E9
:1072080044AC1C4BC8F8003001252B46FEF724BCC3
:10721800002D7FF47FAF5946204607F003F8236816
:107228005A1C22601D700F4B26689D683B6A0BEB49
:107238000302AA4240F2FD803B6AED1A07F00EFDF8
:107248002A463146386A07F08FFD236803442360D5
:10725800FEF71BBCD0550020B44A0020583A002045
:1072680058390020A0130020D01E0020636700209A
:107278001467002075C90208543A0020505D0020A8
:10728800304606F091FF326871687B6A9142834606
:107298003DD106461D46FEF7C8BF304606F084FFBE
:1072A800DFF818822BE79A1C32607A4A59781170F5
:1072B800D91C316099785170191D3160DB78937051
:1072C800FEF7E3BB0AEBC80B30468BF8021006F05A
:1072D8006BFF32682AF838001346511C316013F8E6
:1072E800021B8BF80310336053788BF80430D31CDF
:1072F800336093788BF80630131D33600135D278EC
:107308008BF805204D457FF424ADFEF7BEBB511C1C
:10731800316012781D46131C064618BF0123FEF77C
:1073280084BF5A1C194632605B4811F8022BC270A0
:1073380031605B780371042A03D9FF2A7EF464AEB6
:1073480011E756490978994205D8022A7EF45CAEBD
:10735800FF2B7EF459AE236801255A1922601D704F
:10736800B8F1000F3EF491AB4D4BC8F800302B46F6
:10737800FEF772BB3A6AA3EB020807F06FFC4246BD
:107388004946386A07F0F0FC236803442360002D5F
:107398003EF47BABD1E652462BE7304606F004FFBD
:1073A800A884304606F000FF33687268E884D11A72
:1073B80003297FF7E3AD1A46591C316012F8021B06
:1073C800A97732605B7885F82030304606F0ECFE0D
:1073D800336872686884D1E500F07F00032828BF0D
:1073E8000020012524F082FB2B46FEF735BB042A3A
:1073F8007EF44BABFFF70FBA2A4A1368012523F432
:10740800004313602B46FEF727BB27482749284A25
:10741800284B036001250B6013602B46FEF71CBB4D
:107428007D62AA46FEF79ABFDA46C7F824B0FEF78F
:1074380095BF07F013FC5A463146386A07F094FCAA
:1074480023680125034423602B46FEF705BB01256D
:1074580029F0C8F92B46FEF7FFBAC50800F0070364
:1074680001350133EDB2DFF858802846194688F80F
:10747800013016F0A1FCFFF75ABB0F4A9978128821
:10748800012512FB00F22B4692FBF1F2A8F800202E
:10749800FEF7E2BAB7320020D01E002035360020B1
:1074A8008D420108CC3900204C6B0020A06B0020D5
:1074B800086C0020C3C5000884480020604A0020EA
:1074C800005800202DE9F04F2DED068B844B854A9E
:1074D8001C7893B000F59C412031814607911160DA
:1074E800002C00F0B286804A1268904240F2D7839E
:1074F8007E4A029216687E497E4A0191013C1C70C0
:107508007D4B009206F480560493002E40F0D583FC
:107518007A4B1B78022B01F0D780042B01F04281B3
:10752800012B01F0F680764B9945049B9B7800F27D
:107538006085002B40F06185724B0393029B1E68A7
:1075480016F4805740F02186DFF8E491009BB3F9E8
:107558000620019B5D8BAA42B4BF002501256A4B1A
:107568001B68D90040F1B383039B1B7813F0010318
:1075780000F0B4830199498C914241F30C82002DAB
:1075880040F0B383614C94F88C20002A40F0AD831E
:107598005F4A6049106890F82D0000220A604A602E
:1075A8008A605D4A002840F0A1831070002B40F0EB
:1075B800A2835A4B1A78002A79D10199009C488BEA
:1075C800B4F90070898BB4F902408742CCBF802699
:1075D800002646F040038F42A8BF33469B0843F07D
:1075E80080068442C8BF3346009F43F040068C4261
:1075F800B8BF33469B08B7F90440B7F9066043F0B3
:1076080080078442C8BF3B4643F040078C42B8BF5E
:107618003B469B0843F080073C4C8642C8BF3B462C
:1076280043F0400794F88EE08E42B8BF3B469E4533
:1076380001F0F183A4F8902084F89220384984F866
:107648008E300E78002E01F0D7825F2B01F0658313
:107658006F2B01F0A283039B1B78DA0727D494F8D9
:10766800921021BBB4F99030322B20DD94F88E2093
:107678000120572A84F8920001F09C86029B1B681F
:107688005F0741F1FC815A2A41F0F98194F894305E
:10769800002B41F0C88794F8963083F0010384F8F2
:1076A8009630002B42F031800C202AF043FC1D4B11
:1076B80005931D4D029B1B685C0700F1E4860DF1E4
:1076C800400A1A4E06950022CAF804203446109241
:1076D80040F6330B4FF0190840F28337009D2CE039
:1076E800C83000206C300020C4300020105C00201E
:1076F800D05500207278002010570020BE2A0020A4
:10770800404B4C00F7570020344A0020FC1E002054
:10771800D4390020F0470020582500207F5700204A
:10772800C41A002074390020D039002030310020DC
:107738008031002004344C4522D0A178E378994266
:1077480018FB0170F6D294F801E00EF1040E18FB54
:10775800037135F91E305B45A8BF5B46B3F5617F01
:10776800B8BF4FF461739842E4DA9942E2DB2178BA
:107778002729DFD85046043407F00AF94C45DCD1F4
:10778800CB4A069D1378CB4A9AE8030082E80300A7
:10779800002B40F06086C84B1A78002A00F0D88584
:1077A800C64B0693C348012107F001F9002840F0B1
:1077B800EB82049BDB78002B40F0E6822B881FB21B
:1077C80027F001071FFA87F84345A5F8008001F064
:1077D8000180BB4F4FF002090E204FF0140B4FF001
:1077E800FF0A87F8009087F801B087F802A02AF00E
:1077F800A1FB4946AF48B5F8008007F0D8F8002843
:1078080041F05A8228F002039BB243452B800BD0EB
:10781800AB4B02201421FF2218700E2059709A7069
:107828002AF088FBB5F8008018F003011ABF01217F
:1078380008460120FDF764FD24219E4807F0B7F8AB
:1078480030B9039A1378590744BF23F0040313701F
:10785800059B1B6813F00A0F1BD00521954807F0FC
:10786800A6F8002801F06D802F887B0741F1D981A7
:107878009048062107F09BF8002801F04F80780611
:1078880041F1C78107218B4807F091F8002840F0A3
:10789800ED870C21874807F08AF82A88002800F02D
:1078A8007C8342F480739A422B8009D0844B022750
:1078B8001421FF220E201F7059709A702AF03AFB8B
:1078C800804B1B78082B00F074830E2B00F071831B
:1078D800029BD3F8008018F4806F12D07A4B1B7982
:1078E800002B00F033821421724807F060F800285A
:1078F80040F031821AF07EFF17F064FD029BD3F846
:107908000080039B93F80090704B19F0010900F078
:10791800C58201221A70069B00991B68B1F90610EE
:107928005A896B4801279142077080F27682694B29
:107938004FF07E521A60019B674FB3F818A0009B66
:1079480097F90420B3F90030387897F801C0002A75
:10795800A3EB0A0714BF01224FF0FF32002FB8BF74
:107968007F42B7F5FA7FA8BF4FF4FA77B84280F2A2
:1079780051823F1A07EE907AF8EEE77A574F9A4508
:10798800C7ED007A03DDF1EE677AC7ED007A009B58
:10799800B3F902E0AEEB0A03002BB8BF5B42B3F5C4
:1079A800FA7FA8BF4FF4FA73984280F230821B1A0C
:1079B80007EE903AF8EEE77AF245C7ED017A03DD73
:1079C800F1EE677AC7ED017A009BB3F90400A0EBEA
:1079D8000A03002BB8BF5B42B3F5FA7FA8BF4FF488
:1079E800FA736345CCBFA3EB0C03002302FB03F33C
:1079F80007EE903AF8EEE77A5045C7ED027ABCBF39
:107A0800F1EE677AC7ED027A18F4805200F0DA8155
:107A1800B1F5FA6F324BA8BF4FF4FA61B1F57A7F2E
:107A28001878B8BF4FF47A71A1F57A71002840F040
:107A3800E481DFF8BCE02B488EFB013CCB17C3EB9D
:107A48006C1303F1010C6FF0630830F91CC030F9B6
:107A5800130008FB0313ACEB000103FB01F38EFBDF
:107A6800031EDB17C3EB6E1303441BB207EE903AF9
:107A7800B8EEE78A87ED038A002A40F028842B882D
:107A88005A0640F101811849184A91ED018AD2ED50
:107A9800019A92ED026A91ED034A92ED030A91ED83
:107AA800029A92ED007AD1ED005AD7ED011A21E041
:107AB800985E0020344A00209D560020D8390020C6
:107AC8001C2A0020B44A00208C370020F8570020D8
:107AD800902500200C250020684A00209C370020B3
:107AE800C43A0020BC6800206C1A00207C1A0020D0
:107AF8001F85EB5197ED002AD54AD64938EE445AEE
:107B080079EEC63A77EE007A65EE233A75EEC96AE1
:107B180075EE890A37EE401A66EEA76AB0EE633A48
:107B2800A0EE813A13F00303B0EE665A78EE044AE9
:107B380079EE867AA0EE815AF0EE638AA4EEA73A2F
:107B4800D4EEA78AA4EEE75A33EE263AF0EE687A26
:107B5800F0EE674AF6EE008A35EE88AAE0EEC14AF2
:107B680028EEC33A35EE635A77EE293A77EEE67A8D
:107B7800AAEE233A25EE285A76EE403A34EE49AA80
:107B8800E0EE817A74EEA64AAAEE235A34EE094A48
:107B980037EE697A64EEA84A63EE036AE4EE074AB0
:107BA80075EEC85A36EE006A67EEA87AB0EE667AC5
:107BB80095EE057AE5EE056AE5EE867AB1EE648A19
:107BC800F0EE665AF0EE476AB1EE674AE8EE246ACC
:107BD80063EE270A67EEA43AE4EE275AB1EE450AA7
:107BE800B0EE609AB0EE631AA4EE277A23EE244A28
:107BF800E7EEA76AA5EE249AA0EE031AE8EE245A47
:107C0800B0EE448A31EEA16AE0EE240AA5EE278A96
:107C180066EEA16A72EE028AE5EE033A61EE211A77
:107C280026EE096AA4EEA47AA0EE274A0CBFD7ED87
:107C3800022ADFED892A82ED005AA2EE256AE8EED3
:107C4800A06AE2EE081A73EEA33A27EE227A34EE1F
:107C5800044AF0EE005AE3EEA26AA4EE226AA1EE0C
:107C6800A57AC7ED016AC1ED366A81ED356A87EDFF
:107C7800006A81ED377A82ED013AC2ED027AC2EDEF
:107C8800034A0BB987ED027AB9F1000F40F0A481DD
:107C980026F0C2FD13B0BDEC068BBDE8F08F6F4B2C
:107CA80002931E686E4B6F4A009306F480566E4B23
:107CB80001920493002E3FF42BAC00216B4806F090
:107CC80076FE00287FF424AC22F07CFF20E47302C7
:107CD8003FF54AAC039B1B7803F001035D4C00227F
:107CE80084F88C20002D3FF453AC614A01211170B7
:107CF800002B3FF45EACF6067FF55BAC5D4B1B7862
:107D0800DC063FF556AC002F7FF453AC26F022FB7F
:107D180000287FF44EAC584B1B78002B01F06A8486
:107D2800564B9B78002D41F0CE843BB1544A554BBD
:107D380012681B689B1A002BC1F2D6841020454C90
:107D48002AF0F8F8012384F88D3032E4039B1B787D
:107D5800D9077FF5CFAD4FF40F7029F0BBFB002892
:107D68003FF4CCAD17F054FC4FF40F7029F054FBDE
:107D780000283FF4C3AD17F04BFC4FF40F7029F007
:107D88004BFB0028EED1B9E5059B1B6898077FF5EA
:107D980015ADB5F8008018F0010F7FF433AD48F049
:107DA800010398452B803FF42DAD374B0222142157
:107DB8001A700E20FF2259709A702AF0BBF8B5F895
:107DC80000801FE5019B588B8142C0F2F984B1F510
:107DD800FA6FD4BFC0EB0101C0F5FA614FF47A73B2
:107DE80003FB01F1294B93F800E0C0F5FA60B1FB01
:107DF800F0F1BEF1000F3FF41CAE5B78244801FBA4
:107E080003F380FB0301DB17C3EB611111E6DFED20
:107E1800127AD1E5DFED107AB0E5B1F5FA6F80F2AC
:107E2800D284187A8B1A03FB00F3C2F5FA6293FB2B
:107E3800F2F3C3F1640307EE903AF8EEE77A9FEDA8
:107E4800157A154B67EE877AC3ED007A73E500BFA4
:107E5800B41A0020FC1E002000000000105C002066
:107E680072780020D055002010570020344A002096
:107E780058250020587A0020C41A0020904A002073
:107E880078690020E46500201C2A0020C43A0020FC
:107E98001F85EB510AD7233C0C2500201B78029341
:107EA800002B7FF438ADBE4A1268002A3FF433AD88
:107EB800BC4A039212F8030CDFF838B31146D71EF8
:107EC80026F01EFA9BF800A0039A002800F07E8591
:107ED800029BBAF1000F41F0378307F10801787966
:107EE80026F00EFA002841F04383AF49B87A26F00D
:107EF80007FA002800F07D85BAF1020F41F04483AB
:107F0800AA49F87B26F0FCF9002841F03983A849F2
:107F1800387D26F0F5F9002800F07D85BAF1040FC8
:107F280041F04283A349787E26F0EAF9002841F01F
:107F38003783A149B87F26F0E3F9002800F07D8552
:107F4800BAF1060F41F028839C4997F8230026F0E0
:107F5800D7F9002841F01C83994997F8280026F0A2
:107F6800CFF9002800F07D85BAF1080F41F00483AD
:107F7800944997F82D0026F0C3F900283FF4CBACBC
:107F88000922134602EB820217448F4A7878B9789F
:107F98008BF8003010705170BDE422F480739BB2EE
:107FA8009A422B807FF482AC884B1B78082B7FF495
:107FB8008CAC2A8822F040039BB29A422B803FF473
:107FC80087AC834B02271421FF220E201F705970A3
:107FD8009A7029F0AFFF7BE47E4A7F4B11781868CE
:107FE80001F0010105F065FB13B0BDEC068BBDE89F
:107FF800F08F13B9049A01239370784B049A1D7873
:1080080092F8214003931B2026F0B2F9012C05F0C9
:108018000108814600F09A8605F00205049A704E20
:1080280092F82030DFF8D0A16E4F05959346052BC6
:1080380000F20987DFE813F08E0084000600FA00DA
:10804800FC00EF00012C04BF05238BF82030B8F1A9
:10805800000F12D0019B3088B3F918100022134684
:1080680061F30F0260F31F4261F30F03009861F39D
:108078001F4303600323426005935B4DDBF8141034
:108088002A68914280F07F8547F230510322CBF86D
:108098001C108BF8202002200DF02EF922F092FD02
:1080A8002968DBF81C200A440421CBF818208BF837
:1080B8002010012C40F03E872A68DBF81810914206
:1080C80080F0C1869AF8000020B926F051F90028FE
:1080D80040F0B9863A6822F002023A602A6873884A
:1080E800642101FB03234FF480600022CBF8103099
:1080F8008BF820208BF803200DF0CEF89BF8203069
:1081080095E726F03BF9012807D1374D72882B688F
:10811800642101FB0233CBF81030B9F1000F02D013
:10812800B379002B79D1012C00F08D862E4DDBF828
:1081380010102A689142C0F0CC8601238BF82030B9
:10814800012C68D0F379012B74D026F097F89BF8AE
:1081580020306CE7B8F1000FD3D1059D4FF4806053
:10816800B9F1000F00F049830DF0AEF8049A00232E
:108178001361002D3FF4E2A9284629F0DBFE029B9B
:108188001E6816F480573FF4DFA91D21174806F032
:108198000EFC00287FF4D8A9154B03F1500931E0F3
:1081A800FC570020EA290020F4290020F9290020A2
:1081B800FE290020032A0020082A00200D2A00207A
:1081C800122A0020172A002000580020B44A002054
:1081D8001C2A00204069002044690020F75700202D
:1081E800B4680020CC39002078690020344A002087
:1081F8003031002000000020C41A002004339945C3
:1082080000F027861A78262AF8D19978DA789142E8
:10821800F4D2FFF79BB9AE4D60E726F02FF80322A2
:108228004FF47A738BF82020CBF81C30A84D32E736
:10823800A74D3EE726F022F8032240F6B8338BF824
:108248002020CBF81C30A24D25E7A24F3B78002B0D
:1082580001F0EA80A04BDFF8A482DFF8A4B2DFF8CF
:10826800A4A2019345465E46009099460EE019F88F
:1082780004109847032C28DC88B93B782AF8020FA9
:1082880001349C4205F1040580F24481072CE1B2D7
:108298003046DBF80430EADD984700B2EDE738F8FD
:1082A80024206B88801A4FF47A719B1A01FB00F026
:1082B80040F6CA0290FBF3F00844904240F2EE23E5
:1082C800A8BF10469842B8BF184600B2D5E71D218E
:1082D800824806F06CFB28B100F077BD0436A64250
:1082E8003FF4CDAB31782629F8D1B278F3789A42A9
:1082F800F4D2049BDB78002B7FF4C1AB774806F0FF
:1083080056FBDFED777A002801F0928038EE678A15
:1083180074487549FDEEC87ACAF57A73CDED007ACE
:10832800BDF90020120380FB0240D2171BB2C2EB3A
:10833800A01203FB02F343F30F33534407EE903AC2
:10834800F8EEE77A0123C7ED037A0B70FFF797BBC6
:10835800DFF8B491DFF8B4A1644F069209F15A0826
:108368004FF0010B494619F8010C25F0C9FF00B37D
:1083780099F8040099F8023099F803E000EB4001FD
:1083880007EB8101013BD1F8A02003EB43035344E1
:1083980093420ED097F8CC20C1F8A0300BFA00F029
:1083A80022EA0000069B81F89CE0C1F8A43087F817
:1083B800CC0009F10609C145D4D14D4B444A069376
:1083C80019464C4BDFF848A1126809681B780891D8
:1083D8000793AAF19C094FF0000B9046DAF8043095
:1083E80083B31F7877B3DAF80820A8EB0202002AD3
:1083F8000CDB99F8CC20012101FA0BF122EA0102E9
:1084080008F5FA7189F8CC20CAF80810079ACAB199
:108418009AF8002059780432D2B2002940F0C1827B
:1084280001990098098B30F9122001F1C8008242A5
:1084380040F3218599F8CC109A7841FA0BF3D907C3
:1084480040F1A8850BF1010BBBF1040F0AF10C0AEE
:10845800C4D1FFF7A7B9284B03E004339C423FF48B
:108468009AA919782329F8D19878DA789042F4D221
:108478001A4806F09CFA00283FF48DA9142029F028
:1084880059FDFFF788B9194C94F896305BB1039BF6
:108498001B78D80707D5009BB3F90620019B5B8B97
:1084A8009A4200F3698511210C4806F080FA0028E9
:1084B80000F05F8294F89A302BB994F8943013B98D
:1084C8003223A4F89830012384F89A30FFF7F7B8DC
:1084D80078690020F8310020D0550020344A002067
:1084E80000007A44D34D621084250020FC1E002031
:1084F800D83900208D4C0020303100200C3200206B
:10850800F8560020FA1E002001290020BC55030857
:10851800981F0020DDF80090B94A0292B949126804
:1085280042F2010AA1FB091B12EA0A0A4FEA9B1B45
:1085380000F01C82B44DB548B54CB6492E78007889
:10854800267008701EB1B3490E7886F00106B24C49
:108558000F2184F82410002B00F08083019DAF4B7D
:10856800B5F826C0B5F824E0019D0C9318462D8B6C
:108578000078AB4B0E9594F825500595A94D0095BC
:10858800A3FB00535B0803EB4303C31ADBB20B9056
:10859800CDF824C002F48052089304F128000BF5AA
:1085A8009673CDF8349097F80080DDF81490DFF8D2
:1085B800B4C205949B4C0A910F920021069304962D
:1085C800CDF80CE0049B002B00F07F82059B039DF7
:1085D80033F911201FFA82FEAE454FEA410303D357
:1085E800099DAE4540F2B6825CF82120934580F0A3
:1085F8007682E25EBAF1000F40F08B82013141458C
:10860800E25200F10600DDDB0A9A059C864B84F8ED
:1086180024200F2A49460CBF01220022DDF834909D
:1086280084F825101A7000F02083804B7749794A26
:10863800DFF834B204931C46042001230B70137036
:108648000CF05AFEDBF80030A1686268E3605B1A40
:10865800934284BF002384F82130029B3C781E6833
:10866800002C00F01987019A714DB2F824E0178B9D
:108678006C4916F48056284640F0318332460EE0A5
:10868800437803EB830303EB830303F2EE239BB2EC
:108698000132A24221F8023B00F102000ED015F887
:1086A8001230002B00F05A82022BE9D001320B88DD
:1086B80021F8023BA24200F10200F0D10C9A137893
:1086C80001331370FEF721BF019A0099537DD27DC3
:1086D800013B31F913301AB1C3F53B6308331BB2C0
:1086E800A3F57A7307EE903A9FED527A524AF8EE64
:1086F800E77A40F2FF3167EE877AFCEEE77ACDED54
:10870800037ABDF80C308B4228BF0B461380FEF766
:108718000ABF414CD4F88830A9EB0303002BFEF6BE
:1087280002AF464A464B527C019933F812308A7D93
:10873800DFED446A9FED446AC97D9BB207EE102ABB
:1087480007EE903AB8EEC77AF8EEE77A27EE267A7F
:1087580067EE867A079AC4F88820C7EE876A40F2DF
:10876800FF32FCEEE67ACDED037ABDF80C30934289
:1087780028BF134609B1D31A9BB23448344D017847
:10878800344C35F81160226825F81130921B1344D7
:108798000131294D236001F00F021B0902702B8063
:1087A800FEF7C1BEFCF77CFA2B4B2C4A1B68C31A98
:1087B80093427EF7B8AE204B00221A80FEF7B3BE74
:1087C8001146FFF70FBB1B7AC3F1640307EE903A1B
:1087D800FFF733BB0221224806F0E9F800283FF4EE
:1087E80011A82F8018F0020F7FF41EA802200CF0A9
:1087F8006BFDB5F80080FFF717B80CF04DFDB5E438
:10880800105C0020D34D6210483000201800002072
:108818008D4C002019000020FC1E0020E5300020AF
:10882800ABAAAAAA727800209E57002010570020F1
:10883800403200206F12833F504D0020F068002026
:10884800106900200000C84200008044BF2A0020B0
:10885800C42A0020C02A0020E81E002060E3160079
:10886800344A0020E830002078690020CE4AB2F966
:108878000030002BB8BF5B42B3F5E17FBFF609A813
:10888800B2F90230002BB8BF5B42B3F5E17FBFF607
:1088980000A8C64B93ED057AD3ED077AD3ED096AA4
:1088A80093ED030A77EEA67A30EE070AF7EE000A90
:1088B800B0EE007AE7EEC70A30EE000A05F03CFE9B
:1088C800B6EE008A20EE488A9FEDB90A38EE000A13
:1088D800FDEEC07A17EE903A2033402B40F24983E0
:1088E8009FEDB40AB44FDFEDB37A87ED000ABDEE11
:1088F800C87AC7ED017A17EE103A2033402BC7ED3E
:10890800027A00F27E85B0EE480A05F09BFD0A2047
:1089180087ED030A29F00EFBFEF7BBBF27F04003E3
:108928009BB2BB422B803EF4ADAFA44B022714216F
:10893800FF220E201F7059709A7029F0FBFAFEF77B
:10894800A1BF2B8823F00407BFB2BB422F803EF49F
:108958008FAF9A4B02201421FF2218700E205970F5
:108968009A7029F0E7FA2F88FEF782BF94490E78AB
:10897800E8E594F89430002B3EF4A1AE039B1B78F5
:1089880013F001037EF49BAE012284F8943084F83E
:108998009520FEF794BE8B4C012284F88C20FFF7BB
:1089A800A4B9012900F0CA8499F8CC20012303FA5C
:1089B8000BF30BF1010B1343BBF1040F89F8CC3017
:1089C8000AF10C0A7FF40AADFEF7ECBE511D787966
:1089D80025F096FC00283FF488AABAF1010F40F070
:1089E800C78507F10D01B87A25F08AFC002840F008
:1089F800CB857549F87B25F083FC00283FF487AACE
:108A0800BAF1030F40F0BC857049387D25F078FC39
:108A1800002840F0C9856E49787E25F071FC002851
:108A28003FF487AABAF1050F40F0BA856949B87FC3
:108A380025F066FC002840F0AF85674997F82300C9
:108A480025F05EFC00283FF487AABAF1070F40F032
:108A58009F85624997F8280025F052FC002840F0CD
:108A68008B855F4997F82D0025F04AFC00283EF4D5
:108A780052AFBAF1090F3EF44EAFFFF781BA5D2A43
:108A880000F08D825B2A00F0F4845E2A00F04085B5
:108A9800562A00F05E85972A00F06185A72A00F023
:108AA8002D85504D2B889E0740F0FA84A2F1B7031C
:108AB800072B00F29E82DFE813F080029C029C02E2
:108AC8009C028E029C0287029502039B002B3FD0DA
:108AD8005CF8212093454FEA4103FFF48AAD424AEE
:108AE800414DD25C05EB030E002A00F0D780022A24
:108AF80047D19EF8012002EB820202EB820202F2C9
:108B0800EE2292B2032933DD12B2BAF1000F3FF41C
:108B180075AD089D20F81520B9F1000F03D10B9D04
:108B2800022D7FF66BADB0F802900288B0F804E031
:108B38004A4496442D4A0FFA8EFE82FB0E522C4D63
:108B4800A2EBEE7225F803E012B24FF0010955E5E9
:108B58001A464B00069D4CF821504BE5D3B2022B28
:108B680004D9032B7FF4A2AD734691E53B468FE50C
:108B7800012505FA01FE0A9D25EA0E0512B20A959D
:108B880038E5E25ABEE71B4A1278002A7FF47CAA2D
:108B9800B8F1000F3FF478AA012C40F054819BF8FB
:108BA8002030FFF744BA00BF803900208C1A00201B
:108BB800DB0FC93F000000006C1A00201C2A0020AF
:108BC8008D4C0020FC1E0020F9290020FE290020E1
:108BD800032A0020082A00200D2A0020122A00203B
:108BE800172A0020D039002040320020565555550C
:108BF8006C1F0020482500203146BB4805F0D7FEF1
:108C0800002800F0A68084F8936022F0C7FAFEF7E7
:108C180022BD47F04003BB422B807FF486AEFEF7AF
:108C280031BE47F004039F422B800AD0AF4B02208D
:108C38001421FF2218700E2059709A7029F07AF9C1
:108C48002F88AB4BAB4AB3F90430AB4982FB030224
:108C5800DB17C3EBA2030B80FEF70ABEA74BA84A9B
:108C68000C9201221A70A74B00931B219E4805F015
:108C78009EFE00287FF4D9ACA34BDFF8B4B204936E
:108C88001946DBF80030CA688B609B1AC82B00F2C3
:108C9800F483029B1E6806F480560FE5CAB2022AC6
:108CA80040F24983032A7FF46CAF0E9A0F9D039E0E
:108CB800002D08BF324625E728F001039BB2434543
:108CC8002B803FF48FAD0E2087F8009087F801B015
:108CD80087F802A029F02EF9B5F8008082E5002275
:108CE8000FE0437803EB830303EB830303F2EE23E4
:108CF8009BB20132A24221F8023B00F102003FF48C
:108D0800DDAC15F812301BB1022BEAD00B88F0E766
:108D1800D3B2032BFAD83B46EBE7B2F5FA7FFEF65F
:108D2800C6AC94F89230002B7EF4C1AC039B1B7840
:108D3800012213EA020584F8922000F0568321F0FC
:108D480041FF724B0593724DFEF7B4BC0025FFF747
:108D580065B9039B6F4A1B781060D8077EF57FAC16
:108D68006D4B1B78002B3EF4A2AC049BDB78002BE8
:108D78007EF49DAC94F893300133DBB2032B84F876
:108D880093307EF694AC654B5B7813B9002D7EF476
:108D98008EAC21F017FFFEF75EBCB2F5FA7FFEF647
:108DA80086AC94F89230002B7EF481AC039A12784A
:108DB800012184F89210D10700F1278322F0EEF9FF
:108DC800524B0593524DFEF775BC049BDB78002B84
:108DD8007FF488AADFED527A524938EE678ACAF5DD
:108DE800FA63FDEEC87A1BB2CDED007ABDF900201A
:108DF800120381FB0201D217C2EBA11203FB02F39B
:108E080043F30F33534407EE903AB8EEE78A87ED01
:108E1800038AFFF767BA444A42491068B4F99020B8
:108E2800C66981FB06018911F617701A00F5FF4023
:108E38007F3082423EF702AC891B0A4412B2A4F882
:108E48009020FEF7FBBB059D002D3EF477ABFFF7A6
:108E580093B9364A019BD588009A1B8BB2F9062034
:108E6800591B8A4240F382802B449A42B4BF0025A2
:108E78000125FEF774BBC8398A4268DA99F8CC1024
:108E88009A7841FA0BF3DB073FF5DCAA524201203E
:108E9800099229F035F97B1E099A162B00F21981DF
:108EA800DFE813F05A016D014201900180012E01A3
:108EB8001A01CE01B901F201A401170190010901BB
:108EC8002E011A01CE01F500E100CF0033021C0289
:108ED800070225F0D3F9032140F6B8328BF82010A9
:108EE800CBF81C20FFF7D7B8344A00201C2A0020F2
:108EF8008039002067666666862500209E57002018
:108F0800E5300020727800201057002074390020C6
:108F1800D0390020E86500208D4C0020904A0020C0
:108F280000007A44D34D62100C530020986800204A
:108F380078690020AB460499DBF80020CB69059DD1
:108F480013448B61002D3EF4F9AAFFF715B999F87F
:108F5800CC30012202FA0BF223EA020308F5FA7276
:108F680089F8CC30CAF80820FFF76CBA0125FEF75B
:108F7800F6BA05F067FAB5E40021BC4805F017FD1C
:108F880000287FF490AA322384F89600A4F8983039
:108F9800FFF789BA002A0CBF0120022078E7B44BFA
:108FA80000220120B349B44C0B60B44B22700593E6
:108FB800B34D29F0A5F8FEF77DBB012022F096FD00
:108FC800AE4B0593FEF776BB032022F08FFDAB4B2B
:108FD8000593FEF76FBB002022F088FDA74B059391
:108FE800FEF768BB022022F081FDA44B0593FEF733
:108FF80061BB792A00F058837A2A00F04C839E2AB4
:1090080000F042839D2A00F03883AE2A00F02E83B8
:10901800AD2A00F02483EF2A00F01E83FD2A00F019
:109028000B83FB2A00F07F83FE2A00F07983F72A5E
:1090380000F073837B2A00F04083904B0593FEF782
:1090480039BBD9F8D0008F4B81781144C829A8BF03
:10905800C82121EAE17181709B78002B40F03E83A2
:1090680027F0DCFBA0E4D9F8D000864B4178114406
:10907800C829A8BFC82121EAE17141709B78002B5B
:10908800EED0132025F0BEF9D9F8D000E8E7D9F8DA
:10909800D0007C4B01781144C829A8BFC82121EA17
:1090A800E17101709B78002BDAD0122025F0AAF923
:1090B800D9F8D000D4E7734B08989B7841791144CC
:1090C8006429A8BF642121EAE1714171002B40F0B5
:1090D8002D83D9F8D000C3E7D9F8D000694B0179BE
:1090E80093F802E01144C829A8BFC82121EAE17118
:1090F8000171BEF1000F40F01F83102FB6D1AFE70A
:10910800D9F8D0005F4BC17893F802E01144C82920
:10911800A8BFC82121EAE171C170BEF1000F40F07B
:10912800EA820F2FB6D19BE70899564B0F7909931E
:109138001744642FA8BF642727EAE7770F7125F043
:109148007BF9099B9B78002BC3D00320394625F077
:1091580059F9D9F8D00083E708984A4B01781144A7
:10916800FA29A8BFFA2121EAE17101709B78002B46
:10917800AFD0012025F046F9D9F8D00070E708985B
:10918800404B817811446429A8BF642121EAE17128
:1091980081709B78002B9CD0022025F033F9D9F8F8
:1091A800D0005DE70898374BC1799B78114481F36B
:1091B8000801C171002B8CD0052025F023F9D9F8BE
:1091C800D0004DE708982F4B817993F802E01144BD
:1091D8006429A8BF642121EAE1718171BEF1000F01
:1091E80040F0B4820D2F7FF467AF72E7D9F8D00052
:1091F800244B017A9B781144C829A8BFC82121EAC9
:10920800E1710172002B3FF42BAF0B2025F0FAF827
:10921800D9F8D00024E7D9F8D0001A4B81799B7887
:109228001144C829A8BFC82121EAE1718171002B26
:109238003FF416AF092025F0E5F8D9F8D0000FE77C
:10924800D9F8D0000F4B417993F802E01144C829AE
:10925800A8BFC82121EAE1714171BEF1000F40F0B9
:109268007D82112F7FF4F0AEFAE600BF344A002069
:10927800CC320020D4390020B856002074390020A0
:10928800D0390020EC330020D9F8D000C84BC17980
:109298009B781144C829A8BFC82121EAE171C1718E
:1092A800002B3FF4DDAE0A2025F0ACF8D9F8D00049
:1092B800D6E6D9F8D000BE4B90F836109B7811440A
:1092C8006429A8BF642121EAE17180F83610002BD7
:1092D8003FF4C6AE172025F095F8FAE6D9F8D00085
:1092E800B34B90F837109B781144FE29A8BFFE2194
:1092F80021EAE17180F83710002B3FF4B1AE162057
:1093080025F080F8D9F8D000AAE60898A84B41784B
:109318001144B1F5967FA8BF4FF4967121EAE17127
:1093280041709B78002B3FF4D4AE152025F06AF8E5
:10933800D9F8D00094E60E9AFFF7E4BB00999B7821
:1093480031F91220B2F5617F4FF4966191FBF3F386
:1093580062DB40F633019142A8BF11460C2FA1F5FC
:10936800617191FBF3F100F0F280182F7FF41CABD0
:10937800C9B2C8290B46A8BFC823D9F8D020D77DC1
:10938800D8B2B8423FF410ABDF1B894BD07548BF49
:109398000737FF109B780137FFB23BB9002F3FF426
:1093A80003AB384628F0ACFEFFF7FEBA182025F0CC
:1093B80029F8F3E77F4A804B059210461A687F49DF
:1093C8004FF47A73B3FBF2F3C3EB431203EB82035C
:1093D8000268DB00A1F8A83053077EF56AA9784B2C
:1093E800784D0A221A80FEF765B90F2028F0A2FDF1
:1093F800B4F8903084F89250FA3BA4F89030FEF715
:1094080056B9B0EE670AFFF782BA6F4A6949059103
:1094180013606C4DFEF74EB90C2F7DD0182F7FF4DA
:10942800C3AA00210B46A8E7684A0192FFF774B85F
:1094380038EE678A664B67491870FDEEC87ACAF538
:10944800FA63CDED007ABDF90020120381FB020119
:10945800D217C2EBA1121BB203FB02F343F30F3383
:10946800534407EE903AF8EEE77AC7ED037AFEF731
:1094780006BB594B0122022094E5584A029B1E68FC
:10948800136823F004031360049A012306F480563A
:1094980082F82130FFF712B906F48056FFF70EB9AB
:1094A8000023BB2A109300F0BB80B72A00F0B480D9
:1094B800BE2A00F0AF80BD2A7FF49BAD4FF6FE7147
:1094C800474A3C48D6890590908933440144D38162
:1094D800918111F0BBFD04F0F5FA11F09FFDFAF748
:1094E800D7FC012028F00CFEB4F890300022FA3B9B
:1094F800A4F8903084F89220FEF7DCB8394A2D4B56
:10950800059313782F4D43F004031370FEF7D2B878
:10951800354B0222032045E500273946334B0A9193
:109528005B78BB423FF440AA214B0993384622F0AE
:10953800DDFA099B0A999B781BB1C9B20C2024F06B
:1095480061FF0137FFB229E71A46FEF71BBDCFB20C
:10955800E4E7FAF735FE94F88E20FFF79CBA154A2F
:10956800234B05924FF4C8721A80164DFEF7A2B825
:1095780001221346FEF706BD08221346FEF702BD78
:1095880003221346FEF7FEBC02221346FEF7FABC7E
:1095980007221346FEF7F6BC06221346FEF7F2BC76
:1095A80005221346FEF7EEBC04221346FEF7EABC7A
:1095B800EC33002074390020005C00201053002098
:1095C800D6680020D0390020E8650020D05500205A
:1095D80084250020D34D62101A330020CC39002096
:1095E800704A0020587A002068330020B8560020BE
:1095F800D8680020002D3EF4A1AB5D4C94F88D3066
:10960800002B3DF4D6AF28F079FC002384F88D3088
:10961800FDF7CFBF022153E719464FF6FE734FE718
:10962800194602234CE7534B84F8941084F89500AC
:109638000593514DFEF728BF0021012022F07EF945
:10964800B4F890304B4A0592963B0022A4F890302B
:1096580084F89220FEF72EB800210846EEE7FF2195
:1096680000201DF0F7F894F88E20D4E401210020A2
:109678001DF0F0F894F88E20CAE40021FF201DF0B8
:10968800E9F894F88E20C0E4002101201DF0E2F8EA
:1096980094F88E20B6E4394A364B0593137A43F092
:1096A80001031372FEF706B8344A324B0593137A56
:1096B80023F001031372FDF7FDBF4FF4FA61022096
:1096C80022F03CF9B9E4002B97D02D492D4A0968BE
:1096D8004FF47A7000FB031313608EE7142024F014
:1096E80091FED9F8D000BBE4214C21F06BFA84F844
:1096F8008D50FDF75EBF0F200A93099224F082FE79
:10970800D9F8D0000A9B099A0BE50B2028F012FC27
:10971800184B0593184DFDF7CDBF002104208DE7A8
:10972800002103208AE70021022087E70E2024F089
:1097380069FED9F8D00093E410200A93099224F026
:1097480061FED9F8D0000A9B099AD6E40D200A9345
:10975800099224F057FE0A9B099A43E511200A93BF
:10976800099224F04FFED9F8D0000A9B099A78E5AF
:10977800FC1E002074390020D039002084570020B6
:1097880078690020E46500202DE9F047C74C63683C
:1097980020469847002800F0C380C54B1B7801225B
:1097A800042B84F83C2000F0BD80B4F91610B4F9FD
:1097B8001820B4F91A3021636263A363BD4B1B8878
:1097C800002B69D0BC4DD4ED0C7AD5ED004A95ED4F
:1097D800050A95ED015A95ED067AD5ED035A95EDF2
:1097E800026AF8EEE76AD5ED047AA4EEA60AA5EEB9
:1097F800267A67EEC07AA5EEC07AE6EE267A85ED7F
:10980800057AC5ED067A2AF037FCD4ED0D6AD5ED58
:10981800094A95ED0E0A95ED0A5A95ED0F7AD5EDA0
:109828000D7AD5ED0C5A95ED0B6A2063F8EEE66AD1
:10983800A4EEA60AA5EE267A67EEC07AA5EEC07A4F
:10984800E6EE267A85ED0E7AC5ED0F7A2AF014FC3D
:10985800D4ED0E6AD5ED124A95ED170A95ED135A17
:1098680095ED187AD5ED167AD5ED155A95ED146A59
:109878006063F8EEE66AA6EEA40AA6EE857A67EEBD
:10988800C07AA0EE657AE6EE867A85ED177AC5EDA0
:10989800187A2AF0F1FBA063884FA17F88480FF05F
:1098A800C1FE3B88002B40F08480864ED6F8E050FD
:1098B800854B1B685B0743D4B5F90070216B636B5C
:1098C800A06B824A824E92ED026AD2ED006AD2ED16
:1098D800015AC91B2163B5F90270DB1B6363B5F933
:1098E80004703568C01B07EE900AB8EEE75A07EE19
:1098F800901AB8EEE77A07EE903AF8EEE77A36EE85
:10990800056A36EE877A77EEA57A0135A06382ED8F
:10991800026A82ED007AC2ED017A3560BDE8F0870F
:10992800BDE8F0876B4BB4F91600B4F91810B4F918
:109938001A2018802063598061639A80A2633DE7EA
:10994800B6F89820322A00F08880002A66D196F866
:109958009530002BB0D06048D6F8FC205F4980FBDA
:109968000273D217C2EB23122A80D6F8002180FB9B
:109978000273D217C2EB23126A80D6F80431A78A81
:1099880080FB0302DB17C3EB2213DB1BAB80002336
:10999800CB6086F8953011F059FB04F093F811F07C
:1099A8003DFBFAF775FA012028F0AAFBD6F8E0503B
:1099B80082E7444E226BD6F8E050B3F5C87F4FF0EB
:1099C800000323632B80398818BFD6F8E400B7F862
:1099D800008008BF0020B1F5C87F18BFD6F8E8306E
:1099E800616B02440B440020B8F5C87F6063C6F879
:1099F800E420C6F8E830688052D0D4F838E0D6F8C9
:109A0800EC10A0637144B8F1010FA880C6F8EC10FF
:109A180068D008F1FF38A7F8008049E7D6F8FC00BD
:109A2800236B00210344C6F8FC3021632980D6F853
:109A38000001636B61630344C6F800316980A36B5E
:109A4800D6F80401A1630344012AC6F80431A980A9
:109A580075D0013AA6F8982079E72B8820491F4845
:109A6800276BA6F8F0300023B5F802E0B5F804C07B
:109A7800C0684B608B602363C6F8FC702B80616BF9
:109A8800C6F8001163636B80A16BC6F80411A36369
:109A9800A6F8F2E0A6F8F4C0C6F8F800AB80D8E75C
:109AA800A36BC6F8EC30A063A880B2E78839002021
:109AB80054360020382E00203C2E0020D868002084
:109AC800B8390020FC1E0020105C0020A46700208C
:109AD800A0670020583600201F85EB51704A0020EF
:109AE800F81F0020DFF88CC0DFF884E0C8328CFB58
:109AF80002A9C833D217C2EBE9128CFB03A9DB1702
:109B0800C3EBE913C8316B802A808CFB013CA28A25
:109B1800CB17C3EBEC139B1AAB80CEF80C0011F0FB
:109B280095FA03F0CFFF11F079FAFAF7B1F9404648
:109B380028F0E6FAB7F80080D6F8E05069E70B207D
:109B480086F89A1086F8942028F0F4F9D6F8E050B0
:109B5800074BB6F8F020B6F8F270B6F8F400D6F86D
:109B6800F8102A806F80A880B6F89820D96070E72E
:109B7800704A00201F85EB512DE9F0478C4B1B786C
:109B8800DB07074644D58B4B8B4D1C788B4E012C3D
:109B980059D01CD3022C07D189498A4A09881288CE
:109BA800914201D901241C70EB7AE3B12B89D3B11E
:109BB800854B1B78BBB115F093F9002800F09B800A
:109BC8002B7B83422CBF0121002131700CE07C49A2
:109BD8007E4A098810886A7B801A8842E2DAEB7A22
:109BE8000024002BE2D131782A79632A06D8022C86
:109BF800774E00F0BA803378002B5DD1754AAB7A86
:109C08008C4238BF0C461470002B4CD1BDE8F0874D
:109C18006B4B694D19885B88E878CB1A83EAE37245
:109C28008142A2EBE3721DD32B788B421AD3614B8E
:109C38001C78E01E012861D96749097802294FD0AC
:109C4800012C5E4EA5D15F4A5D491288687B098860
:109C5800121A914239DD5D4A12888A42A4D2002440
:109C68001C70A1E7B1EB400FE1DC524B1C78E11E00
:109C7800012940F29480022ADEDC57494F4E0878C9
:109C8800DFF84481DFF844C1DFF838E1002103241C
:109C9800022834701C7088F80010ACF80010AEF878
:109CA800001081D11FE0012C71D0022C0BD10720AC
:109CB800BDE8F04728F03EB97068381A474B98421B
:109CC80058DD72709AE7BDE8F08702241C706BE7D4
:109CD800022AD2DD4049097802294FF0040464D1F0
:109CE8003949364E09783E48022ACCBF0022012263
:109CF800C28081804BE70221317075E7022A9BDC24
:109D080095F800C091FBFCFC0CF1010CBCF1080FAC
:109D1800DFF8B4A0304EA87895F801E096F80080F6
:109D28002A4CDFF8A090254EA8BF4FF0080C8AF8FF
:109D380000C01FFA8CFA10FB0AF01EFB0AFE80B264
:109D4800DFF88CA02080A9F800E000244FF0640E12
:109D5800B8F1020F34701C70CAF804408AF801E0A8
:109D68007FF439AF0FFA8CF1BDE73078A0B9012341
:109D780077603370C2F164021A4B00FB02F083FB78
:109D88000023C017A0EBA3506430707036E708209A
:109D9800BDE8F04728F0CEB87368F81A8EE7032CB0
:109DA80096D10D49097802299AD0044EFCE600BFE5
:109DB800F7570020BC3A002058390020CC3A002040
:109DC80084370020C03A00209A370020BE3A00208D
:109DD800C43A0020544D0020543600207F96980045
:109DE800583600206BCA5F6B2DE9F04F2DED028BC2
:109DF80093B0054618F0FEFCAE4B1E7826B113B0A2
:109E0800BDEC028BBDE8F08FAB4B1B685805F6D54F
:109E1800DFF80483D8F80020002A00F01381A74C4B
:109E2800D4F8283103F5F43348339D42C0F00A8151
:109E3800A34F94F82C113B68C4F82851013184F8D9
:109E48002C11990701F1CF8113F0140F41F0948080
:109E580013F0080F94F82C3140F0668113F00709CD
:109E680001F00A81282B974F01F039825E20904734
:109E7800954B1B78002B6BD0904C944AD4F830311A
:109E8800EB1A934201F21B80DFF8909299F8006078
:109E98009EBBDFF88C82D8F80000FBF729FAC0B225
:109EA80001280ED9022841F01883894B1A78002A14
:109EB80041F0CF84D4F83821AA1AB2F57A6F81F02C
:109EC8005885844E3268002A42D099F80030BBB9D0
:109ED800814BD8F800001B689B781E3B012B4FF084
:109EE800020141F2BD84043014F026FD0122002352
:109EF80089F8002084F8443128E0764E32683AB375
:109F0800D4F8403140F6B731EB1A8B4220D994F897
:109F18003C31002B01F0D882013BDBB284F83C31A4
:109F2800002B01F0B78194F8440112F8011B94F852
:109F38004531DFF8ECE1326001330A18DEF8000041
:109F480084F8442184F84531FBF7D6F9C4F8405128
:109F5800624A3B6812780133012A0A9300F00087AD
:109F68005F4B1B7863B15F4E33684BB1534CD7F8E6
:109F78000080D4F85831A8EB0303632B00F28E86D7
:109F8800594B1B7873B1594E33685BB14B4CFAF798
:109F980087FED4F86031029044F61F62C31A9342D8
:109FA80000F20681524B1B78002B4DD1514B1B7888
:109FB80043B1424CD4F8B03203F50043E8339D4234
:109FC80080F044874C4B1B78002B3FF418AF3B4E76
:109FD8004A4C4B4D06F2B9272068FBF789F900284F
:109FE8003FF40DAF2068FBF77BF92B7880465A1EAB
:109FF80033B120682A70FBF77BF90028F2D1FEE61E
:10A0080003223946781E2AF0DAFF96F8B83296F815
:10A01800B92286F8BB8283F47F4383F0FF039B1A3F
:10A028001FFA88F89BB2B8EB132FD5D196F8BA224D
:10A03800DBB29A42D0D1781E13F090FF2B781844E7
:10A048002870C9E71F4F13E72E4C2278002A40F0EA
:10A058006786DFF8D09099F80040002C40F0958092
:10A06800294E3078002841F07F83144C274ED4F8CD
:10A07800A8223178264B93FBF1F313449D4295D3E4
:10A08800244A94F8AC32C4F8A852D75CF90701F115
:10A09800F784BA0701F18B847B0701F11D8494F8DA
:10A0A800AC323178013393FBF1F201FB123384F8BF
:10A0B800AC327BE79D560020105C00200420002075
:10A0C8007439002078690020EE4D00203F0D030010
:10A0D80004000020E8390020E4390020EF4D00207A
:10A0E800FC4D0020D46C0020044E0020084E0020B7
:10A0F800484E0020594E00200E4E0020144E0020DD
:10A10800184E0020E04D0020504E0020584E0020F0
:10A11800A0860100544E00205C4D0020EC39002040
:10A12800E0390020514E002013F0030A7FF496AE68
:10A138005E209047D8F8003014209847184B194AE9
:10A14800B3F9043082FB03124FEAE379C9EBA209A1
:10A158000FFA89F95FFA89F018F0D0FAC9F30720E5
:10A1680018F0CCFAD8F800305E209847D8F80030BC
:10A178001C209847504618F0C1FA504618F0BEFA0D
:10A1880094F82C31D8F8002068E6074E376E002F77
:10A1980041F0E080054B89F80070C3F8A85205E744
:10A1A8008039002067666666604E00200420002023
:10A1B80094F86631002B41F07D80E94B1B6803F071
:10A1C8000802002A48F603414AF60B404BF60F42B4
:10A1D80049F6074804BF0246884613F0040F4FF0BB
:10A1E800190118BF90469A0684F8661103D548F4F9
:10A1F800804848F0200814F065FEC8F309090028D3
:10A2080041F08A84D74B9B79002B41F0D1849B463F
:10A2180064204FF0FF334FF0000ACDF82880CDF8C6
:10A228002C80CDF83090ADF836B0ADF838308DF8D8
:10A238004600ADF834A0CDF83AA0CDF83EA0CDF850
:10A2480042A00DF1280EBEE80F00DFF824C384F801
:10A2580005A0ACE80F009EE80F00ACE807002CF85A
:10A26800023B61464FF001081B0C4FF0FE0E1F2009
:10A27800C82201F81E3984F802E0A27184F8078028
:10A28800E07094F87601207180F0F10383EA0313FB
:10A29800DAB2130983F0E70343EA022383EAC2032D
:10A2A8001BB283EA0312D2B2C3F3072383EA121361
:10A2B80043EA022383EAC2031BB283F0C80282EA9C
:10A2C8000212D2B2C3F3072383EA121343EA02232A
:10A2D80083EAC2031BB283EA080E8EEA0E1E5FFAF7
:10A2E8008EFEC3F3072282EA1E1242EA0E2200EB18
:10A2F800080382EACE0E0CEB080084F87631A4F845
:10A3080000E011F8013B83EA0E0383EA0313DBB292
:10A318001A0982EA1E2242EA032282EAC3031BB216
:10A328001FFA83FE8142A4F800E0EAD183F07C039F
:10A3380083EA0313DBB21A0982EA1E2E8EEA032E81
:10A348008EEAC30E0FFA8EFE1FFA8EFADFF824C2C9
:10A35800A4F800A05FFA8EFE4FEA1A2A84F828A013
:10A3680084F827E00CF5CF7904F1220BDCF8000023
:10A37800DCF80410DCF80820DCF80C30C846A8E843
:10A388000F000CF1100CDC45C146EFD1DCF80000E1
:10A39800C8F80000DFF8E0819CF8043089F8043040
:10A3A80008F1270984F8C5E184F8C6A118F8011F47
:10A3B8003068FAF7A1FFC145F8D194F86721002A5F
:10A3C80040F07D8768493B6808780A2184F867115E
:10A3D800002801F02F81DFF8A4C10128BCF8001083
:10A3E800059141F205840228BCF8029001F0AB8384
:10A3F800BCF804100491032801F0F3830428BCF886
:10A4080006B001F0E8830528BCF808E001F0DE8317
:10A418000628BCF80A8001F0D5830728BCF80C1080
:10A4280001F0CD83BCF80E20039294F876010A93CC
:10A43800024682F0300383EA0313DBB24FEA131CAF
:10A448004A4806928CF07A0C4CEA032C0088227158
:10A458008CEAC303DFF828C1C0EB00208CFB002C7A
:10A468008444C017C0EB6C220792059A4FF0000A8B
:10A4780062F30F0A049A69F31F4A1BB24FF00009EE
:10A488004FF0000C83EA031062F30F096EF30F0C10
:10A49800039ACDF82CA04FF0000EC0B261F30F0E56
:10A4A800C3F3072368F31F4C62F31F4E4FF00008F5
:10A4B8009DF81C20CDF834C083EA10136BF31F49B4
:10A4C800CDF83090CDF838E08DF83C808DF83D20FF
:10A4D80043EA00230DF1280983EAC00EB9E80F000A
:10A4E8000FFA8EFE8EF0C80A8AEA0A1ADFF880C0D0
:10A4F80084F805805FFA8AFACEF3072EACE80F00DD
:10A508008EEA1A1E4EEA0A2399E8030083EACA0370
:10A518001BB283F0230E4CF8040B8EEA0E1E5FFA72
:10A528008EFEC3F3072282EA1E12069B604642EAA9
:10A538000E2203F1010882EACE0E20F814194FF01A
:10A548002309FE211622C82384F87681A4F800E0A6
:10A558000CF1020C84F80790A170E27012E000BFC1
:10A568007439002058390020F8560020504D00203A
:10A578000C20002006200020A32100207278002053
:10A5880003082080A37110F8013B83EA0E0383EAD5
:10A598000313DBB21A0982EA1E2242EA032282EA84
:10A5A800C3031BB21FFA83FE6045A4F800E0EAD19A
:10A5B80083F0F40383EA0313DBB21A0982EA1E2E3E
:10A5C8008EEA032E8EEAC30E0FFA8EFE1FFA8EFC59
:10A5D800DFF82084A4F800C04FEA1C2A5FFA8EFE38
:10A5E80084F81EE084F81FA0D8F80410D8F80820D2
:10A5F800D8F80000D8F80C3008F5CF7CACE80F008C
:10A60800D8F81000D8F81410D8F8182004F2BD199A
:10A61800ACE8070004F29F1884F8BDA184F8BCE1F7
:10A6280018F8011F3068FAF767FEC145F8D194F8A9
:10A638006E81B8F1000F40F04786E54B94F876C17B
:10A64800B3F90010B3F90220B3F904309FEDE16AC1
:10A65800DFF89C9384F8058007EE103A3B680A936C
:10A668008CF06A0383EA031306EE901AD9B20B0939
:10A6780083F0D50343EA012383EAC1031BB283EACB
:10A6880003115242C9B207EE902AC3F3072383EAA3
:10A69800111343EA0123F8EEE77AF8EEE66AB8EE1A
:10A6A800C77A83EAC1031BB267EE867A66EE866ACA
:10A6B80027EE067A002083F0C80ECDED0C7ACDED9A
:10A6C8000B6A8DED0D7A0E900F9010908EEA0E1792
:10A6D8000DF1280AFFB2C3F3072EBAE80F008EEA7D
:10A6E800171E4EEA072E8EEAC70E0FFA8EFEA9E84D
:10A6F8000F008EF01E079AE8070087EA07185FFA2E
:10A7080088F8CEF3072787EA181747EA082789E861
:10A71800070087EAC8071C214FF0050A4FF01E08FA
:10A728004FF0FE0EC8220CF10103E17084F86EA10F
:10A7380084F8078084F802E0A271A9F1100184F876
:10A7480004C009F10C00278084F8763111F8013B28
:10A758007B4083EA0313DBB21A0982EA172242EA32
:10A76800032282EAC3031BB29FB281422780EDD144
:10A7780083F0270383EA0313DBB21A0982EA17225C
:10A7880082EA032282EAC3031BB21FFA83FCDFF8C2
:10A798006482A4F800C05FFA83FE4FEA1C2C84F898
:10A7A80025C084F824E008F5CF7904F1220AD8F806
:10A7B8000000D8F80410D8F80820D8F80C304F4614
:10A7C8000FC708F11008D045B946F0D1824FB8F844
:10A7D8000030A9F8003007F1240884F8C2E184F8B1
:10A7E800C3C117F8011F3068FAF786FDB845F8D1DC
:10A7F80094F86F310393002B40F06C85774B1B68FE
:10A80800052213F0140F84F86F2140F0FE86DFED67
:10A81800747A94F876C16E4B724AB3F90410B2F99F
:10A828000620714F7148CDED0C7A8CF0220383EA33
:10A8380003135FFA83FE4FEA1E1383F0590343EABA
:10A848000E23B2F5FA6F83EACE031BB2A8BF4FF40A
:10A85800FA6283EA031EB2F57A7F5FFA8EFEB8BF0A
:10A868004FF47A72C3F307234FF0640883EA1E1388
:10A87800A2F57A7208FB02F243EA0E2387FB0287ED
:10A8880083EACE0ED2174FF0000980FB0180C2EB9D
:10A89800A712C9170FFA8EF7CDF82890CDF82C908B
:10A8A800CDF83490C1EBA00387F0C8090DF1280852
:10A8B800ADF83A20ADF83830C64689EA0919BEE83D
:10A8C8000F005FFA89F9C7F3072787EA191747EADC
:10A8D800092787EAC909464FDEF800E084F804C072
:10A8E8000FC70FFA89F989F04A0383EA0310C0B247
:10A8F800C9F3072383EA10133A460CF1010143EA2E
:10A90800002383EAC00342F810E900204FF04A0907
:10A918004FF0FE0C4FF0140E84F87611C8216071C8
:10A928002380043784F8079084F802C084F803E091
:10A93800A171184612F8011B414081EA0111C9B200
:10A948000B0983EA102343EA012383EAC10109B210
:10A9580088B2BA422080EDD181F0140181EA011158
:10A96800C9B24FEA111E8EEA102E8EEA012E8EEA27
:10A97800C10E0FFA8EFE1FFA8EF7DFF878A0278037
:10A988004FEA172C5FFA8EFE84F81CE084F81DC08D
:10A99800DAF80410DAF80000DAF80820DAF80C30EF
:10A9A800BAF818B00AF5CF79A9E80F00DAF810005C
:10A9B800DAF81410A9E8030004F29F17A9F800B008
:10A9C800BB4684F8BBC184F8BAE104F2BB1913E0B2
:10A9D8008039002088C3E43AA3210020743900207C
:10A9E8000000000072780020D34D6210676666662A
:10A9F8000C200020062000201BF8011F3068FAF701
:10AA08007BFCD945F8D1CB4BCB4A1B781278013B5C
:10AA180012F00100DBB214BFC0214021172B02D86D
:10AA2800C64AD35C0393C64B1A8893071ABF002300
:10AA380041F01001012312F4027F18BF022312F023
:10AA4800100F18BF062312F0200F18BF102300287C
:10AA580040F07F874FF0030994F876C10A938CF091
:10AA6800460383EA0313DAB2130983F0920343EA35
:10AA7800022383EAC2031BB283EA0310C0B2C3F302
:10AA8800072282EA101242EA002282EAC00212B2C7
:10AA980082F0C80E8EEA0E1E00235FFA8EFE9DF825
:10AAA8000CB08DF82CB00320C2F307228DF82F903C
:10AAB80082EA1E128DF82D308DF82E108DF8300098
:10AAC80042EA0E2998E8070089EACE0E0FFA8EF8B6
:10AAD800DFF87CE2E37188EA0819AEE803005FFA60
:10AAE80089F9C8F3072888EA191848EA092181EA88
:10AAF800C90994F808808EF800200FFA89F988EAC5
:10AB0800090282EA02185FFA88F8C9F3072282EA82
:10AB1800181242EA0822607AA17A94F80B906371BD
:10AB280082EAC80212B2504080EA0010C0B2C2F3F2
:10AB3800072282EA101242EA002282EAC00212B216
:10AB4800514081EA0111C9B2C2F3072282EA111207
:10AB580042EA012282EAC10212B289EA020989EABA
:10AB680009195FFA89F9C2F3072282EA191242EA3F
:10AB7800092294F80C80607BA17B84F804C082EAE7
:10AB8800C90212B288EA020888EA08185FFA88F847
:10AB9800C2F3072282EA181242EA082282EAC802AD
:10ABA80012B2504080EA0010C0B2C2F3072282EA13
:10ABB800101242EA002282EAC00212B2514081EA2F
:10ABC8000111C9B2C2F3072282EA111242EA012234
:10ABD80082EAC102E17B94F8109013B281EA030281
:10ABE80082EA0212D2B2C3F3072383EA121343EABA
:10ABF800022383EAC2031BB289EA030282EA021231
:10AC0800D2B2C3F3072383EA121343EA022383EA87
:10AC1800C2031BB283F0320282EA0212D2B2C3F339
:10AC2800072383EA121343EA022383EAC2031BB20F
:10AC38009AB24FF0FE080920C8210CF1010CDBB2D2
:10AC480084F802804FEA1228E070A17184F876C176
:10AC5800228084F812806374DAF80000DAF80410AD
:10AC6800DAF80820BAF80CB00EF5C87CACE8070092
:10AC78000EF5D07A8CF80290ACF800B084F8B08168
:10AC880084F8AF3117F8011F3068FAF735FBBA4579
:10AC9800F8D1029BC4F86031FFF784B9DFF8B4B08B
:10ACA800DFF8B4A0DFF8B490412013F09DFBBBF9A6
:10ACB80002308AFB0320DB17C3EBA00080B213F03D
:10ACC80079FBBBF900308AFB0320DB17C3EBA0003C
:10ACD80080B213F06FFBBBF904308AFB0320DB174B
:10ACE800C3EBA00080B213F065FB99F80010306840
:10ACF800FAF702FB94F85C3113F0010200F0F483D8
:10AD0800104AC4F858810133DBB2A2FB0312D208FF
:10AD180002EB8202A3EB420384F85C31FFF730B9FF
:10AD2800094B0A491868FAF7B7FA00232370FFF7A6
:10AD380090B900BFB44A0020F75700200456030812
:10AD4800D0390020CDCCCCCC4C4E0020A04D0020DA
:10AD58000C2000208039002067666666FA7900209A
:10AD6800B44E306800283FF4FBA84FF0000ADFF823
:10AD78000483B14CAB465546FAF7BAFAF8B1F5B9BF
:10AD88004FF00109AA463068FAF7AAFA83B27E2B77
:10AD980000F0718298F80120002A49D194F84811EE
:10ADA800B1B11B2B84F8482100F054820D2B45D0FB
:10ADB800306888F80190FAF79BFA0028E3D1AA4690
:10ADC80050460AAA9D495D4613F026FBFFF7C8B80E
:10ADD8007D2B00F0258494F84C2122B180F02003CB
:10ADE800DBB284F84C1194F84721062A10D8B4F83D
:10ADF8004A1130681944A4F84A11A118013281F89F
:10AE0800503184F84721FAF773FA0028BBD1D6E706
:10AE1800B4F84A2188F8019013449BB21A0A52FAEE
:10AE280083F3FF2BA4F84A31306802D1844DA3E79D
:10AE38003068FAF75DFA0028A5D1C0E73068A4F8B1
:10AE48004A21FAF755FA00289DD1B8E794F8B432A8
:10AE5800C4F8B052012B40F23B8394F8B5227949EB
:10AE6800981801EB8001013202F001028E6984F822
:10AE7800B522BEB1744F0B970DF14808123FA523B8
:10AE880048F8207D802284F8103115232946404651
:10AE980084F8112184F81231B047002840F09E82CE
:10AEA80094F8B432694A013382FB0312A2EBE372CD
:10AEB80002EB42029B1A84F8B432FFF783B8644A63
:10AEC800644BD4F8341138681B8892F80BE0624A56
:10AED800401A4FF47A71DEB201FB0EF11B0A967725
:10AEE800167588424FF00006D37753759670167121
:10AEF80080F0DC82594B5A49DFF874811B68594E3F
:10AF0800D1F800E088683168C4F8305188FB03C67E
:10AF1800DB17C3EB6613544E88FB01C803F5FA73BD
:10AF280086FB0E9C86FB00964FEAEE7EC017CEEBA2
:10AF3800AC0E9BB2C0EBA60CCE1701F5EA40C6EBEF
:10AF48006816303093761B0A783600123031D37683
:10AF58004FEA2E284FEA2C2382F81CE082F81D8045
:10AF680082F820C082F8213082F8246082F8230019
:10AF780082F82210FEF788BF5E209047D8F800308C
:10AF880030209847374BD3F800905FFA89F017F0D4
:10AF9800B5FBC9F3072017F0B1FB94F82C3113F077
:10AFA80003097FF4EFA83149D4F828212B4B8A42B2
:10AFB8001B6840F28C84002BB8BF5B422C4A1BB242
:10AFC80082FB03124FEAE37BCBEB621B4FF0640971
:10AFD80009FB1B390FFA89F90FFA8BFB5FFA89FA1B
:10AFE8005FFA8BF2C9F30729CBF3072BD8F80030A7
:10AFF80002925E209847D8F8003010209847029AAD
:10B00800104617F07BFB584617F078FBD8F800304D
:10B018005E209847D8F8003021209847504617F00E
:10B028006DFB484617F06AFB3B68D8F80020FEF72E
:10B038000FBF00BFDC390020042000204A21002077
:10B04800542100200456030829210020565555553F
:10B058008C370020843700201C4E002078390020CF
:10B06800683900207C390020676666663F4B4C00D3
:10B078001F85EB51040000205E209047D8F800306F
:10B0880002209847FF2012F0F1FE0378FF2B00F012
:10B09800E58390F901304FEAE3795FFA89F9D8B28C
:10B0A80017F02CFB484617F029FBD8F800305E2033
:10B0B8009847D8F8003003209847FF2012F0D6FEB2
:10B0C8000378FF2B1DBFB0F90830DEB2C3F30729A0
:10B0D8004FF00009304617F011FB484617F00EFBF9
:10B0E800AF4B1B78042B74D0DFF8E0A2B4F82E2104
:10B0F8009AF80010DFF8D89292FBF1F301FB1323C2
:10B108009BB2B9F80020A4F82E311E01B6B2642310
:10B1180003FB02134A00B3FBF2F346EA0326C3F328
:10B1280003225E20D8F80030B6B216439847D8F804
:10B13800003006209847F0B217F0E0FA300A17F00E
:10B14800DDFA984AB4F82E31517AB9F800900133F3
:10B158000129A4F82E3100F00E85537B09EB8909EB
:10B168001FFA89F9002B40F0FE83D8F800308E4E84
:10B178005E209847D8F800303A209847A6FB093651
:10B1880076091FFA86FA5FFA8AF017F0B7FA4FEADB
:10B198001A2017F0B3FAD8F800305E209847D8F88C
:10B1A80000303B209847642303FB16939BB27F48EB
:10B1B800053380FB0320DB17C3EBA000C0B217F0F8
:10B1C8009DFA002017F09AFA794EB379002B40F0D7
:10B1D8004B833B681F0700F1378294F82C31D8F86D
:10B1E8000020FEF73FBEDFF8EC919FED728A4FF02A
:10B1F800240A5E2090475046D8F8003098476E4B96
:10B20800F9EC016A9B8A07EE103AF8EEE66AB8EEA6
:10B21800C77A0AF1010AC6EE877A5FFA8AFA67EEF8
:10B22800887AFDEEE77ACDED027ABDF908B05FFACB
:10B238008BF017F063FACBF3072017F05FFABAF137
:10B24800270F02D0D8F80020D3E73B68D8F80020B1
:10B25800FEF7FABD3068FAF74BF800287FF4A8AD7E
:10B26800306884F8469188F80190FAF741F8002888
:10B278007FF489ADA3E5306884F846A184F847A136
:10B2880084F8489188F801A0FAF732F800287FF48A
:10B298007AAD94E594F8441194F8453147484A1C2E
:10B2A8000133006884F8442184F84531FAF724F81A
:10B2B800FEF74CBE013B84F86631FFF77EB8013AD1
:10B2C80084F86721FFF7B3B908F1FF3884F86E8175
:10B2D800FFF78EBA03F1FF3B84F86FB1D9E44FF062
:10B2E80000095E20D7F800A084F82C919047D8F880
:10B2F8000030334E17209847484617F0FFF9314B76
:10B30800A3FB0A239B0BA6FB03125209C2EB0212F2
:10B31800A3EB8203D8B217F0F1F9D8F800305E2019
:10B328009847D8F8003018209847274BA3FB0A23E2
:10B338009B09A6FB03125209C2EB0212A3EB82037C
:10B34800D8B217F0DBF9484617F0D8F9D8F800203A
:10B35800FEF78CBD0024DFF8808027464FF0500AA6
:10B3680002E0DBB283F3118816F804B0601C59467A
:10B37800304412F01DFF002840F0CF810BF101038B
:10B388001C44EFF311838AF31288326E9442E8DB8F
:10B398000022DBB2326683F31188FEF7FBBE00BFE2
:10B3A800544D00208C3700201F85EB516766666678
:10B3B8005839002000007A4488390020E0390020FC
:10B3C8008988888873B2E745D34D62109A37002080
:10B3D80084370020B83900207D2702080A9EBE4223
:10B3E80040F2DE833D46002141F2210015F8013B81
:10B3F80081EA03235A0013F4004F80EA020192B253
:10B4080089B208BF11464A0080EA020311F4004FCE
:10B4180099B293B218BF0B46590013F4004F80EA53
:10B42800010289B292B208BF0A46530012F4004FD3
:10B4380080EA03019BB289B208BF19464A0080EA34
:10B44800020311F4004F99B293B218BF0B465A0089
:10B4580013F4004F80EA020192B289B208BF114684
:10B468004B0011F4004F80EA03029BB292B208BF6E
:10B478001A46530080EA030112F4004F9BB289B2C6
:10B4880008BF1946B542B1D1404602F0CBFEA649E5
:10B498000A9DA6486D1A152DA8BF15252A4628F01D
:10B4A800ABFCA34A94F8B4321570FBE4A14B39689D
:10B4B8001B78C4F83411013B012B3FF61BAD10215A
:10B4C80002239170137115E513F06CFAFEF73EBD77
:10B4D800994A02EB83029669CBE413F053FA974B2F
:10B4E80001221A70FEF7EDBC954B1B88D80513D4C2
:10B4F800D90600F13083980600F13B83590600F124
:10B508005183180700F15083D90700F14F8313F0D6
:10B51800020F0CBF04220C228A498B4B91F800B011
:10B52800DB780BF0010B0BB14BF0020B53200292AE
:10B5380012F05AFF854B1B8803EB830303EB83034D
:10B54800980080B212F036FF002012F033FF804BD3
:10B5580080491B883068C3EBC3135B0081FB032160
:10B5680019444FEAE37ACAEB612A5FFA8AFA51462C
:10B57800F9F7C2FE99F80030029A306842EA0B0BDC
:10B588008AEA030A002189F800A0F9F7B5FE5946AE
:10B598003068F9F7B1FE99F8003030688BEA030398
:10B5A800DBB2194689F80030F9F7A6FE94F85C3149
:10B5B800002B7FF4A5AB4F2012F016FF25F0E6FF15
:10B5C80025F0E4FF25F0E2FF01213068F9F794FE49
:10B5D800614A99F8003092F800A030680AF0010A30
:10B5E800514683F0010389F80030F9F785FE99F890
:10B5F800003030688AEA030A514689F800A0F9F752
:10B608007BFE94F85C31FFF77BBB544B9FED547A7B
:10B61800D3ED007AF8EEE77A67EE877AFFF7F9B8A4
:10B62800306884F84C91F9F763FE00287FF4ABABDF
:10B63800FFF7C5BB0146804686468346049081468F
:10B6480005900390FEF7F1BE0AA9464813F0C8F921
:10B65800D8F800305E209847D8F800301320984773
:10B66800BDF92860F0B217F049F8C6F3072017F0C3
:10B6780045F8D8F800305E209847D8F800301B20ED
:10B688009847BDF92A60F0B217F038F8C6F30720DA
:10B6980017F034F8D8F800305E209847D8F8003012
:10B6A800232098474E2017F029F8002017F026F895
:10B6B8000AA92C4813F094F9D8F800305E2098476E
:10B6C800D8F8003012209847BDF92860F0B217F07A
:10B6D80015F8C6F3072017F011F8D8F800305E20E7
:10B6E8009847D8F800301A209847BDF92A60F0B278
:10B6F80017F004F8C6F3072017F000F8D8F8003060
:10B708005E209847D8F8003022209847452016F048
:10B71800F5FF002016F0F2FF5FE541463A2012F0EF
:10B72800A3FC0743FFB229E614210020782F00204C
:10B738008D2F0020544D00200456030804000020DB
:10B74800D0390020F75700201057002084370020F8
:10B75800504D002003082080587A002078390020B6
:10B768000AD7233C80969800B349B44B0093A1F1C3
:10B778003F07B34BB34A099101F8404C0AA8B249B4
:10B78800089702F026FE089F7B1C08933C70089BD4
:10B798002922591C08911A70089BEA22591C089101
:10B7A8001A70089BC822591C08910AA81A7027F019
:10B7B800D5FB00F101080AA94246089828F01CFBAD
:10B7C800089A02EB08030133089302F80840089B23
:10B7D8005A1C08921C70089B5A1C08921C70089BE3
:10B7E8005A1C08921C70089B5A1C08921C70089BD3
:10B7F8005A1C08921C70089B5A1C08921C70089BC3
:10B808005A1C08921C70089B5A1C08921C70089BB2
:10B818005A1C08921C70089B5A1C08921C70089BA2
:10B828005A1C08921C70089B5A1C08921C70089B92
:10B838000122991812A808911A7050F8283DDB1BAC
:10B848003B7016F07DFF814B3470C3F8A852FEF7A9
:10B85800ADBBC4F838511E70FEF733BB48461FE431
:10B86800F9F73AFDFEF742BBD8F80030DFF80CA232
:10B87800DFF804925E209847D8F8003028209847CF
:10B88800DAF8003089FB0329DB17C3EBA9095FFA53
:10B8980089F016F033FFC9F3072016F02FFFD8F808
:10B8A80000305E209847D8F8003004209847338944
:10B8B800002B40F05281DAF8086086F31006F0B2E7
:10B8C80016F01CFFC6F3072016F018FF81E4CA46DD
:10B8D800CB464A46FFF78ABB574B0B93A3F1400868
:10B8E80000222121A3F13D0903F8402C88F8021019
:10B8F80088F80120CDF8289022F02CFD544B554AA9
:10B908001B88554900280ABF1146032704275805F4
:10B9180000F12C81DA0700F1408103F002034F4A5D
:10B92800002B1CBF032711463A464D4828F064FAFD
:10B9380009EB070312A84B4A013340F8203D9B1A34
:10B94800002209F8072088F8013016F0F9FEFEF702
:10B95800A6BB454AD278002A0CBF4FF004094FF025
:10B968000509FFF779B89AF8003099FBF3F9FFF762
:10B97800FCBB0122D8F800001A70F9F7B1FC0646A2
:10B98800D8F80000F9F7ACFC76067EF49AAA8E285F
:10B998007EF497AA99F80030002B7EF4AEAA334BB8
:10B9A800334A1A602D2384F83C31FEF791BA224AB3
:10B9B800304B0B920DF14808A2F13D0048F8200DDC
:10B9C8001988DFF8B890A2F1400300204FF00A0E62
:10B9D80002F8400C082283F801E040469A7002F011
:10B9E800FDFBD9F800302449DA1781FB0313C2EBB9
:10B9F800A30399B2404602F0F1FB13F071FAD9F8AB
:10BA080008900A9B4FEA1942591C0A911A700A9B1E
:10BA18004FEA1922591C0A911A700A9B5A1C0A9259
:10BA280083F800900A9B5A1C0A921870404616F038
:10BA380087FEFEF731BB00BFA04D0020BE56002098
:10BA4800548103085C8103086881030804200020EE
:10BA5800D039002038810308408103085081030849
:10BA6800634D0020614D002010570020E839002068
:10BA78001C4E0020843700206766666668390020FF
:10BA8800DFF8A0919FED608AB9F902305F4A0B9206
:10BA980007EE903AF8EEE77A0DF1480867EE887AF3
:10BAA800A2F14003FDEEE77AA2F13D0148F8201D1E
:10BAB80002F8400C0822CDED027A5A701E229A70C4
:10BAC800BDF80810404602F089FBB9F9003007EECE
:10BAD800903AF8EEE77A404667EE887AFDEEE77A24
:10BAE800CDED027ABDF8081002F078FBB9F9043000
:10BAF80007EE903AF8EEE77A404667EE887AFDEE70
:10BB0800E77ACDED027ABDF8081002F067FB4046EF
:10BB180016F016FEFEF7BDBA3D4B3E4A1B889279D9
:10BB280003EB830303EB83039B001FFA83FB002AC9
:10BB380067D0394B1B681BB2039313F0D1F9039BF1
:10BB480040B2FEF768BB114690469646934604926B
:10BB58000392FEF76ABC3422DEE413F0C1F916F052
:10BB6800CDFD002016F0CAFDFFF733BB03272B4994
:10BB7800DAE62422D0E4D8F800305E209847D8F8D6
:10BB88000030392098475FFA89F016F0B7FD4FEA80
:10BB9800192016F0B3FDFFF717BB21490427C3E6A8
:10BBA800002171E41022B7E42022B5E40822B3E4AE
:10BBB800194B8346B3F900306420FEF72CBB03927F
:10BBC800FEF733BC11460392FEF72FBC1146904690
:10BBD8000392FEF72ABC1146904696460392FEF75A
:10BBE80024BC11469046964693460392FEF71DBC28
:10BBF8001146904696469346049291460392FEF764
:10BC080014BC4FF0FF3396E758A08B41A04D00209D
:10BC180084370020583900206839002044810308FF
:10BC280048810308803900202DE9F04FDB4F2DEDC6
:10BC3800028B3D6815F0040883B010D0D84C94F8F6
:10BC4800BC3263B1D4F8C06246F2A713861B9E4289
:10BC580000F2FB8003B0BDEC028BBDE8F08F15F05D
:10BC68001009F7D0CE4CD4F8C06246F2A713861B51
:10BC78009E42EFD9C4F8C002C246B8F1000F40F0A6
:10BC8800E88017F051F8C74AC74B92ED087AD3ED10
:10BC9800007A0190F4EEC77AF1EE10FA80F275811D
:10BCA80007EE900AF8EEE77AC04A67EE877AFDEE6B
:10BCB800E77A17EE903A002BC2ED007A40F3EB8159
:10BCC800BB4AB2F900209A4200F3E581B949B1F9BB
:10BCD80000109942C0F2DF818A1AC91A07EE901A39
:10BCE800B8EEE77A07EE902AF8EEE77AF7EE006A00
:10BCF80087EE276A3D68B04A05F0040807EE10AAE7
:10BD080076EEC66A07EE903AB8EEC77AF8EEE77AAA
:10BD180027EE267AA6EE277AFDEEC77AC2ED007ADC
:10BD2800AB0750D5D4EDB67ADFEDA45AD4F8DC329F
:10BD3800B8EE677A67EE255A002B00F0A58107EE6A
:10BD4800903AF8EEE76AD4EDBA7AB8EEE76AC6EE4A
:10BD5800267A9B4A9B4B9B89D2ED004A94EDB45AB4
:10BD68009FED994A94EDB56A934A27EE247A06EE38
:10BD7800903A67EE277AF6EE004AB0EE457AA7EEDB
:10BD8800A47A924BF8EEE66A5B6A66EE846AF0EE95
:10BD9800474AB7EE007AA4EEA56A77EE665A07EE30
:10BDA800103AB8EEC77A77EE857A27EE257AC4ED91
:10BDB800B47AF0EE477AE6EE267ABDEEE77AC4ED7D
:10BDC800B57A82ED007A824B1B78122B00F0458100
:10BDD8000023C4F8E032C4F8E432C4F8E832C4F806
:10BDE800DC32C4F8D832B8F1000F40F001819FED81
:10BDF800796A744BDFED745A5B89D4EDB46A07EE47
:10BE0800103AB8EEC77AF7EE007AE7EE657A66EE92
:10BE1800A56A67EE867AE6EE877AB0EE670AC4ED21
:10BE2800B47A28F029F980EAE073A3EBE073042BD5
:10BE380040F31181002840F32A810538664B1860C9
:10BE480003B0BDEC028BBDE8F08FC4F8C00205F06A
:10BE58001009DFF898B1BBF80030002B4DD05F48CF
:10BE6800584A416892F806A0D4F8C4229FED5C0AAB
:10BE7800DFED5C0A019300290AF1FF3AB2FBFAF2FE
:10BE88008A46B8BF01F1070AA1EBEA0102EB010AF1
:10BE9800BAF1000F5246B8BF0AF10702D21007EEF6
:10BEA800902AF8EEE77AC0F804A027EE800A28F076
:10BEB800ABF9F7EE007A77EEC07A9FED4B0AD4F82B
:10BEC800CC2267EE807A9245FDEEE77AC4EDB27A2D
:10BED80000F0EB80019BC4F8CCA2013B9BB200228E
:10BEE800ABF80030C4F8D022C4F8D4224FF0000ACE
:10BEF800B9F1000F3FF414AFC3E6DFF8C8A0D4F8D7
:10BF0800C4329AF806209FED360ADFED360ADFF8CC
:10BF1800BCB0013AB3FBF2F307EE903AF8EE677A59
:10BF2800B7EE008A27EE800A28F06EF9DFED2E7A48
:10BF380038EE400A20EE270A28F09EF8BAF80830B2
:10BF4800DFED216A07EE103AD4F8C832C01AB8EE0D
:10BF5800C77A07EE900AA7EE668AB8EEE70ADBED25
:10BF6800097AF8EEE77A20EE080A67EEA67AA7EED5
:10BF7800870A28F081F8104BCBF824008246186015
:10BF8800B9F1000F3FF4CCAE7BE63D68074B4FF0AC
:10BF9800FF3205F004081A60C2E600BF74390020B9
:10BFA8000420002068670020E07A0020E87A00205A
:10BFB800DE7A0020E47A002078390020BD37863503
:10BFC800B0680020FC5200206F12833A0848002015
:10BFD80054360020000000007C39002004000020B6
:10BFE80008942537B1DC423ED048874AD6680020FD
:10BFF800334B1B88002B7FF42DAED4F8EC32DFEDE9
:10C00800316A314AC4F8ECA2AAEB030307EE903A6E
:10C0180007EE106AF8EEE77AB8EE477A67EEA67A86
:10C0280087EE876AFDEEC67A17EE903A934236DBC2
:10C0380040F2DC52934235DC83EAE372A2EBE3720E
:10C04800092A7FF7D4AE002B31DD0A3B07EE903A80
:10C05800B8EEE76ACDE60020F0E694EDB47AD4EDC8
:10C06800B57A1A4BD4F8E822D4F8DC1292FBF1F135
:10C07800BDEEC77AFDEEE77A17EE100A17EE902AA2
:10C08800588019809A80A3E6DFED117A61E63FF4C3
:10C09800D5AE0530D2E63D6805F0040840E69FEDD0
:10C0A8000D6AA6E69FED0C6AA3E6002317E73FF4A6
:10C0B8009EAE0A3307EE903AB8EEE76A99E600BFFB
:10C0C800D66800200024744924FAFFFF583600205F
:10C0D800000000000040BAC40040BA442DE9F8430B
:10C0E800344B1B685B0701D4BDE8F883324C334DF1
:10C0F80094F8F092B9F1010F51D1EB6928469847AD
:10C108002B69284698472B6A04F53E7004F53D7163
:10C1180098472B4BD4F8FC729B79D4F8C462D4F8B6
:10C12800F80207F101089845D4F8003308BF84F8ED
:10C13800BC9203F1010208BF4FF00008032A23D084
:10C148002049C4F8002394F8042341F823001ABBBB
:10C1580004EB870704EB8803C7F80803D3F8082320
:10C16800AB89C4F8FC82B61A30440022C4F8C40271
:10C1780084F8F022002BB7D0134A642B1268B8BF9A
:10C1880064231361BDE8F8830E4B012298600023F5
:10C1980084F80423C4F8003324F076FED8E76B69EA
:10C1A80028469847AB69284698470122EB8984F8C6
:10C1B800F022DFE77439002004200020084800201E
:10C1C800FC520020B06C00200C530020F8B5534BF3
:10C1D8001B681C0700D4F8BD514C524E524D736871
:10C1E80004F57271074630469847B4F9C803B4F9A4
:10C1F800CA23B4F9CC33317E286028466A60AB6024
:10C208000DF010FA494A137859073ED4D4F8D003F0
:10C21800474B1B7883B1474B2968B3F90AC0B3F978
:10C228000CE0B3F90E606A68AB68A1EB0C01A2EBF5
:10C238000E029B1B85E80E000028CCD03E4B381A16
:10C2480098423FD9B4F9E053B4F9DC13B4F9D47384
:10C25800B4F9D623B4F9DE63B4F9D8333548394490
:10C2680032442B4401EBD17102EBD27203EBD3734E
:10C278005B1049105210002541818281C381C4F8A6
:10C28800D053BDE8F840F7F79BBF2C4EB5F9000036
:10C29800B5F90410A4F8D40323F0040313700022A2
:10C2A800B5F90830A4F8DC03C4F8D0733260B28062
:10C2B800A4F8D613A4F8DE13A4F8D833A4F8E0330E
:10C2C8003846A5E70020F9F751F82B68B4F9D423CC
:10C2D8009342B4F9DC23B8BFA4F8D4339342C8BF5F
:10C2E800A4F8DC33B4F9D6236B689342B4F9DE239F
:10C2F800B8BFA4F8D6339342C8BFA4F8DE33B4F964
:10C30800D823AB689A42B4F9E023C8BFA4F8D8335D
:10C318009A42BFF660AFA4F8E033F8BD7439002044
:10C32800042000205C7A0020E8560020587A00207B
:10C33800EC7A0020804A00207FC3C9018A4A002085
:10C34800152303701623C370172383712D2343709D
:10C358002E2303712F23C3717047002870B51EDB8D
:10C368000928044620DD012303EB83035B00B0FBAF
:10C37800F3F2092AF8D87BB10D4EB4FBF3F0092883
:10C38800CCBF57223022A6FB03E5024403FB10442E
:10C39800EB0801F8012BF0D100230B7070BD2D23A1
:10C3A8000B7040420131DBE7303001F8010BF3E755
:10C3B800CDCCCCCC884230B44FF001042ED301FB55
:10C3C80004F4B0FBF4F58D42F9D284B1AAB901E0C6
:10C3D800B0FBF4F5092DCCBF572230222A4404FBC8
:10C3E800150003F8012BB4FBF1F4002CF0D1002266
:10C3F8001A7030BC7047B0FBF4F5092DCCBF37225A
:10C4080030222A4404FB150003F8012BB4FBF1F495
:10C41800002CF0D100221A7030BC70470546002A63
:10C42800EBD1D7E703685A1C0260197070472DE9F1
:10C43800F047089C2578002B804689460CBF4FF0B2
:10C44800200A4FF0300A661C35B3002A29DD33462E
:10C4580001E0024698B113F8011B501E0029F8D1DB
:10C46800971E60B13D46013D51464046C8476B1C8A
:10C47800002BF8DC257827EAE770013055B1041B5A
:10C4880029464046C847301916F8015B002DF7D1F8
:10C49800BDE8F087BDE8F087002A04DC2846BDE83F
:10C4A800F0870020EBE7571EDCE783684268D0ED91
:10C4B800037A00EB83010133934281ED040A836020
:10C4C80004BF0023836000EB830393ED047A0368C1
:10C4D80070EE277A9A42C0ED037A77EEC77AC0EDFC
:10C4E800037A0CDA013307EE103AF8EEC76AB7EEB2
:10C4F800007A87EEA60A036030EE070A704707EE57
:10C50800102AB8EEC77A87EE870A704790ED057A49
:10C5180090ED004AD0ED066AD0ED014AD0ED047ADC
:10C5280090ED035AD0ED025AA4EE007AB0EE406ABC
:10C53800B0EE470AB0EE667AA6EE247A67EEC07AC5
:10C54800A0EE457AE6EE257A80ED057AC0ED067A0A
:10C558007047D0ED057A90ED013AD0ED003AD0ED74
:10C56800064A90ED024A90ED077A90ED035A90ED55
:10C57800086AD0ED045AC0ED067AF0EE406A27EE5C
:10C58800830AC0ED056AA3EEA60A80ED087AA4EE38
:10C59800240AA5EE470AA5EEC60A80ED070A7047E9
:10C5A800D0ED007A90ED017A30EE670AE7EE007A76
:10C5B800B0EE670AC0ED007A704770470A449142AE
:10C5C80014D030B40139551E41F2210211F8014F3F
:10C5D800082380EA042004044CBF82EA400040009B
:10C5E800013B80B2F7D18D42F0D130BC70470023B7
:10C5F80026220360027027228270012243600271A2
:10C60800837170472DE9F341056906460F467DBBE6
:10C61800D0F80080C8F30A0323B30023D6F80080BB
:10C62800019318F011F9042819D1224C236943F019
:10C6380001032361BBB2A8F8003018F005F90428FB
:10C648002ED108F102030193019B3F0C1F8018F0C3
:10C65800FBF82369042823F00103236125D06FF038
:10C66800010505E018F0F0F8042805D04FF0FF3573
:10C67800284602B0BDE8F0810E4C236943F002035E
:10C688002361C4F81480236943F04003236118F040
:10C69800DBF82369042823F002032361BDD0E5E712
:10C6A800236923F001032361D9E733680433336036
:10C6B800DEE700BF00200240F8B504460D468E189C
:10C6C8000027B54201D12069F8BDE368591CE16033
:10C6D800234415F8012B1A720429F2D1A1682046C7
:10C6E800FFF790FFE7602061EBE7024B1868F8F767
:10C6F80003BE00BF7C1E002003682DE9F04F03F144
:10C708003845644EAD0A0124755D05F01F066D09B4
:10C71800022D04FA06F400F0A280032D00F0A48094
:10C72800012D52D08088B0FA80F4C4F11F04A4B25D
:10C73800E50803EB850504F007042E6AA4000F271B
:10C74800A74026EA07062E622E6A01F0030702FABE
:10C7580004F47A1E3443012AC1F3810CC1F3001892
:10C768002C62C1F3411135D9C60700F197808507BE
:10C7780000F1A380440700F1B180020700F1BF80F7
:10C78800C60600F1CD80850600F1DB80440600F185
:10C79800E980020600F1F780C60500F105818505EC
:10C7A80000F11381440500F12181020500F12F8178
:10C7B800C60400F13D81850400F14B81440400F179
:10C7C8005981020455D4BDE8F08F334D6E69344366
:10C7D8006C61A7E7002422464FF0010E4FF00309D1
:10C7E80004E00132102A04F10204ECD00EFA02F639
:10C7F80036EA0005F5D1D3F808A009FA04F5ED43A7
:10C808000AEA050AC3F808A0D3F808B00CFA04FA33
:10C818004AEA0B0AC3F808A0B3F804A01FFA8AFA78
:10C828002AEA06069E80B3F804A008FA02F646EA49
:10C838000A06B6B29E801E682E401E60D3F800A07D
:10C8480007FA04F646EA0A061E60D3F80CA001FAB5
:10C8580004F605EA0A0A46EA0A05DD60C1E70E4D54
:10C86800AE693443AC615DE70B4DEE693443EC616E
:10C8780058E71A6822F040421A601A6842EA877735
:10C888001F60DA6822F0404242EA8171D960BDE84F
:10C89800F08F00BFCC730308001002401A6822F022
:10C8A80003021A601A683A431A60DA6822F003022F
:10C8B8000A438507DA607FF55DAF1A6822F00C023B
:10C8C8001A601A6842EA87021A60DA6822F00C02D3
:10C8D80042EA81024407DA607FF54FAF1A6822F016
:10C8E80030021A601A6842EA07121A60DA6822F0FF
:10C8F800300242EA0112DA6002077FF541AF1A6896
:10C9080022F0C0021A601A6842EA87121A60DA68CE
:10C9180022F0C00242EA8112C606DA607FF533AF20
:10C928001A6822F440721A601A6842EA07221A60EA
:10C93800DA6822F4407242EA01228506DA607FF55D
:10C9480025AF1A6822F440621A601A6842EA872200
:10C958001A60DA6822F4406242EA81224406DA6008
:10C968007FF517AF1A6822F440521A601A6842EA33
:10C9780007321A60DA6822F4405242EA0132DA6079
:10C9880002067FF509AF1A6822F440421A601A6855
:10C9980042EA87321A60DA6822F4404242EA813277
:10C9A800C605DA607FF5FBAE1A6822F440321A60D9
:10C9B8001A6842EA07421A60DA6822F4403242EA08
:10C9C80001428505DA607FF5EDAE1A6822F440224F
:10C9D8001A601A6842EA87421A60DA6822F440222A
:10C9E80042EA81424405DA607FF5DFAE1A6822F434
:10C9F80040121A601A6842EA07521A60DA6822F48A
:10CA0800401242EA0152DA6002057FF5D1AE1A6897
:10CA180022F440021A601A6842EA87521A60DA68F9
:10CA280022F4400242EA8152C604DA607FF5C3AEBE
:10CA38001A6822F040721A601A6842EA07621A609D
:10CA4800DA6822F0407242EA01628504DA607FF512
:10CA5800B5AE1A6822F040621A601A6842EA876224
:10CA68001A60DA6822F0406242EA81624404DA60BD
:10CA78007FF5A7AE1A6822F040521A601A6842EA97
:10CA880007721A60DA6822F0405242EA0172DA60EC
:10CA980097E6036803F138422DE9F04F920A584DA2
:10CAA800AA5C02F01F0552090124022A04FA05F4BF
:10CAB80000F08C80032A00F08E80012A3CD001F01F
:10CAC80003077A1E012AC1F3810CC1F3001880887C
:10CAD800C1F3411135D9C60700F19680850700F1E9
:10CAE800A280440700F1B080020700F1BE80C606AC
:10CAF80000F1CC80850600F1DA80440600F1E88078
:10CB0800020600F1F680C60500F10481850500F1F2
:10CB18001281440500F12081020500F12E81C6042E
:10CB280000F13C81850400F14A81440400F15881F8
:10CB3800020455D4BDE8F08F324A55692C4354613C
:10CB4800BDE7002422464FF0010E4FF0030904E030
:10CB58000132102A04F10204ECD00EFA02F636EA89
:10CB68000005F5D1D3F808A009FA04F5ED430AEA5F
:10CB7800050AC3F808A0D3F808B00CFA04FA4AEA80
:10CB88000B0AC3F808A0B3F804A01FFA8AFA2AEA25
:10CB980006069E80B3F804A008FA02F646EA0A06DA
:10CBA800B6B29E801E682E401E60D3F800A007FA19
:10CBB80004F646EA0A061E60D3F80CA001FA04F649
:10CBC80005EA0A0A46EA0A05DD60C1E70D4A9569E1
:10CBD8002C43946173E70B4AD5692C43D4616EE703
:10CBE8001A6822F040421A601A6842EA87771F6082
:10CBF800DA6822F0404242EA8171D960BDE8F08FDC
:10CC0800CC730308001002401A6822F003021A606D
:10CC18001A683A431A60DA6822F003020A43850761
:10CC2800DA607FF55EAF1A6822F00C021A601A68A3
:10CC380042EA87021A60DA6822F00C0242EA8102AC
:10CC48004407DA607FF550AF1A6822F030021A60A4
:10CC58001A6842EA07121A60DA6822F0300242EAD9
:10CC68000112DA6002077FF542AF1A6822F0C002AB
:10CC78001A601A6842EA87121A60DA6822F0C0025B
:10CC880042EA8112C606DA607FF534AF1A6822F4E8
:10CC980040721A601A6842EA07221A60DA6822F4B7
:10CCA800407242EA01228506DA607FF526AF1A68EB
:10CCB80022F440621A601A6842EA87221A60DA6827
:10CCC80022F4406242EA81224406DA607FF518AF16
:10CCD8001A6822F440521A601A6842EA07321A6047
:10CCE800DA6822F4405242EA0132DA6002067FF53D
:10CCF8000AAF1A6822F440421A601A6842EA873278
:10CD08001A60DA6822F4404242EA8132C605DA60E3
:10CD18007FF5FCAE1A6822F440321A601A6842EABB
:10CD280007421A60DA6822F4403242EA0142850575
:10CD3800DA607FF5EEAE1A6822F440221A601A68AB
:10CD480042EA87421A60DA6822F4402242EA8142C3
:10CD58004405DA607FF5E0AE1A6822F440121A60E2
:10CD68001A6842EA07521A60DA6822F4401242EA64
:10CD78000152DA6002057FF5D2AE1A6822F4400249
:10CD88001A601A6842EA87521A60DA6822F4400286
:10CD980042EA8152C604DA607FF5C4AE1A6822F00E
:10CDA80040721A601A6842EA07621A60DA6822F06A
:10CDB800407242EA01628504DA607FF5B6AE1A680D
:10CDC80022F040621A601A6842EA87621A60DA68DA
:10CDD80022F0406242EA81624404DA607FF5A8AE3C
:10CDE8001A6822F040521A601A6842EA07721A60FA
:10CDF800DA6822F0405242EA0172DA6098E610B529
:10CE08000409013C052C17D80C4B33F8142000F00A
:10CE18000F0042FA00F313F001030DD0012303FAC7
:10CE280000F00138104026F093FD054A054B125DCD
:10CE3800104403EBC00010BD002010BDB8730308F8
:10CE4800C47303082C5900202DE9F04F4A484B4B76
:10CE58004B4C4FF090414FF0010A4FF002094FF050
:10CE680004084FF0080C4FF0100E202740268025AC
:10CE780030F8022B12F0010F03D01960A3F804A0B8
:10CE8800083312F0020F03D01960A3F80490083396
:10CE980012F0040F03D01960A3F80480083312F0CD
:10CEA800080F03D01960A3F804C0083312F0100F5C
:10CEB80003D01960A3F804E0083312F0200F02D061
:10CEC80019609F80083312F0400F02D019609E80CD
:10CED800083312F0800F02D019609D80083312F4D5
:10CEE800807F05D04FF4807B1960A3F804B0083325
:10CEF80012F4007F05D04FF4007B1960A3F804B04A
:10CF0800083312F4806F05D04FF4806B1960A3F8D2
:10CF180004B0083312F4006F05D04FF4006B1960A9
:10CF2800A3F804B0083312F4805F05D04FF4805B97
:10CF38001960A3F804B0083312F4005F05D04FF469
:10CF4800005B1960A3F804B0083312F4804F05D0D1
:10CF58004FF4804B1960A3F804B00833D20B04D007
:10CF68004FF4004219609A80083301F58061A142AC
:10CF78007FF47EAFBDE8F08FB87303082C5900200A
:10CF880000180048002867D003682DE9F04F03F126
:10CF980038445C4EA40A0125345D04F01F06640978
:10CFA800022C05FA06F558D0032C00F0A580012CB8
:10CFB80058D08088B0FA80F4C4F11F04A4B2E50800
:10CFC80003EB850504F007042E6AA4000F27A74089
:10CFD80026EA07062E622E6A01F00307A2407C1E8D
:10CFE8003243012CC1F3810CC1F300182A62C1F34A
:10CFF80041113CD9C60700F18980850700F1958069
:10D00800440700F1A380020700F1B180C60600F1D1
:10D01800BF80850600F1CD80440600F1DB80020662
:10D0280000F1E980C60500F1F780850500F105816A
:10D03800440500F11381020500F12181C60400F1C5
:10D048002F81850400F13D81440400F14B810204E5
:10D0580000F15981BDE8F08F70472B4CA669354324
:10D06800A561A6E7284C666935436561A1E70024F8
:10D0780022464FF0010E4FF0030904E00132102A56
:10D0880004F10204E6D00EFA02F636EA0005F5D1FC
:10D09800D3F808A009FA04F5ED430AEA050AC3F82B
:10D0A80008A0D3F808B00CFA04FA4AEA0B0AC3F845
:10D0B80008A0B3F804A01FFA8AFA2AEA06069E8096
:10D0C800B3F804A008FA02F646EA0A06B6B29E8049
:10D0D8001E682E401E60D3F800A007FA04F646EA40
:10D0E8000A061E60D3F80CA001FA04F605EA0A0A3B
:10D0F80046EA0A05DD60C1E7034CE6693543E561A8
:10D1080057E700BFCC730308001002401A6822F0EA
:10D1180003021A601A683A431A60DA6822F00302B6
:10D128000A438507DA607FF56BAF1A6822F00C02B4
:10D138001A601A6842EA87021A60DA6822F00C025A
:10D1480042EA81024407DA607FF55DAF1A6822F08F
:10D1580030021A601A6842EA07121A60DA6822F086
:10D16800300242EA0112DA6002077FF54FAF1A680F
:10D1780022F0C0021A601A6842EA87121A60DA6856
:10D1880022F0C00242EA8112C606DA607FF541AF9A
:10D198001A6822F440721A601A6842EA07221A6072
:10D1A800DA6822F4407242EA01228506DA607FF5E5
:10D1B80033AF1A6822F440621A601A6842EA87227A
:10D1C8001A60DA6822F4406242EA81224406DA6090
:10D1D8007FF525AF1A6822F440521A601A6842EAAD
:10D1E80007321A60DA6822F4405242EA0132DA6001
:10D1F80002067FF517AF1A6822F440421A601A68CF
:10D2080042EA87321A60DA6822F4404242EA8132FE
:10D21800C605DA607FF509AF1A6822F440321A6051
:10D228001A6842EA07421A60DA6822F4403242EA8F
:10D2380001428505DA607FF5FBAE1A6822F44022C8
:10D248001A601A6842EA87421A60DA6822F44022B1
:10D2580042EA81424405DA607FF5EDAE1A6822F4AD
:10D2680040121A601A6842EA07521A60DA6822F411
:10D27800401242EA0152DA6002057FF5DFAE1A6811
:10D2880022F440021A601A6842EA87521A60DA6881
:10D2980022F4400242EA8152C604DA607FF5D1AE38
:10D2A8001A6822F040721A601A6842EA07621A6025
:10D2B800DA6822F0407242EA01628504DA607FF59A
:10D2C800C3AE1A6822F040621A601A6842EA87629E
:10D2D8001A60DA6822F0406242EA81624404DA6045
:10D2E8007FF5B5AE1A6822F040521A601A6842EA11
:10D2F80007721A60DA6822F0405242EA0172DA6074
:10D3080002047FF5A7AE1A6822F040421A601A6834
:10D3180042EA87771F60DA6822F0404242EA817168
:10D32800D960BDE8F08F002852D0036803F1384275
:10D338002DE9F04F920A514DAA5C02F01F055209DF
:10D348000124022A04FA05F443D0032A00F090804D
:10D35800012A43D001F003077A1E012AC1F3810C88
:10D36800C1F300188088C1F341113CD9C60700F108
:10D378008980850700F19580440700F1A3800207A2
:10D3880000F1B180C60600F1BF80850600F1CD80AE
:10D39800440600F1DB80020600F1E980C60500F1D1
:10D3A800F780850500F10581440500F11381020528
:10D3B80000F12181C60400F12F81850400F13D812F
:10D3C800440400F14B81020400F15981BDE8F08F5B
:10D3D80070472B4A95692C439461BBE7284A5569E5
:10D3E8002C435461B6E7002422464FF0010E4FF05B
:10D3F800030904E00132102A04F10204E6D00EFA0F
:10D4080002F636EA0005F5D1D3F808A009FA04F5C2
:10D41800ED430AEA050AC3F808A0D3F808B00CFAE5
:10D4280004FA4AEA0B0AC3F808A0B3F804A01FFAE2
:10D438008AFA2AEA06069E80B3F804A008FA02F6D9
:10D4480046EA0A06B6B29E801E682E401E60D3F8D1
:10D4580000A007FA04F646EA0A061E60D3F80CA0F4
:10D4680001FA04F605EA0A0A46EA0A05DD60C1E798
:10D47800034AD5692C43D4616CE700BFCC73030819
:10D48800001002401A6822F003021A601A683A4330
:10D498001A60DA6822F003020A438507DA607FF52A
:10D4A8006BAF1A6822F00C021A601A6842EA870207
:10D4B8001A60DA6822F00C0242EA81024407DA6054
:10D4C8007FF55DAF1A6822F030021A601A6842EAE6
:10D4D80007121A60DA6822F0300242EA0112DA60B2
:10D4E80002077FF54FAF1A6822F0C0021A601A6867
:10D4F80042EA87121A60DA6822F0C00242EA811210
:10D50800C606DA607FF541AF1A6822F440721A60E5
:10D518001A6842EA07221A60DA6822F4407242EA7C
:10D5280001228506DA607FF533AF1A6822F440627B
:10D538001A601A6842EA87221A60DA6822F440629E
:10D5480042EA81224406DA607FF525AF1A6822F4A0
:10D5580040521A601A6842EA07321A60DA6822F4FE
:10D56800405242EA0132DA6002067FF517AF1A68C4
:10D5780022F440421A601A6842EA87321A60DA686E
:10D5880022F4404242EA8132C605DA607FF509AFEB
:10D598001A6822F440321A601A6842EA07421A608E
:10D5A800DA6822F4403242EA01428505DA607FF502
:10D5B800FBAE1A6822F440221A601A6842EA8742CF
:10D5C8001A60DA6822F4402242EA81424405DA60AD
:10D5D8007FF5EDAE1A6822F440121A601A6842EA22
:10D5E80007521A60DA6822F4401242EA0152DA60FD
:10D5F80002057FF5DFAE1A6822F440021A601A6845
:10D6080042EA87521A60DA6822F4400242EA8152FA
:10D61800C604DA607FF5D1AE1A6822F040721A604B
:10D628001A6842EA07621A60DA6822F0407242EA2F
:10D6380001628504DA607FF5C3AE1A6822F04062A1
:10D648001A601A6842EA87621A60DA6822F0406251
:10D6580042EA81624404DA607FF5B5AE1A6822F0C6
:10D6680040521A601A6842EA07721A60DA6822F0B1
:10D67800405242EA0172DA6002047FF5A7AE1A68E6
:10D6880022F040421A601A6842EA87771F60DA6817
:10D6980022F0404242EA8171D960BDE8F08F10B1B2
:10D6A800036882881A85704710B1036882889A6176
:10D6B800704738B100298388026814BF00211021FF
:10D6C8008B409361704730B1036882881B8A1A4285
:10D6D80014BF01200020704703685B6A18472DE9D2
:10D6E800F041044618460D461646984625F036FC85
:10D6F8002768E6722844A07229467D694346324667
:10D708002046AC46BDE8F0416047036810B50446C2
:10D718001B689847236820469B689847A37B01337A
:10D72800A37310BD10B5036804469B689847FF2390
:10D7380001226373227310BD08B5FFF760FB38B18F
:10D748002D2282710022C2712021BDE80840EAE53D
:10D7580008BD0B4B984206D0A3F5784398420DD0EC
:10D768004FF0FF3070470022064B03EB02135A8933
:10D77800013292B25A81588980B270470122F3E788
:10D78800003001409C55002070B50646806882B084
:10D7980010B104688088208541F08001706840F2EB
:10D7A800E93400E0ECB10589013C15F0020FA4B2A0
:10D7B800F8D0017340F2E93100E091B104890139F0
:10D7C80014F0010F89B2F8D0017B70680021F4F7DA
:10D7D80069F9B36813B11A689B889361012002B094
:10D7E80070BD8DE80C00FFF7B4FF9DE80C00ECE776
:10D7F80038B583680446154613B11A689B881385A3
:10D80800606840F2E93300E07BB30289013B12F023
:10D81800020F9BB2F8D0017340F2E93300E023B362
:10D828000289013B12F0010F9BB2F8D0037B6068BC
:10D8380040F2E93300E0DBB10189013B11F0020F4E
:10D848009BB2F8D0057340F2E93300E083B1028956
:10D85800013B12F0010F9BB2F8D0037BA36813B110
:10D868001A689B889361012038BDFFF772FFDEE7D5
:10D87800FFF76FFFF2E7F0B504460078012883B0A0
:10D888000D4616461AD002281ED11F46A36841F03D
:10D89800800113B11A689B8813856068F3F7BEFD91
:10D8A8003B46324600216068F4F7FCF8A368ABB148
:10D8B8001A689B889361012003B0F0BD94F90400B5
:10D8C800421C01D0022802DD002003B0F0BD6179BE
:10D8D80000962A46F4F73CFD03B0F0BD0120F4E7BA
:10D8E80070B50478012C1AD0022C16D1836801F087
:10D8F8007F0113B11C689B88238504461546406840
:10D90800F3F78CFD29466068F3F788FDA3687BB1BF
:10D918001A689B889361012070BD002070BD134672
:10D92800BDE870400A46417990F90400F4F70AB955
:10D93800012070BD427A02B9704710B504460368E9
:10D94800406804F10A0198470023637210BD437AC6
:10D958005A1C0344D2B242729972037A934200D895
:10D9680002B9704710B504460368406804F10A011B
:10D9780098470023637210BD98B10B4B012210B475
:10D9880002FA01F103F1750402E00333A34209D05E
:10D998001A788242F9D15A780A42F6D001205DF805
:10D9A800044B70470020FAE72C56030810B40023F4
:10D9B800094C01E0272B0AD003EB43020133A15C99
:10D9C8008142F7D122445DF8044B907870470020DB
:10D9D8005DF8044B704700BF2C56030870B54488A7
:10D9E80006460D46C4F30B0422460021284627F0BC
:10D9F80000FB3369094A934209D3094A934206D284
:10DA0800224628461946BDE8704026F0F5B923B1EC
:10DA180021462846BDE87040184770BD24B7030862
:10DA280014B80308064B07498B4202D30023184653
:10DA380070471A88C2F30B029042F8D01433F3E708
:10DA480088B2030824B70308024A136823EA0000CF
:10DA58001060704700340020F8B5174D2B78A52BBF
:10DA680028D16B78BE2B25D1022229464FF6FF70AC
:10DA7800FEF7A4FD114FAC1C22884AB1A618BE427D
:10DA880018D2052A16D92146FEF798FD3446F3E741
:10DA980021460222FEF792FD0222A118FEF78EFD12
:10DAA8000634074B641B1C8041F60F53C31A5842B7
:10DAB8005841F8BD0020F8BD00F003080000040834
:10DAC800062600202DE9F04FDFF848914C4F8BB027
:10DAD8000326A7EB09071822002104A827F089FAD2
:10DAE800484BCDF8109005971A69120604D5464A96
:10DAF8005A6002F188325A6001228DF824203422BB
:10DB0800DA60424B424C1B88ADF80030022269466D
:10DB180004A8FEF7D1FD022269464FF6FF70FEF712
:10DB28004DFDDFF8F4A080464FF0000B544536D386
:10DB38000AAC002524F8245D0222214604A8FEF739
:10DB4800BBFD022221464046FEF738FD40BAC043DD
:10DB5800ADF80800022202A904A8FEF7ADFD079857
:10DB680060B106ABC0F104022946184427F041FA17
:10DB7800069904A8FEF746FD079508909DF82430FD
:10DB8800089A23B11F490B6943F080030B61013EDA
:10DB98002DD0002A9FD1FFF75FFF50B32CE0658896
:10DBA8008DF80DB0C5F30B05AB1DADF80830238813
:10DBB800C3F30B02ADF80A201B0B062202A904A826
:10DBC8008DF80C30FEF778FD062202A94046FEF7D4
:10DBD800F5FC616880462A4604A8FEF76DFD616879
:10DBE80040462A46FEF7EAFC143480469EE7002A9F
:10DBF800D1D00520F5F77AFF0BB0BDE8F08F00BF54
:10DC0800000004080020024023016745A1560308CC
:10DC180088B2030800F0030824B703080378202B10
:10DC2800024600F10100F9D0092BF7D02D2B2CD09A
:10DC38002B2B03BF5378B7EE000A0246B7EE000A53
:10DC4800A3F13001C8B209289FED467A10D8F2EE48
:10DC5800046A07EE901AF8EEE77A12F8013FE7EE49
:10DC6800267AA3F13001C8B20928B0EE677AF0D954
:10DC78002E2B4CD003F0DF03452B0BD0F7EE007AA8
:10DC880067EE276A20EE260A70475378BFEE000A2F
:10DC98000246D5E710B451782D2959D02B290ABF4F
:10DCA8009178501C901C0024A1F13003092B53D803
:10DCB800002303EB830301EB430310F8011FA1F1D9
:10DCC8003002092AA3F13003F3D9B3F59A7F28BFAC
:10DCD8004FF49A73072B42D9DFED236A1A46F7EE01
:10DCE800007A083A072A67EEA67AFAD803F00703FB
:10DCF8002BB1F2EE046A013B67EEA67AFBD124B39E
:10DD0800C7EE276A5DF8044B20EE260A7047537861
:10DD1800A3F13001C8B2092802F10102AAD8F2EE33
:10DD2800046AF0EE665A07EE901AF8EEE77A12F8EF
:10DD3800013F87EEA66AA3F13001C8B2092866EE52
:10DD4800A56A37EE067AEED994E767EE276AD9E72F
:10DD5800901C91780124A7E7F7EE007ACFE7F7EE59
:10DD6800007AC5E70000000020BCBE4CB5EEC00A32
:10DD7800DFED317AF1EE10FACCBF30EE270A30EE43
:10DD8800670ADFED2E7A20EE270A30B5FDEEC07A5D
:10DD980087B017EE904A054684EAE470002303A989
:10DDA800A0EBE47001930093029323F081F9002C17
:10DDB800ACBF20232D2303A88DF8003025F0CEF822
:10DDC800012803A924D002282DD0032805BF302319
:10DDD800684668468DF8013027F013F9684625F043
:10DDE800BDF80338C4B222466946284627F040F9F0
:10DDF80000232B55284625F0B1F82E22431C2A541F
:10DE08000DEB0401E81827F019F9284607B030BDD2
:10DE1800302368468DF801308DF802308DF80330D4
:10DE280027F0EFF8DAE7302368468DF801308DF8EF
:10DE3800023027F0E6F8D1E76F12033A00007A447F
:10DE48002DE9F041064615460846B6FBF2F43CB902
:10DE580005FB1464124B1B5D00F8013BBDE8F08123
:10DE6800B4FBF2F767B90E4B05FB174705FB1464C3
:10DE7800DA5D00F8012B1B5D00F8013BBDE8F0817D
:10DE8800B7FBF2F8B8F1000F02D04046FFF7D8FF11
:10DE980005FB1878024B13F8082000F8012BE3E77C
:10DEA800748103082DE9F04714461D4606460023F1
:10DEB8004FF47A722046294625F0FAFCDFF84881AB
:10DEC8004B4A4C4F88FB00310144C31782FB002E9C
:10DED800C3EB611188FB012887FB00278644464A6B
:10DEE800C3EBEE2EC1EB011C82FB0E29A0EB8C0CC0
:10DEF8000744424A86F806C0C3EB27474FEAEE7C40
:10DF080008EB010ACCEBA90C82FB07824FEAE17807
:10DF18000CEB4C0CC8EB6A18AEEBCC0EC8EB08182F
:10DF2800DFF8E8C086F804E0A1EB880171718CFB8A
:10DF38000010F917C1EBE21240F2B55101FB127261
:10DF4800C3EBE050B2F5896F4FEA800740DA40F240
:10DF5800DA239A4244DCB2F5B77FB4BF4FF0000C25
:10DF68004FF0010C4FEA4C08254B08EB0C0103EB72
:10DF7800C1031FFA8CFEB3F88E00224908EB0C038C
:10DF880001EBC30116310B2301E031F8020D824287
:10DF98001BDA013BF9D11A4BC44403EBCC0C012327
:10DFA800BCF87800B37007F2B2770132121ABE4497
:10DFB800F270A6F800E0204629464FF47A72002352
:10DFC80025F076FC3281BDE8F0870133DBB2E9E762
:10DFD8004FF0030EF44640F296504FF00608CCE797
:10DFE8004FF0020EF44640F229404FF00408C4E70F
:10DFF800C5B3A29107452EC2ABAAAA2A73B06D1663
:10E008002C560308A456030889888888792D03119B
:10E01800104B2DE93048D3E9004554EA05020BD1ED
:10E028000346012200201871587198719A70DA70AD
:10E0380018801881BDE83088074B1A6814EB020B6A
:10E0480045F1000C5A466346FFF72CFF0120BDE856
:10E05800308800BFE01E002078690020F0B40288F4
:10E068008578164FC37804794179A2F2B27202F02A
:10E07800030606EB4606013D05EB860507EB45055D
:10E08800013BB5F878608579008940F2B557920868
:10E0980007FB0232931903EB430304EBC303C3EBFF
:10E0A800031301EB8303C3EB031305EB8303002185
:10E0B8004FF47A72C2FB0301F0BC70472C56030878
:10E0C800FAB170B48E18044603E0101A14D1B142A4
:10E0D80014D014F8012BA2F14103192B11F8013BBC
:10E0E800A3F1410598BF2032192D03F12000ECD986
:10E0F800D01A01D1002BEAD170BC7047002070BC47
:10E108007047104670474FF0FF32FFF7D9BFA0F1B4
:10E118006103192B98BF20387047A0F14103192BD0
:10E1280098BF20307047202805D0093804288CBFB4
:10E1380000200120704701207047613819288CBFE2
:10E14800002001207047413819288CBF0020012089
:10E158007047303809288CBF002001207047A0F193
:10E168003003092B07D920F02000413819288CBF2B
:10E178000020012070470120704730B40268114622
:10E18800531C036011F8024B0160D31C51780360E3
:10E198009378151D05601B0443EA0123D0782343B7
:10E1A80043EA006030BC70470368591C1A46016096
:10E1B80012F8021B0260587841EA00207047036891
:10E1C8005A1C02601878704738B50446006815462E
:10E1D80025F012FE22682A44226038BD036810B474
:10E1E8000A0A5C1C04601A7003685A1C02601970E1
:10E1F8005DF8044B704703685A1C026010B419702C
:10E2080003680A0A5C1C04601A7003680A0C5C1C28
:10E2180004601A700368090E5A1C026019705DF8D0
:10E22800044B704703685A1C026019700368090A96
:10E238005A1C0260197070472DE9F047002488B015
:10E2480080460F461E46A14605AD531C0393117820
:10E2580039B3252933D1931CCDF810900393507806
:10E2680030284ED04FF0000AA0F13003DBB2092B62
:10E2780042D96C2819D0642800F0938024D8252826
:10E288001CD063D9582876D063281BD131784046F2
:10E29800B847039A531C03931178043601340029B4
:10E2A800D7D1204608B0BDE8F087039B5A1C0392DB
:10E2B8001B78642B7CD02AD8252B54D125214046A5
:10E2C8000134B847039AC0E7732833D044D9752876
:10E2D8004FD106F1040E30682B4600220A217646FB
:10E2E800FEF768F8049A0095534639464046FEF70B
:10E2F8009EF8039A0444A8E704AA03A922F020FE82
:10E30800B7E7D31C039390784FF0010AACE7732B5F
:10E3180010D05BD9752B3AD0782B96D1A3F158023F
:10E32800B2FA82F2306852092B4610210436FEF701
:10E3380041F8D7E73368049A0093394600234046EA
:10E34800FEF775F804360444039A7EE70028B9D12D
:10E35800204608B0BDE8F0876E28B3D1039A336829
:10E3680004361C6071E72AD9582BD7D0632B8DD07F
:10E378006BE77828A6D1A0F15802B2FA82F2306889
:10E3880052092B461021FEF715F80436AAE706F1C4
:10E39800040E30682B4600220A217646FEF70AF85A
:10E3A800A0E7331D306829461E46FDF7D6FF99E7DA
:10E3B800331D306829461E46FDF7CFFF92E7002B34
:10E3C8007FF443AF204608B0BDE8F0876E2BC6D077
:10E3D8003BE70EB400B584B005AB019053F8042BAD
:10E3E8000649039301A8FFF727FF019B00221A7033
:10E3F80004B05DF804EB03B0704700BF2DC40008FB
:10E408000FB430B583B006AB0B490C4853F8042B56
:10E41800096800680193FFF70FFF094C054620685B
:10E4280003685B6998470028F9D0284603B0BDE81F
:10E43800304004B0704700BF1C4700202047002030
:10E448007C1E0020DFED2B7AB4EEE70AF1EE10FA1D
:10E458004ADDDFED296A9FED297A01E0B0EE670A0F
:10E46800B4EEC70AF1EE10FA70EE667AF6DC9FEDAC
:10E47800247AF4EEC77AF1EE10FA38D5DFED1E6A89
:10E488009FED207A01E0F0EE407AF4EEC77AF1EEE3
:10E4980010FA37EEA60AF6D4DFED1B7AB4EEE70AD7
:10E4A800F1EE10FA14DDDFED137A37EEC00A60EEF4
:10E4B800006A9FED166A9FED167ADFED167AA6EED2
:10E4C800867A20EE266AE6EE877AA6EE270A704755
:10E4D800DFED117AB4EEE70AF1EE10FA44BFDFED92
:10E4E800087A37EEC00AE2E7F0EE407ABFE7B0EE0E
:10E4F800670AD1E7DB0F4940DB0FC940E4CB16417F
:10E50800DB0F49C0E4CB16C1DB0FC93F92E741B925
:10E518009730083C15A82ABEDB0FC9BF09B909E026
:10E52800194690FBF1F301FB13030846002BF7D1C2
:10E53800084670470146FBE7F0EEC07AB0EEE07A95
:10E54800B4EEE77AF1EE10FAB4BFB0EE676AB0EE57
:10E55800476AB5EE406AF1EE10FA46D0B4EEE77AB3
:10E56800F1EE10FA8CBFF0EE675AF0EE475AC5EE9E
:10E57800866A9FED1F3A9FED1F6A9FED1F4A9FED28
:10E588001F5ADFED1F3ADFED1F4ADFED1F5AA6EED7
:10E59800C36AE6EEA34AA6EE864AB7EE006AA6EE7E
:10E5A800845AA6EEA46AE6EE855AC5EE866AB4EEEB
:10E5B800E77AF1EE10FA48BFDFED147AF5EEC00AFB
:10E5C80048BF77EEE66AF1EE10FA48BFDFED107A41
:10E5D800B5EEC00A48BF77EEE66AF1EE10FA48BF1A
:10E5E800F1EE666AB0EE660A7047DFED076ADEE7AD
:10E5F80039094E3DE3B59E3E88FA163E45FE7F3FFB
:10E6080099FB243F69A2163EA7DFA834DB0FC93F58
:10E61800DB0F4940DFED317A30EE277AFDEEC76A2D
:10E6280016EE903A2033402B02D99FED2D0A704701
:10E63800B4EEE70AF1EE10FA4DDD9FED2A6ADFED40
:10E648002A6A01E0B0EE677AB4EEE67AF1EE10FAE3
:10E6580077EE467AF6DC9FED257AF4EEC77AF1EE8E
:10E6680010FA35D5DFED1F6A9FED217A01E0F0EE53
:10E67800407AF4EEC77AF1EE10FA37EEA60AF6D42D
:10E68800DFED167AB4EEE70AF1EE10FA1BDCDFEDE7
:10E69800197AB4EEE70AF1EE10FA44BFDFED137A07
:10E6A80037EEC00A60EE006A9FED136A9FED137A99
:10E6B800DFED137AA6EE867A20EE266AE6EE877AF2
:10E6C800A6EE270A7047DFED0F7A37EEC00AE9E7B2
:10E6D800B0EE670AD4E7F0EE477ABCE7DB0FC93F34
:10E6E80000000000DB0FC940E4CB1641DB0F49C036
:10E6F800E4CB16C1DB0FC9BF92E741B99730083C9C
:10E7080015A82ABEDB0F494007EE901AF8EE677A83
:10E718009FED837A27EE800A20EE070AFDEEC07A85
:10E7280017EE903A2033402B00F28C80DFED7D7A93
:10E73800B4EEE70AF1EE10FA40F3E880B0EE407A62
:10E748009FED796ADFED796A01E0B0EE677AB4EEA1
:10E75800E67AF1EE10FA77EE467AF6DC9FED747AF7
:10E76800F4EEC77AF1EE10FA40F1CD809FED6E6AB3
:10E77800DFED706A01E0F0EE477AF4EEE67AF1EE4A
:10E7880010FA37EE867AF6D4DFED6B7AB4EEE77AD4
:10E79800F1EE10FA51DCDFED697AB4EEE77AF1EECA
:10E7A80010FA44BFDFED627A37EEC77A27EE076AC0
:10E7B800DFED635ADFED637ADFED636A9FED635A3D
:10E7C800E6EE257A67EE065AE6EE276AF7EE007A55
:10E7D800A5EEA67AF0EE675AE7EE055AE7EE457A17
:10E7E80087EEA55ADFED547A30EE277AFDEEC76A38
:10E7F80016EE903A2033402B29D99FED557AF6EE44
:10E80800006AB7EE006AF7EE004AC4EEA57A002364
:10E81800836143610362C36180ED045A67EEA66AAF
:10E8280027EE866A27EE877AC0ED006AC0ED026A95
:10E8380080ED016A80ED037A7047DFED3A7A37EEB2
:10E84800C77AB3E7B7EE005AF0EE455ACAE7B4EE16
:10E85800E70AF1EE10FA5FDD9FED336ADFED336A08
:10E8680001E0B0EE677AB4EEE67AF1EE10FA77EEF0
:10E87800467AF6DC9FED2E7AF4EEC77AF1EE10FABE
:10E8880047D59FED296ADFED2B6A01E0F0EE477A64
:10E89800F4EEE67AF1EE10FA37EE867AF6D4DFED8A
:10E8A800267AB4EEE77AF1EE10FA27DCDFED237A68
:10E8B800B4EEE77AF1EE10FA44BFDFED1D7A37EED9
:10E8C800C77A27EE076ADFED1E4ADFED1E6ADFED25
:10E8D8001E7AE6EE246A67EE064AE6EE267AB7EE78
:10E8E800006AA4EEA77AF6EE006A36EE476AF8EEFA
:10E8F800007A27EE277A66EE266A84E7DFED097A42
:10E9080037EEC77ADDE7B0EE677A3DE7F0EE407A9A
:10E9180024E7B0EE677AC2E7F0EE477AAAE700BFCD
:10E9280027D4D236DB0F4940DB0FC940E4CB164170
:10E93800DB0F49C0E4CB16C1DB0FC93FDB0FC9BFF2
:10E9480092E741B99730083C15A82ABEF304353F31
:10E958000000008070B406688E4217D90139751E10
:10E96800002311F8014F0822634013F0800F4FEA8B
:10E97800430318BF83F0D503013ADBB2F5D18D42CA
:10E98800EFD1721C0260337070BC70470023F8E747
:10E9980010B44C09012250F8243001F01F0102FA8A
:10E9A80001F10B4340F824305DF8044B70474B09E4
:10E9B80001F01F0150F82320012303FA01F111424D
:10E9C80014BF184600207047074A084B10781B7878
:10E9D800074A834296BFC31AC3F180030020126816
:10E9E80018441044704700BF34350020B13400206B
:10E9F8009C4A0020064A074B10781B7883428ABF3E
:10EA0800C3F18003C01AC018C0F17F00704700BF6F
:10EA180034350020B134002030B5134C237883B04E
:10EA28001BB90120237003B030BD10490522002313
:10EA38000D688DF804208DF8053000BFA868FEF732
:10EA48002EFE6A4601A902236868F3F72BF8A86826
:10EA5800FEF72AFE00BF9DF8013003F0010383F0A2
:10EA68000100237003B030BDCD550020885500202B
:10EA780070B5064C0646256803E023685B1BB34265
:10EA880003D8FFF7C9FF0028F7D070BD78690020C8
:10EA98002DE9F04F89B0B2F1000A02900491039376
:10EAA80040F3C5800B46002201EB8A0153F8040BA2
:10EAB8008B420244FAD1039B0592002B00F0AF80F1
:10EAC800059B002B7CD05E4B059A1B68DFF888916C
:10EAD80000920099DAB25118B1F5807F8CBFC2F567
:10EAE8008072009A0192574A92689A4240F2828054
:10EAF800554A1178002206928DF81C2002228DF8C2
:10EB08001820002960D01A0E8DF819200DF11A026C
:10EB18001C0C190A9370147051700620FFF7A8FF97
:10EB28000621D9F80000F2F796FC484A0123137031
:10EB380000BFD9F800309868FEF7B1FD424BD9F80C
:10EB480000201B785068002B06A90CBF042305235E
:10EB58000022F2F7A7FF0024049D029E019FA3460E
:10EB680029684FEA840800220B46013471B1B94282
:10EB78002DD2D9F8000031684068F2F793FF2A686F
:10EB8800336813443360BF1AC5F800B0A24505F1D5
:10EB9800040506F10406E3D1D9F800309868FEF7B9
:10EBA80083FD00BF264B019900981B68421A00920A
:10EBB800234A0B441360039A4AB3009A002A88D167
:10EBC800059809B0BDE8F08F0DF11902A0E7029C85
:10EBD800D9F8003054F80810586800223B46F2F77C
:10EBE80061FF54F808202B683A44DF1B44F80820DA
:10EBF8002F60D1E70598009C1549164A001B05901F
:10EC0800059800230B70137009B0BDE8F08F059BC1
:10EC1800009A9B1A0593059809B0BDE8F08FFFF795
:10EC2800FBFE00287FF44CAF039B0593C8E7039CC9
:10EC38001CB9FFF7F1FE0594C2E700230593BFE76F
:10EC48009C4A0020A0130020CC550020CD55002060
:10EC580034350020B13400208855002070B5104D9F
:10EC6800104E2B7831788B4284B016D00E4A03921E
:10EC78001A4402928CBF0C46CA1A04A98CBFC3F16D
:10EC880080020024012341F8102D02A802220194D9
:10EC9800FFF7FEFE002333702B7004B070BD00BF79
:10ECA800B134002034350020B434002070B5194C3C
:10ECB800194D23782978994284B027D0174A0392AE
:10ECC8001A44029234BF0E46CA1A04A934BFC3F1CB
:10ECD80080020026002341F8102D02A80222019686
:10ECE800FFF7D6FE23781844C0B203062B7848BF36
:10ECF80080F080008342207002D0002004B070BDF4
:10ED0800002301202B70237004B070BD012004B0D3
:10ED180070BD00BFB134002034350020B434002069
:10ED280010B50C4C45F20820FFF7A2FE206806211A
:10ED3800F2F791FB084B20680122C7211A70F2F7FD
:10ED48008AFB06480649074A002303700B701360C4
:10ED580010BD00BF88550020CD5500203435002057
:10ED6800B13400209C4A0020F0B51F4C83B02778AE
:10ED780000234FF0030E00930E4615468DF804301D
:10ED88008DF800E06FB3030E8DF801300DF102032A
:10ED9800010C020A9870197006205A70FFF768FE75
:10EDA800E8B100BF114F3B689868FEF778FC2378FC
:10EDB8003A68002B14BF05230423694650680022D3
:10EDC800F2F770FE3B683246002158682B46F2F78E
:10EDD80069FE3B689868FEF767FC00BF284603B0E9
:10EDE800F0BD0DF10103D3E7CC5500208855002074
:10EDF800F0B5124B9D6885B00DB905B0F0BDED0AB0
:10EE080014D0002704AE7C196410E0021022694671
:10EE1800FFF7AAFF0F2809DD6B4653F8042B0132D0
:10EE28000AD1B342F9D12546AF42ECDBFFF716FF12
:10EE3800034BED021D60E0E7671CF5E7A013002017
:10EE48009C4A00202DE9F04F2DED0E8BDFF8A8A38A
:10EE580099B0DAF80420069050469047002875D0FB
:10EE6800BAF8A85000218AF85110002D41F07E858B
:10EE7800DAF84820BAF93C70BAF93840DAF8206074
:10EE8800BAF93A00DAF82450DFF87093BB1A83EA2B
:10EE9800E371A1EBE371A41BB1F5804FCAF82C40D4
:10EEA800DAF828409AF85210DCBFCAF848703A4697
:10EEB800401B121BCAF83000B248CAF834200AF0C6
:10EEC800B1FBD9F80020940041F14486DAED0C5AE0
:10EED800DFF82CB3DAED0B7AAB499BED406ADBED3A
:10EEE800416A9BED427ADBF80C210968A74B049331
:10EEF800B8EEE58ADAED0D5AF8EEE77AF8EEE58A2B
:10EF0800013277EE867A38EE268A78EE878A8A4248
:10EF1800CBED407A8BED418ACBED428ACBF80C21C0
:10EF280002F0C4841F78142F03F0E4840023DBF874
:10EF380014410593062C01F2BA82DFE814F069182F
:10EF48002B193C173C19280AFF179C178F4BDFF821
:10EF5800B0B21C780493072C01F0FC829BF8213195
:10EF6800089353B15F1E8BF82171012C01F0CF85F6
:10EF780019B0BDEC0E8BBDE8F08F854A5279002A96
:10EF880001F05C83834A1278013AD2B2072C8BF8DD
:10EF9800212102F07685002309937F4BDBF82C2191
:10EFA800D3F800907D4B0793069B9FED7D6ADBEDC0
:10EFB8004AAA7C49CBF82C319A1A07EE902AF8EE27
:10EFC800677AB7EE007AC6EE279A0024764BDFF808
:10EFD8003482764F764E05932546D1ED006A9BED37
:10EFE800499A9FED74AADFED74BA9FED74DA9FED2C
:10EFF80074BADFED74CA9FED74CA77EE6A8A68EE58
:10F00800A68AF4EEC78AF1EE10FA88BFF0EE478AB6
:10F018006E4B98ED008A2344D3ED007AF5EE407AE2
:10F02800F1EE10FA17D06A4B234493ED007A78EE8C
:10F03800476AB0EEE66AF4EEC67AF1EE10FA08D541
:10F04800F5EEC06AF1EE10FACCBF37EE878A37EEDC
:10F05800678A83ED008A5F4B1A88910739D0022DA1
:10F0680037D099F82E105C4B07EE901A234493ED95
:10F07800007A4B42F8EEE76A07EE903A26EE877A76
:10F08800F8EEE77AB4EEE77AF1EE10FA0AD407EE72
:10F09800901AF8EE677AF4EEC77AF1EE10FA88BFA4
:10F0A800F0EE477A4D4B4E4903EB450331F9150015
:10F0B800B3F90C30C01A07EE100AB8EEC77AD207B7
:10F0C800E7EE4A7A41F15082464B93ED008A27EEEB
:10F0D800888A079B9BF86021234493ED01EA78EE28
:10F0E8004EDA002A00F0D0803F4BDBF86421069905
:10F0F8001B688A1A9A4240F3C78099F84830022B55
:10F1080002F01485022D04F06887384B1B689B07B2
:10F118007AD4374B86ED00DA1B689342C0F2AE8092
:10F12800F7EE007AF4EEE7AAF1EE10FA40F1AC80BF
:10F138000799304BD1ED017A93ED007AF0EEE77A3A
:10F14800F4EEC77AF1EE10FA40F19E80D1ED027A22
:10F15800F0EEE77AB4EEE77AF1EE10FA40F3948035
:10F16800D1ED037AF0EEE77AB4EEE77AF1EE10FA31
:10F1780040F38A801D4B1B6898077FD51849174BA9
:10F1880063E000BF3C530020002B002054360020D1
:10F19800EC5B0020644A0020D4390020005C002089
:10F1A800002474495C6C0020E4470020FC470020E0
:10F1B800F0470020CDCCCC3DAE47813F0000000099
:10F1C8000000C84200003443610BB63B506C00207D
:10F1D80024250020D039002030250020704A002046
:10F1E80080390020386C0020646C002074390020BD
:10F1F800606C00206C6C002010530020105C002014
:10F20800E823002018250020D74BD849DFF8C8E3A9
:10F2180031F915C09EED008ADFF8C0E386ED00DA0B
:10F2280003EB450028EE0A8AB0F90C00A0EB0C00AD
:10F2380007EE900AF8EEE77ADEF8000027EE888AF3
:10F24800904278EE4EDABFF66BAFB3F90C20B1F905
:10F2580000E0C748AEEB020E00688EEAEE72A2EB41
:10F26800EE72824210DAB3F90E30B1F90220D21AE6
:10F2780082EAE273A3EBE273984205DD00231846A5
:10F288008BF86031F5F76AFEBA4B234493ED000A18
:10F29800059B29EE000A022D20EE2D0AA3EC010A97
:10F2A800059304F0B486B44BD6ED006A93ED007A6A
:10F2B800B24BD3ED007AB24B93ED006AB14B67EED7
:10F2C800277A234427EEA87AD3ED007A67EE277AC7
:10F2D800F0EE665AE7EEAD5AB1EE467AF4EEC75A4A
:10F2E800F1EE10FA08D4F4EEC65AF1EE10FA8CBF1B
:10F2F800B0EE467AB0EE657A9BED4A6AF7EE007A90
:10F30800B4EEE76AF1EE10FAACBF0123002343B173
:10F31800F0EEE66AF0EEC77AF4EEE67AF1EE10FA6D
:10F3280001D586ED007A022D04F03C86964A974B6B
:10F3380052F825001B68B0EE4E0A9847944A954B40
:10F3480052F825001B68984799F8373023B1924B3B
:10F358001B88002B01F00282B0EE4D8A8F4B38EEED
:10F36800400A234493ED008A83ED000A99F8483057
:10F3780030EE480A20EE298A53B3894B1B78D90707
:10F3880040F1F887F7EE007AF4EEE7AAF1EE10FA0A
:10F398009BF86031C1F21F87002B01F08F82DBF8E8
:10F3A8006431069AD31A7F4A12689A4210DD7E4B5E
:10F3B800D3ED007AF0EEEDDAF4EEE7DAF1EE10FADA
:10F3C80042F1BD83002318468BF86031F5F7C6FD7E
:10F3D800764B9BF87021234493ED000A29EE000A2E
:10F3E80020EE088A87ED008A32B9059B86ED00DA9F
:10F3F80003ED01DA87ED00DA0135032D08F1040881
:10F4080007F1040706F1040604F104047FF400AED2
:10F41800049B1A78072A02F09F80012A02F036839B
:10F42800002307939BF87821002A41F07D83DFF8B9
:10F43800B0915F4BD9F800201968D20491F82C00DC
:10F4480001F1B881DFF89C815A4AB8F81A3092ED78
:10F45800006A594A594CD2ED005AD4ED036A584A09
:10F468008BED626A07EE103A564B92ED005AD3EDD7
:10F47800007AD3ED013A93ED024A8BED606AB8EE5B
:10F48800C77A75EEC64A012236EEC77ACBED5F4AD7
:10F49800CBED635A8BF89021C7EE055A0A8D53427B
:10F4A80006EE103A484BDFED496A93ED005A484B97
:10F4B800D3ED004AB7EE007AF4EEC75A35EE245A77
:10F4C800F1EE10FA88BFF0EE475A35EE275AB8EE3B
:10F4D800C66AF4EEE65AF1EE10FA07EE902AB4EE98
:10F4E800C65AB8BFF0EE665AF1EE10FACBED665A7E
:10F4F800B8EE677A01F10085B4EEC75AF1EE10FA5A
:10F5080088BFB0EE475A304BDFED326AD3ED017A4F
:10F518002F4BD3ED014A77EEA47A25EE265A77EEE3
:10F52800A37AB4EEE76AF1EE10FA08DCB4EEE77AF3
:10F53800F1EE10FA8CBFB0EE676AB0EE476A224B64
:10F548004A8DD3ED027A9FED237A534204EE903A26
:10F5580074EE277AF8EEE44A26EE076AF4EEE47AC7
:10F56800F1EE10FA4BD43FE0704A002080390020B9
:10F57800686C00200C6C00200C000020486B0020F8
:10F58800806C0020186C0020506B00204C6B002011
:10F59800A46B0020A06B0020D0390020502500204B
:10F5A800F7570020646C0020706C0020246C002049
:10F5B800D4390020944800203C4A00209C37002081
:10F5C800A0680020F0470020E44700200000000069
:10F5D800FC4700206F12833A386C0020606C0020D2
:10F5E800105C0020D055002007EE102AF8EE474A9C
:10F5F800F4EEE74AF1EE10FA88BFF0EE674AEA4AFD
:10F60800DFEDEA7A527864EEA74A0AB9F1EE644A65
:10F61800002842F0F980F7EE003AE54D2A78002AF2
:10F6280003F0EE83E34C9FEDE47A94ED024AD4EDC7
:10F63800016AD4ED037A26EE044AA5EE264AA4EE22
:10F64800A74A23EE844AB4EEC74AF1EE10FAB4BFD3
:10F65800F0EE476AF0EE446A98BFB0EE447A012AA9
:10F668008DED0C4A03F06084D4ED067AD4ED052ABA
:10F6780094ED073A66EE277AE5EE227AE4EE837A8D
:10F6880063EEA77AF4EEC77AF1EE10FAF4EEE67AB2
:10F698008CBFB0EE473AB0EE673AF1EE10FACDED16
:10F6A8000D7A98BFB0EE437AB8BFF0EE667A022AB8
:10F6B80000F08481D4ED0A6AD4ED092A94ED0B3A5E
:10F6C80066EE266AE5EE226AE4EE836A63EEA66ACF
:10F6D800F4EEC76AF1EE10FAF4EEE76A8CBFB0EE0A
:10F6E800473AB0EE663AF1EE10FA98BFB0EE437AB8
:10F6F800A8BFF0EE667A032ACDED0E6A00F05E81AF
:10F70800D4ED0E6AD4ED0D2A94ED0F3A66EE266A12
:10F71800E5EE226AE4EE836A63EEA66AF4EEC76A4F
:10F72800F1EE10FAF4EEE76A8CBFB0EE473AB0EEAD
:10F73800663AF1EE10FA98BFB0EE437AA8BFF0EE41
:10F74800667A042ACDED0F6A00F03881D4ED126A8A
:10F75800D4ED112A94ED133A66EE266AE5EE226A94
:10F76800E4EE836A63EEA66AF4EEC76AF1EE10FA75
:10F77800F4EEE76A8CBFB0EE473AB0EE663AF1EEC7
:10F7880010FA98BFB0EE437AA8BFF0EE667A052A61
:10F79800CDED106A00F01281D4ED166AD4ED152A69
:10F7A80094ED173A66EE266AE5EE226AE4EE836A7D
:10F7B80063EEA66AF4EEC76AF1EE10FAF4EEE76AB1
:10F7C8008CBFB0EE473AB0EE663AF1EE10FA98BF49
:10F7D800B0EE437AA8BFF0EE667A062ACDED116A3C
:10F7E80000F0EC80D4ED1A6AD4ED192A94ED1B3A96
:10F7F80066EE266AE5EE226AE4EE836A63EEA66A9E
:10F80800F4EEC76AF1EE10FAF4EEE76A8CBFB0EED8
:10F81800473AB0EE663AF1EE10FACDED126A98BFAB
:10F82800B0EE437AB8BFF0EE676A072A02F040816B
:10F83800D4ED1E7AD4ED1D2A94ED1F3A66EE277A90
:10F84800E5EE227AE4EE837A63EEA77AF4EEC77ADD
:10F85800F1EE10FAF4EEE67A8CBFB0EE473AB0EE6D
:10F86800673AF1EE10FACDED137A98BFB0EE437A0D
:10F87800B8BFF0EE667A082A00F0A080D4ED226ABC
:10F88800D4ED212A94ED233A66EE266AE5EE226A43
:10F89800E4EE836A63EEA66AF4EEC76AF1EE10FA44
:10F8A800F4EEE76A8CBFB0EE473AB0EE663AF1EE96
:10F8B80010FACDED146A98BFB0EE437AB8BFF0EEF7
:10F8C800676A092A02F0F480D4ED267AD4ED252A55
:10F8D80094ED273A66EE277AE5EE227AE4EE837A0B
:10F8E80063EEA77AF4EEC77AF1EE10FAF4EEE67A50
:10F8F8008CBFB0EE473AB0EE673AF1EE10FACDEDB4
:10F90800157A98BFB0EE437AB8BFF0EE667A0A2A45
:10F9180054D0D4ED2A6AD4ED292A94ED2B3A66EE18
:10F92800266AE5EE226AE4EE836A63EEA66AF4EEDE
:10F93800C76AF1EE10FAF4EEE76A8CBFB0EE473A08
:10F94800B0EE663AF1EE10FACDED166A98BFB0EE59
:10F95800437AB8BFF0EE676A0B2A02F0A980D4EDAB
:10F968002E7AD4ED2D2A94ED2F3A66EE277AE5EE1D
:10F97800227AE3EE247A67EEA37AF4EEC77AF1EE00
:10F9880010FAF4EEE67A8CBFB0EE476AB0EE676A1A
:10F99800F1EE10FACDED177A98BFB0EE467AB8BFFF
:10F9A800F0EE667A0AE000BFB44A00206F12833A8C
:10F9B80035360020D06700200000000077EEC77AB7
:10F9C800F7EE006AF4EEE67AF1EE10FACBED4A7A39
:10F9D80043F3278586EEA77A022ADDED0D7A27EE16
:10F9E800044A67EE877A8DED0C4ACDED0D7A4DD03D
:10F9F800DDED0E7A67EE877A032ACDED0E7A45D0D3
:10FA0800DDED0F7A67EE877A042ACDED0F7A3DD0C7
:10FA1800DDED107A67EE877A052ACDED107A35D0BC
:10FA2800DDED117A67EE877A062ACDED117A2DD0B1
:10FA3800DDED127A67EE877A072ACDED127A25D0A6
:10FA4800DDED137A67EE877A082ACDED137A1DD09B
:10FA5800DDED147A67EE877A092ACDED147A15D090
:10FA6800DDED157A67EE877A0A2ACDED157A0DD085
:10FA7800DDED167A67EE877A0B2ACDED167A05D07A
:10FA8800DDED177A27EE877A8DED177AE6490B6850
:10FA980013F0805301F05483F6EE005ACBED665A0A
:10FAA800002A03F0A781E149E14E9BF990019BED03
:10FAB800636ADFF890E3B6F90660CC78D9F80010ED
:10FAC800DBED624A059607EE100AB8F81A60D948C5
:10FAD8009EED004A0996BDEEC66A01F0100601F4D3
:10FAE800805E01F480010078D34F0A9116EE101A57
:10FAF800BDEEE46A00F0010C3F78DBED5F6ADBEDF8
:10FB0800607AB8EEC77A16EE100A002C41F04E80E3
:10FB1800CA4C9DED0C5A94ED006A002E41F0848386
:10FB280025EE866AC64EA5EE076AB0EE675AA6EEBF
:10FB3800265ABDEEC56A16EE10EA16EE107A8E4504
:10FB4800A8BF0F467045C8BF074606EE107AB8EE44
:10FB5800C66A012A86ED006A00F0608194ED046AA5
:10FB68009DED0D5A25EE866AA5EE076AB0EE675A36
:10FB7800A6EE265ABDEEC56A16EE10EA16EE107A03
:10FB88008E45A8BF0F467045C8BF074606EE107AD7
:10FB9800B8EEC66A022A86ED016A00F03F8194ED4C
:10FBA800086A9DED0E5A25EE866AA5EE076AB0EE44
:10FBB800675AA6EE265ABDEEC56A16EE10EA16EE8C
:10FBC800107A8E45A8BF0F467045C8BF074606EE97
:10FBD800107AB8EEC66A032A86ED026A00F01E8122
:10FBE80094ED0C6A9DED0F5A25EE866AA5EE076A1C
:10FBF800B0EE675AA6EE265ABDEEC56A16EE10EAB2
:10FC080016EE107A8E45A8BF0F467045C8BF074646
:10FC180006EE107AB8EEC66A042A86ED036A00F08A
:10FC2800FD8094ED106A9DED105A25EE866AA5EECA
:10FC3800076AB0EE675AA6EE265ABDEEC56A16EEFA
:10FC480010EA16EE107A8E45A8BF0F467045C8BF59
:10FC5800074606EE107AB8EEC66A052A86ED046AEB
:10FC680000F0DC8094ED146A9DED115A25EE866A49
:10FC7800A5EE076AB0EE675AA6EE265ABDEEC56A2B
:10FC880016EE10EA16EE107A8E45A8BF0F4670459C
:10FC9800C8BF074606EE107AB8EEC66A062A86ED91
:10FCA800056A00F0BB8094ED186A9DED125A25EEA6
:10FCB800866AA5EE076AB0EE675AA6EE265ABDEE2A
:10FCC800C56A16EE10EA16EE107A8E45A8BF0F46E2
:10FCD8007045C8BF074606EE107AB8EEC66A072A0E
:10FCE80086ED066A00F09A8094ED1C6A9DED135A21
:10FCF80025EE866AA5EE076AB0EE675AA6EE265A82
:10FD0800BDEEC56A16EE10EA16EE107A8E45A8BF4B
:10FD18000F467045C8BF074606EE107AB8EEC66AA9
:10FD2800082A86ED076A79D094ED206A9DED145A69
:10FD380025EE866AA5EE076AB0EE675AA6EE265A41
:10FD4800BDEEC56A16EE10EA16EE107A8E45A8BF0B
:10FD58000F467045C8BF074606EE107AB8EEC66A69
:10FD6800092A86ED086A59D094ED246A9DED155A42
:10FD780025EE866AA5EE076AB0EE675AA6EE265A01
:10FD8800BDEEC56A16EE10EA16EE107A8E45A8BFCB
:10FD98000F467045C8BF074606EE107AB8EEC66A29
:10FDA8000A2A86ED096A39D094ED286A9DED165A1B
:10FDB80025EE866AA5EE076AB0EE675AA6EE265AC1
:10FDC800BDEEC56A16EE10EA16EE107A8E45A8BF8B
:10FDD8000F467045C8BF074606EE107AB8EEC66AE9
:10FDE8000B2A86ED0A6A19D094ED2C6A9DED175AF4
:10FDF80065EE865AE7EE055AE6EEA57AFDEEE77A55
:10FE080017EE904AA142A8BF2146A042D8BF084693
:10FE180007EE900AF8EEE77AC6ED0B7ABCF1000F10
:10FE280001F0558010E000BF344A00201057002030
:10FE380072780020F7570020985E0020D0670020D5
:10FE480044480020CC670020CF4A1268002A41F0BD
:10FE58004B80CE4A127882B1287858B1CC4ECD4F1B
:10FE68000024E0B23B68B6EC010A984728780134D0
:10FE78008442F6DBC84A12689047049B1A78072A1E
:10FE880001F059830025D9F80020560501F19B801F
:10FE9800C24B1B681C0701F1A480C14B1B78BBB186
:10FEA800C04AB8F81A30B2F906209A4210DCBE4BA4
:10FEB8001B78012B01F00086192B01F0FD850E2B14
:10FEC80006D0082B04D0B94C0023A360CBF83831F6
:10FED8009BF8A24124B1B64B1B889B0741F07A8559
:10FEE8009BF8A831002B41F0138098F81E60002E73
:10FEF80000F00486022E01F0B884032E41F0BC8481
:10FF080098F82020C2EB421102EB8102D20092B293
:10FF180098F81F700237FFB2002B00F02086002AE5
:10FF280000F01D86A3490E68B2FBF6F216B2ABF8D4
:10FF3800D861002F03F0F18407EE906AF8EEE77AB3
:10FF4800F7EE006A86EEA77A984C012FDBED7B6A04
:10FF5800D4ED007A77EEE67A67EE877ACBED777A9A
:10FF680021D0D4ED017ADBED7C6A77EEE67A022FB8
:10FF780067EE877ACBED787A15D0D4ED027ADBED8F
:10FF88007D6A77EEE67A032F67EE877ACBED797A8A
:10FF980009D0D4ED037ADBED7E6A77EEE67A67EE78
:10FFA800877ACBED7A7A049A1278092A03F00187C6
:10FFB800002E40F3A9859FB39BED7B7ADBED777A22
:10FFC80077EE877A012FCBED7B7AC4ED007A21D0CA
:10FFD8009BED7C7ADBED787A77EE877A022FCBED92
:10FFE8007C7AC4ED017A15D09BED7D7ADBED797AC8
:08FFF80077EE877A032FCBEDB1
:020000040801F1
:100000007D7AC4ED027A09D0DBED7E7A9BED7A7AB7
:1000100077EE877ACBED7E7AC4ED037A013F022F2B
:10002000B8BF0227FAB20892002B089F18BF022718
:10003000634BDFED686A1A68049B9178187813782F
:1000400007EE903AF8EEE77AB0EE007A67EEA67A1D
:10005000F4EEC77AF1EE10FA40F34E87DFED5A6AFC
:1000600037EEC77AB0EE676AA7EE266AF0EE466A08
:1000700094ED007A9FED556A27EE066AF0EEC65AB7
:100080008BED526ACBED555A99B107EE101AB8EEC6
:10009000C75A9FED507A66EE064A25EE075AB7EE2C
:1000A000007A37EE457A64EEA54AA5EE247A26EE6C
:1000B000076A9FED477A537926EE877A27EE067A0C
:1000C000CBB1DFED446A9FED446A65EEA65A06EEB9
:1000D000903AF8EEE66A65EEA65AF4EEC65AF1EEEC
:1000E00010FA01F38D83B7EE006A76EE655AC6EE1C
:1000F000256A27EE267A0C289FED388ADFED386ACC
:1001000001F04880B4EEC87AF1EE10FA98BFB0EE74
:10011000478AB4EEE68AF1EE10FAB8BFB0EE668A0E
:100120008BED4C8A002F00F00881B0EE007AF4EEDF
:10013000C77AF1EE10FA05DD37EEC77ADFED226AF5
:10014000E7EE267A94ED017ADFED206A27EE267A33
:10015000F0EEC75A8BED537ACBED565A99B106EEB5
:10016000901A9FED1C6AF8EEE66A27EE075A66EED3
:10017000866AB7EE006A36EE666A25EE255AA5EE67
:10018000266A27EE067ADFED126A93792AE000BF2D
:10019000446B002030630020444800208C5E002027
:1001A000945E002074390020C41A00207278002068
:1001B000B44A00209C370020D0390020984A002003
:1001C000D83900200000C842D7A368416F12033B12
:1001D000000048430AD7233CA4707D3F00C0F94487
:1001E00000C0F9C467EEA67A67EE877AABB107EE76
:1001F000103AB8EEC77A1FED096A5FED096A27EE7B
:10020000257A27EE067AB4EEE67AF1EE10FA41F39B
:10021000E9825FED146A67EEA67A0C2800F09B87EE
:100220005FED126A1FED127AF4EEE67AF1EE10FA43
:1002300088BFF0EE667AF4EEC77AF1EE10FAB8BF36
:10024000F0EE477A012FCBED4D7A76DD53785FEDF6
:100250001F6A07EE903AF8EEE77AB0EE007A67EEA2
:10026000A67A537AF4EEC77AF1EE10FA05DD37EE8E
:10027000C77A5FED2B6AE7EE267A94ED027A5FED9E
:100280002D6A27EE267AF0EEC75A8BED547ACBED25
:10029000575A9BB106EE903A1FED326AF8EEE66AC5
:1002A00027EE075A66EE866AB7EE006A36EE666A91
:1002B00025EE255AA5EE266A27EE067A5FED3C6A02
:1002C000D37967EEA67A67EE877AFBB107EE103A2C
:1002D000B8EEC77A1FED416A5FED416A27EE257AD5
:1002E00027EE067AB4EEE67AF1EE10FA01F38C828C
:1002F000B5EEC07AF1EE10FA02F17C85B7EE006A35
:1003000036EE477AC6EE076A67EEA67A0C2800F04A
:100310005E875FED4E6A1FED4E7AF4EEE67AF1EEFF
:1003200010FA88BFF0EE667AF4EEC77AF1EE10FAB2
:10033000B8BFF0EE477ACBED4E7A092800F0F78689
:1003400098F82140002C40F0AC8600238BF8A831AF
:10035000BE4B1B7823B9BE4CA778002F41F05483C5
:10036000049B1C78072C7EF404AEF4F79DFCB94B7B
:10037000049A401B1478D880FEF7FBBD9BF86031CF
:10038000002B3FF429A8002318468BF86031F4F7BE
:10039000E9FDFFF721B8B04A1178DBF81861AF4BDF
:1003A0009FEDAF7AF5005A1982ED007A002978D0D6
:1003B000AC48B0EE476AF0EE476A0022F0EC017AF2
:1003C000013267EEA77A05EE902AB4EEE77AF1EEF5
:1003D00010FAF8EEE55AB8BFB0EE677A8A4276EEC8
:1003E000A76AA7EEA56AE9D1F5EEC06A5A19F1EE3F
:1003F00010FA82ED007A54DDC6EE265A9A4A9B49DD
:100400000988F7EE007A75EEE75AD2ED007A65EECC
:10041000A77AFDEEE77A17EE902A812A42F35984F3
:100420008A42A8BF0A4607EE902AF8EEE77A904A79
:10043000A81902EB800292ED057AD2ED003A92ED16
:10044000066A92ED014AD2ED046AD2ED034A92EDBA
:10045000025AA3EEA77AA4EE276A66EEC76AA7EE51
:10046000646ABDEEC77AE5EE276A17EE100A8128A6
:1004700082ED056AC2ED066A42F328848142A8BF74
:10048000014607EE901AF8EEE77AFCEEE77ACDED3A
:10049000077ABDF81C2059198A8016B9132F03F06A
:1004A000AB84152F41F0DE841D446A4BAA8823F8E3
:1004B0001620DBF814416F4A013482FB0432111913
:1004C000E217C2EBA102C2EBC202A41ACBF814419C
:1004D0006948DBF81C21069B684C01682478CBF83E
:1004E0001C319A1A11440160002C40F0D78007EEAD
:1004F000902A634DDFF8A081624EB8EEE78A05F5D9
:10050000F07405F51377F5EC017A9AED070ADAF83D
:100510000832F8EEE77A204627EE800A9847A4F1E1
:10052000E000DAF828319847A4F17000DAF8983141
:100530009847D5F8EC00DAF8AC309847D6ED007A59
:10054000A8EC010AE0EE087A2434A742E6EC017A2E
:10055000D9D1049B1C78072C7EF404ADF4F7A4FBDE
:10056000049A3C4B1478069A801A1880FEF7FABC5D
:100570009BED557AB1F90000DBED566AB1F902E066
:10058000414AF4EEC76A80EAE0738EEAEE71A3EBAB
:10059000E073F1EE10FAA1EBEE71B8BFF0EE476A2E
:1005A0008B42B8BF0B4607EE103A1378B8EEC77A05
:1005B00027EE0A7A002B00F05C81344B93ED005A51
:1005C000B5EEC05AF1EE10FA40F3BA85304BD3EDD8
:1005D000004AF5EEC04AF1EE10FA40F3B18534EE70
:1005E000C77A66EECB5A87EE246AC5EE856AB7EE07
:1005F000007AB4EEC76AF1EE10FA88BFB0EE476A2F
:10060000B5EEC06AF1EE10FA76EE876AB8BFB0EECA
:100610004D6A66EE266AF4EEC76AF1EE10FA88BFFC
:10062000F0EE476AF5EEC06AF1EE10FAB8BFF0EEF0
:100630004D6A184B93ED007A67EE877AA7EEA68A8B
:10064000FEF74BBD0122FEF7A5BC00BF9D56002062
:10065000EC33002058360020062B0020FC2D002013
:1006600000000000E8230020082B0020042B0020BD
:10067000242D00209324499290670020FC2A00201A
:100680003C53002094670020446C0020406C002004
:10069000486C00203C6C0020045C002007EE902A8F
:1006A0009E4B9F4C9F49A04FCDF81CB0F8EEE78AB7
:1006B000059304F5B875984600268B46049BDAED41
:1006C000077A1B78172B6DD094ED007AB8EEC78AA5
:1006D000082B28EE278A07D1B0EE480A089323F0AA
:1006E000CFFC089BA8F80000D9F8002090000BD59B
:1006F000002E03F00985B0EE480ADAF8083205F159
:1007000070009847B0EE408AB0EE480ADAF8283117
:10071000A5F170009847DAF8983128469847049B6D
:100720001B78032BB0EE408A37D0D4F8F000DAF80B
:10073000AC30B0EE480A9847D7ED007AABEC010A2E
:10074000E0EE287A0136032E05F1240508F10208AF
:1007500004F10404E7EC017AB0D1049BDDF81CB08D
:100760001C78F8E6714B724A234493ED007AD2ED7F
:10077000007A704B67EE277AF7EE006AF4EEE67ABD
:10078000F1EE10FA93ED007A88BFF0EE667A67EE2C
:10079000877A27EE888AFEF7E5BD23F071FCA8F87A
:1007A0000000C2E794ED007A0AEB4602B8EEC78A71
:1007B000128FA8F8002028EE278A95E75E4BDFF815
:1007C000B0811A785D4CD3075CBFB8F81820ABF83D
:1007D00084215B4AD4ED037A128807EE102AB8EE22
:1007E000C77AF4EEC77AF1EE10FA42F24480554C23
:1007F000238807EE103AB8EEC77AF4EEC77AF1EE26
:1008000010FAC1F26981504A504C92ED006AD4ED61
:10081000006A9BF99021CBED626A76EE665A012A56
:10082000CBED606ACBED5F5A8BED636A01F03387E5
:10083000069BCBF89431002437EEC77AFCEEE77ABA
:10084000434D8BED667A17EE902AABF88421012296
:1008500095ED005A8BF890213E4A944242F23B803B
:100860003D4BD3ED007AD3ED013A93ED024AFEF70A
:1008700017BE3A4B93ED006AB4EEEB6AF1EE10FA54
:1008800041F1A780F7EE005A75EEC65A3CEEC77AE2
:1008900065EE8C5A324BA7EE256A93ED007A26EE70
:1008A000076AB5EEC06AF1EE10FA40F24984CBEE69
:1008B000065AB7EE007AB0EE476AA6EEE56AF0EEA9
:1008C000466AA8E6274AD2ED007AB0EEC87AB4EEBE
:1008D000E77AF1EE10FA7EF77FAD234AD2ED007A87
:1008E000B0EEED7AB4EEE77AF1EE10FA7EF774AD81
:1008F0001E4AD8ED007A92ED007AF0EEE77AF4EE37
:10090000C77AF1EE10FA7EF567AD01220699CBF8B1
:1009100064118BF86021FEF74ABD00BF58360020F5
:100920003C530020045C0020946700203C250020FC
:10093000346C0020306C0020F75700209C370020DA
:10094000A4680020A66800203C4A0020906800208F
:10095000AC6800208FD00300F04700204C6C0020D2
:10096000406C0020746C0020706C0020786C0020BB
:10097000D0550020814C824B82481A6847780793F3
:100980002646814BB6F9060005944FF47A76B6FBFD
:10099000F2F2C2EB421602EB8602D600B6B2B542C4
:1009A00004931C7802F0A081DAF87C30BAF9381090
:1009B000DAF8602003F1010E07EE901A0A44BEF146
:1009C000010FCAF87CE0CAF86020F8EEE77A02F07E
:1009D0009881DAED1B5ADAED1D6A07EE10EA37EE60
:1009E000E56AB8EEC75A012D86EE057A37EE257A0C
:1009F00077EEC77A8AED1C7AE7EE866A8AED1B7A73
:100A0000F0EE667ACAED1E6ACAED1D6A02F023870F
:100A1000DAF89030BAF93A10DAF8642003F1010EEE
:100A200007EE901A0A44BEF1010FCAF890E0CAF826
:100A30006420F8EEE77A02F07F81DAED205ADAEDF1
:100A4000226A07EE10EA37EEE56AB8EEC75A012DC2
:100A500086EE057A37EE257A77EEC77A8AED217A27
:100A6000E7EE866A8AED207AF0EE667ACAED236AAE
:100A7000CAED226A02F01887DAF8A430BAF93C10FD
:100A8000DAF8682003F1010E07EE901A0A44BEF16D
:100A9000010FCAF8A4E0CAF86820F8EEE77A02F07D
:100AA0006681DAED255ADAED276A07EE10EA37EEAD
:100AB000E56AB8EEC75A012D86EE057A37EE257A3B
:100AC00077EEC77A8AED267AE6EE276A8AED257AEE
:100AD000F0EE667ACAED286ACAED276A02F00D8741
:100AE000059BDFF8C4B0D880BAF8A820049B013A6F
:100AF0001C78AAF8A820079900224A608A60CA6078
:100B0000FEF72DBAABF8D861002B3FF421AC1F4C97
:100B10000227FFF78DBA1E4B1E4A19681288174B21
:100B2000C96919805A8019B0BDEC0E8BBDE8F08FF1
:100B3000194B1A4D1A7812F0010F2A7840F02885C7
:100B4000002A00F04986920015491648DFF85C90AB
:100B5000DFF85C8023F054F9FFF77AB90A4B04936D
:100B6000DFF844B0B4E4BBF8D861013E36B2002EE1
:100B7000ABF8D861C8DD054CFFF721BA5836002024
:100B8000005C0020EC5B0020543600209C370020E5
:100B90000C53002008260020F7570020353600208F
:100BA0000C26002044480020E8230020105C002090
:100BB000D0550020002E01F07583BCF1000F42F0EB
:100BC000EF86D14C9DED0C5A94ED006ACF4E25EE88
:100BD000866A002F42F05084A5EE076AB0EE675A8D
:100BE000A6EE265AFDEEC44ABDEEC56A14EE900A82
:100BF00016EE10EA16EE107A8E45A8BF0F46704525
:100C0000C8BF074606EE107AB8EEC66A012A86ED1E
:100C1000006A00F0638194ED046A9DED0D5A25EEA3
:100C2000866AA5EE076AB0EE675AA6EE265ABDEEB2
:100C3000C56A16EE10EA16EE107A8E45A8BF0F466A
:100C40008645B8BF074606EE107AB8EEC66A022A95
:100C500086ED016A00F0428194ED086A9DED0E5A1E
:100C600025EE866AA5EE076AB0EE675AA6EE265A0A
:100C7000BDEEC56A16EE10EA16EE107A8E45A8BFD4
:100C80000F468645B8BF074606EE107AB8EEC66A2C
:100C9000032A86ED026A00F0218194ED0C6A9DED35
:100CA0000F5A25EE866AA5EE076AB0EE675AA6EEE1
:100CB000265ABDEEC56A16EE10EA16EE107A8E457B
:100CC000A8BF0F468645B8BF074606EE107AB8EEB5
:100CD000C66A042A86ED036A00F0008194ED106A6A
:100CE0009DED105A25EE866AA5EE076AB0EE675AAA
:100CF000A6EE265ABDEEC56A16EE10EA16EE107A7A
:100D00008E45A8BF0F468645B8BF074606EE107A47
:100D1000B8EEC66A052A86ED046A00F0DF8094ED1D
:100D2000146A9DED115A25EE866AA5EE076AB0EEAB
:100D3000675AA6EE265ABDEEC56A16EE10EA16EE02
:100D4000107A8E45A8BF0F468645B8BF074606EE07
:100D5000107AB8EEC66A062A86ED056A00F0BE80F3
:100D600094ED186A9DED125A25EE866AA5EE076A83
:100D7000B0EE675AA6EE265ABDEEC56A16EE10EA28
:100D800016EE107A8E45A8BF0F468645B8BF0746B7
:100D900006EE107AB8EEC66A072A86ED066A00F0FB
:100DA0009D8094ED1C6A9DED135A25EE866AA5EE92
:100DB000076AB0EE675AA6EE265ABDEEC56A16EE71
:100DC00010EA16EE107A8E45A8BF0F468645B8BFCA
:100DD000074606EE107AB8EEC66A082A86ED076A5C
:100DE0007CD094ED206A9DED145A25EE866AA5EE1E
:100DF000076AB0EE675AA6EE265ABDEEC56A16EE31
:100E000010EA16EE107A8E45A8BF0F468645B8BF89
:100E1000074606EE107AB8EEC66A092A86ED086A19
:100E20005CD094ED246A9DED155A25EE866AA5EEF8
:100E3000076AB0EE675AA6EE265ABDEEC56A16EEF0
:100E400010EA16EE107A8E45A8BF0F468645B8BF49
:100E5000074606EE107AB8EEC66A0A2A86ED096AD7
:100E60003CD094ED286A9DED165A25EE866AA5EED3
:100E7000076AB0EE675AA6EE265ABDEEC56A16EEB0
:100E800010EA16EE107A8E45A8BF0F468645B8BF09
:100E9000074606EE107AB8EEC66A0B2A86ED0A6A95
:100EA0001CD094ED2C6A9DED175A65EE865AE7EE3C
:100EB000055AE6EEA57AFDEEE77A17EE904AA142D2
:100EC000A8BF2146A042D8BF084607EE900AF8EE18
:100ED000E77AC6ED0B7A002A3EF4BAAF92000C49CD
:100EE0000A4822F08DFF0B4A1268002A3EF4B5AF83
:100EF0001EF058FEFEF7B1BFF0EE676AFFF7B8B814
:100F0000B0EE465AFEF703BBD067002044480020ED
:100F10000C260020446B0020B349B44AD1F8EC10F1
:100F2000126844F620608142A8BF0146B1F57A7F7D
:100F3000B8BF4FF47A7189B212F0100FABF8AA1152
:100F4000D9F8002000F0C385D20442F15580A84AA8
:100F500017687E8E7608A74CA748DBF8AC21D4ED45
:100F6000037AA0FB01018809642191FBF0F11429A7
:100F7000BDEEE77A0BEB4204A8BF142101328A428E
:100F8000CBF8AC2117EE10EAA4BF0022CBF8AC21BD
:100F90000BEB4202A4F8B0E1B2F9B02107EE102A3F
:100FA000B8EEC77A77EEC77AFDEEE77ACDED057A2F
:100FB000BDF9141081EAE172A2EBE172B24202F3D0
:100FC00026828E494FF07E520A60FEF792BFDAF811
:100FD0000830002B3EF460AF8949A1F14C009847DE
:100FE000884B1B681C077EF55CAF824CD4ED027AFF
:100FF000B2EE0E7AF0EEE76AF4EEC76AF1EE10FA9E
:1010000042D5814B1B8858073ED5804B804AB3F9A7
:101010000430BBF89E1182FB0302DB17C3EBA20373
:101020005B1A9BB218B210F1B30FBCBF03F5B473D7
:1010300018B2B328C8BFA0F5B473764AC8BF18B2B7
:10104000754B12791B78002A4FF6FF7218BF0122E8
:1010500019077EF526AF664B196810FB02F30A7E6E
:101060006E499BB212FB03F381FB03121A44DB1798
:10107000C3EB221307EE103AB8EEC77A77EEC77AC1
:10108000C4ED027AFEF70DBF604B614AB3F904303C
:1010900082FB0312DB17C3EBA203ABF89E31FEF712
:1010A00000BF1E215148FDF786FC00283FF44DA9E2
:1010B000554B1B885E063FF548A99BF8FC31A342BF
:1010C00042F058864D4B9BED800AD3ED018ADBED53
:1010D0004E5A9FED536ADFED536A20EE657A68EE53
:1010E000007AA8EE287AE5EEA87AB4EEC67AF1EE98
:1010F00010FA88BFB0EE467AB4EEE67AF1EE10FA56
:10110000F4EEC67AB8BFB0EE667AF1EE10FA88BF98
:10111000F0EE467AF4EEE67AF1EE10FAB8BFF0EEB1
:10112000667A8BED4C7ACBED4E7AFFF70EB9FDEE79
:10113000C87A3D4A17EE903A9680D380FFF700B9FF
:10114000DFED3A6AFFF775BAD9F800104F023EF5A5
:10115000A7ACFEF7A9BC9FED327ADFED326A3249C7
:10116000F4EEC77AF1EE10FA98BFB0EE677AFDEEB2
:10117000E77AB4EEE67AF1EE10FA17EE903AB8BFDD
:10118000B0EE667A012F8BED4D7A4B803FF75EA86B
:10119000FFF7D6B8B4EEC87AF1EE10FA98BFB0EE09
:1011A000478ABDEEC77AB4EEE68ADFF87CE0F1EE5E
:1011B00010FA17EE103AB8BFB0EE668A8BED4C8A83
:1011C000AEF80030002F7EF4B0AFFFF7B9B8BDEE37
:1011D000E77A154B17EE102A9A80FFF79AB8002B82
:1011E0003EF4FAA8FEF7DFB8F00E0020344A0020E3
:1011F000D43900209C370020D34D62100C00002011
:101200005C53002074390020D03900208039002040
:1012100067666666684A0020587A00208988888850
:1012200000C0F94400C0F9C4583600200000000096
:10123000BCF1000F41F0C28325EE866AD24EA5EEC6
:10124000076AB0EE675AA6EE265ABDEEC56A16EEDC
:1012500010EA16EE107A8E45A8BF0F467045C8BF3B
:10126000074606EE107AB8EEC66A012A86ED006AD5
:101270003FF434AE94ED046A9DED0D5A25EE866A76
:10128000A5EE076AB0EE675AA6EE265ABDEEC56A0D
:1012900016EE10EA16EE107A8E45A8BF0F4670457E
:1012A000C8BF074606EE107AB8EEC66A022A86ED77
:1012B000016A3FF413AE94ED086A9DED0E5A25EED7
:1012C000866AA5EE076AB0EE675AA6EE265ABDEE0C
:1012D000C56A16EE10EA16EE107A8E45A8BF0F46C4
:1012E0007045C8BF074606EE107AB8EEC66A032AF4
:1012F00086ED026A3FF4F2AD94ED0C6A9DED0F5A53
:1013000025EE866AA5EE076AB0EE675AA6EE265A63
:10131000BDEEC56A16EE10EA16EE107A8E45A8BF2D
:101320000F467045C8BF074606EE107AB8EEC66A8B
:10133000042A86ED036A3FF4D1AD94ED106A9DED69
:10134000105A25EE866AA5EE076AB0EE675AA6EE39
:10135000265ABDEEC56A16EE10EA16EE107A8E45D4
:10136000A8BF0F467045C8BF074606EE107AB8EE14
:10137000C66A052A86ED046A3FF4B0AD94ED146A9E
:101380009DED115A25EE866AA5EE076AB0EE675A02
:10139000A6EE265ABDEEC56A16EE10EA16EE107AD3
:1013A0008E45A8BF0F467045C8BF074606EE107AA7
:1013B000B8EEC66A062A86ED056A3FF48FAD94ED55
:1013C000186A9DED125A25EE866AA5EE076AB0EE00
:1013D000675AA6EE265ABDEEC56A16EE10EA16EE5C
:1013E000107A8E45A8BF0F467045C8BF074606EE67
:1013F000107AB8EEC66A072A86ED066A3FF46EAD2B
:1014000094ED1C6A9DED135A25EE866AA5EE076AD7
:10141000B0EE675AA6EE265ABDEEC56A16EE10EA81
:1014200016EE107A8E45A8BF0F467045C8BF074616
:1014300006EE107AB8EEC66A082A86ED076A3FF40F
:101440004DAD94ED206A9DED145A25EE866AA5EE09
:10145000076AB0EE675AA6EE265ABDEEC56A16EECA
:1014600010EA16EE107A8E45A8BF0F467045C8BF29
:10147000074606EE107AB8EEC66A092A86ED086AB3
:101480003FF42CAD94ED246A9DED155A25EE866A45
:10149000A5EE076AB0EE675AA6EE265ABDEEC56AFB
:1014A00016EE10EA16EE107A8E45A8BF0F4670456C
:1014B000C8BF074606EE107AB8EEC66A0A2A86ED5D
:1014C000096A3FF40BAD94ED286A9DED165A25EE9E
:1014D000866AA5EE076AB0EE675AA6EE265ABDEEFA
:1014E000C56A16EE10EA16EE107A8E45A8BF0F46B2
:1014F0007045C8BF074606EE107AB8EEC66A0B2ADA
:1015000086ED0A6A3FF4EAAC94ED2C6A9DED175A19
:1015100065EE865AE7EE055AE6EEA57AFDEEE77A25
:1015200017EE904AA142A8BF2146A042C8BF01467B
:1015300007EE901AF8EEE77AC6ED0B7ACBE4F3F7F4
:10154000B3FB049B11491A78079B072AA0EB030001
:1015500088807EF49BACF3F7A7FB0546FEF797BCAB
:10156000F3F7A2FB049A09991278084B0593401AE5
:10157000012A588000F09082072A7DF455AFF3F7D6
:1015800093FB0790FDF752BF4448002058360020D7
:10159000002A00F02181DBED563A9BED554ADBED48
:1015A000607AB9499BED5F6A91ED007ADBED534AB1
:1015B0009BED525AB54CB64EF4EEC43AF3EE045AD3
:1015C000F1EE10FA77EEA56A00F1EE8294ED025A80
:1015D00025EE645AB0EE674AA5EE064AB4EEE64A36
:1015E00034EE655AF1EE10FA48BFB0EE475A012AC0
:1015F00086ED005A00F0F08094ED065A25EE645A0C
:10160000B0EE674AA5EE064AB4EEE64A34EE655AF5
:10161000F1EE10FA48BFB0EE475A022A86ED015AA1
:1016200000F0DA8094ED0A5A25EE645AB0EE674A6B
:10163000A5EE064AB4EEE64A34EE655AF1EE10FA2B
:1016400048BFB0EE475A032A86ED025A00F0C48024
:1016500094ED0E5A25EE645AB0EE674AA5EE064A9E
:10166000B4EEE64A34EE655AF1EE10FA48BFB0EE39
:10167000475A042A86ED035A00F0AE8094ED125AC0
:1016800025EE645AB0EE674AA5EE064AB4EEE64A85
:1016900034EE655AF1EE10FA48BFB0EE475A052A0B
:1016A00086ED045A00F0988094ED165A25EE645A9F
:1016B000B0EE674AA5EE064AB4EEE64A74EE655A05
:1016C000F1EE10FA48BFF0EE475A062AC6ED055A69
:1016D00000F08280D4ED1A5A65EEE45AB0EE674A03
:1016E000A5EE864AB3EE045AB4EEE64A74EE455AC5
:1016F000F1EE10FA48BFF0EE475A072AC6ED065A37
:101700006AD0D4ED1E5A65EEE45AB0EE674AA5EEF3
:10171000864AB4EEE64A74EE455AF1EE10FA48BF36
:10172000F0EE475A082AC6ED075A55D0D4ED225A92
:1017300065EEE45AB0EE674AA5EE864AB4EEE64A94
:1017400074EE455AF1EE10FA48BFF0EE475A092AF6
:10175000C6ED085A40D0D4ED265A65EEE45AB0EEF4
:10176000674AA5EE864AB4EEE64A74EE455AF1EEB3
:1017700010FA48BFF0EE475A0A2AC6ED095A2BD094
:10178000D4ED2A5A65EEE45AB0EE674AA5EE864AD1
:10179000B4EEE64A74EE455AF1EE10FA48BFF0EEA8
:1017A000475A0B2AC6ED0A5A16D0D4ED2E5ADFF846
:1017B000FC90DFF8FC8065EEE44AE4EE867AF4EE15
:1017C000E67A77EEC57AF1EE10FA48BFF0EE477A86
:1017D000C6ED0B7AFEF73CBBDFF8D090DFF8D08087
:1017E000FEF736BBB5EEC07AF1EE10FA01F1FE82DB
:1017F000B7EE006A36EE477AC6EE076AFEF70BBD13
:10180000DFED246AFEF775BCDFED226AFEF77CBDD2
:1018100021494A79002A3DF402AF204A1278002A71
:101820003DF4FDAE0B781E499FED1E4A07EE903A3F
:101830000B88B8EE677A07EE902A06EE903AF8EE3B
:10184000E77AF8EE666A67EE277AB7EE007AC7EEB7
:10185000A63AF4EEC43AF1EE10FA88BFF0EE443A3C
:10186000F4EEC73AF1EE10FAB8BFF0EE473AFDF7E2
:10187000D8BEBBF8AA2102F57A7292B2FEF74CBB31
:10188000094A5288FEF748BBCC670020D067002089
:10189000444800200000C842583900209A370020F0
:1018A00084370020713DAA3FF8560020105C0020CC
:1018B000D0550020AB49059107EE102A084619784B
:1018C000B0F904009AED070ABBF81041B8EEC77AE8
:1018D000F7EE006A0022132986EE879ACBF80C21D6
:1018E00001F0AD82A04AA14901EB84060025CBF8A6
:1018F0000051CBF8045167EE897A92ED001AD2EDCF
:10190000053A92ED122A92ED173AD2ED091AD2ED6C
:101910000E4A92ED016A92ED064A92ED0A7AD2EDF4
:101920000F5AD2ED132AD2ED186A92ED045AD2ED75
:10193000030A69EE288A29EE088AE1EE273AA2EE28
:10194000283AE1EE884AA6EE274AE7EE085A92EDD9
:10195000167A92ED0D6A92ED021AD2ED0C1AC6EDCE
:10196000003AE2EEA86A25EE635A27EE437A92ED3A
:101970000B2AD2ED152AC6ED204AA0EEE34A26EE48
:10198000646AD2ED143A82ED054AA1EE275AF0EED0
:10199000477AE1EEE45AA2EE086AE2EEC36AE3EEA9
:1019A000A87A82ED065AC2ED0E5A82ED0F6A86EDD4
:1019B000403AC2ED176AC2ED187ACBF80851059B80
:1019C000621C02F01F029880ABF81021049BFDF707
:1019D000ADBA674B93ED006AFEF763BF654B9FEDB1
:1019E000667AD3ED087AF4EEC77AF1EE10FA00F2D7
:1019F000DC859FED627A624CD4ED037A77EE877ACC
:101A0000C4ED037AFEF770BA5E4E3378013B0D2BBE
:101A100024D8DFE813F016072407BF06F2062300D8
:101A200023007106AC0687060E005D0651064606C9
:101A30000F07554B1B78002B02F02A821A201CF04E
:101A40009BFC002842F02482504B1B78002B42F074
:101A50001F82092333700FF021F8A778012F00F0BF
:101A60008E852379012B01F05F87022B7EF478AC01
:101A70003378012B7EF474AC444B1B78002B7EF43E
:101A80006FAC0FF079FFFEF76BBCF3F70DF909901F
:101A9000FDF787BA334B0593F3F706F93C49DBF8BA
:101AA000742109680790821ACBF874010598511ABD
:101AB0008280C180FDF7BABCF0EE667AFDF782BF86
:101AC000344B9B7B002B3EF402AAFEF705BAD700ED
:101AD0003FF53AAAFEF70DBABBF88441944240F2B2
:101AE000AF859BF89C41002C40F017872A4A2B4D6C
:101AF00092ED007AD5ED007A9BF99021CBED627AD8
:101B000077EE676A012ACBED607ACBED5F6A8BEDE9
:101B1000637A02F08381069BCBF89431204A9FEDD3
:101B2000177A92ED005A8BED667A01228BF890219C
:101B3000FEF792BE0120F3F715FADBF86421069B4D
:101B40009A1AFDF7E3BA174BD8ED007A93ED007AB5
:101B5000F0EEE77AF4EEC77AF1EE10FA7DF73CACDE
:101B6000FDF734BC58360020902D0020242B002097
:101B7000406C0020686700208FC2753C00000000A8
:101B80009C370020EA330020B64A0020B74A0020E4
:101B9000984A00205C5800203C4A002090680020B1
:101BA000AC680020786C0020D4ED014A64EEC54A90
:101BB000B0EE674AA4EE864AB4EEE64A74EE654A91
:101BC000F1EE10FA48BFF0EE474A012AC6ED004A8E
:101BD0003FF402AED4ED054A64EEC54AB0EE674A62
:101BE000A4EE864AB4EEE64A74EE654AF1EE10FAC7
:101BF00048BFF0EE474A022AC6ED014A3FF4ECAD79
